:020000040800F2
:10800000808700206581000843D3000871C70008FD
:1080100041D3000899970008111B010800000000D7
:1080200000000000000000000000000099E60008C9
:108030005DB200080000000031DB00082DEE0008F2
:10804000FD1B01087F8100087F8100087F810008F7
:108050007F8100087F8100087F8100087F81000800
:108060007F8100087F8100087F8100087F810008F0
:108070007F8100087F8100087F8100087F810008E0
:108080007F8100087F8100087F8100082598000813
:108090009D9700087F810008BD9700087F81000838
:1080A0007F8100087F8100087F8100087F810008B0
:1080B0007F81000861EF00087F8100087F81000850
:1080C0007F8100087F8100087F8100087F81000890
:1080D0007F810008410C0108BD0C01088D0D0108CD
:1080E0007F8100087F8100087F8100080000000078
:1080F0000000000000000000000000000000000080
:1081000000000000000000007F8100087F8100085F
:1081100075FE000869FF00087F8100087F81000864
:108120007F8100087F8100087F8100087F8100082F
:108130007F8100087F8100087F810008ED9A000898
:108140007F810008199A0008559A00087F8100086D
:10815000DFF80CD000F078FC00480047E94901083E
:10816000808700200648804706480047FEE7FEE774
:10817000FEE7FEE7FEE7FEE7FEE7FEE7FEE7FEE7D7
:10818000C1EE000851810008202A04DB203A00FAE1
:1081900002F1002070479140C2F1200320FA03F35E
:1081A000194390407047202A04DB203A21FA02F05C
:1081B0000021704721FA02F3D040C2F12002914021
:1081C00008431946704740EA01039B0703D009E0C2
:1081D00008C9121F08C0042AFAD203E011F8013BB3
:1081E00000F8013B521EF9D27047D2B201E000F80C
:1081F000012B491EFBD270470022F6E710B513464B
:108200000A4604461946FFF7F0FF204610BD30B578
:1082100005462A460B4612F8010B13F8014B08B12C
:10822000A042F8D01CB1002802D06D1CF1E728460E
:1082300030BD421C10F8011B0029FBD1801A704789
:1082400030B504460020034600E05B1C934203D295
:10825000E05CCD5C401BF8D030BDF0B480EA010298
:10826000D40F4200B2EB410F02D20246084611463B
:108270004A0042D0C30DDDB2C1F3C752AD1A202D62
:1082800035DAC1F3160141F4000204B15242C5F1DE
:10829000200602FA06F12A411044B3EBD05F23D046
:1082A000C4B1012DA0EBC35009DCF0BC4FF000427B
:1082B00002EAC352DBB200F5000000F009BB400047
:1082C00000F1807000EBC350A0F1807040EAD170E3
:1082D000490009E0490841EAC071A0EBC35000F52C
:1082E0000000400800EBC350F0BC00F0E8BA614267
:1082F000012202EB4101001BF6E7F0BC704781F060
:108300000041AAE780F00040A7E780EA010210B52B
:1083100002F00043400022D04A001FD0010E01EBC2
:108320001261C0F35600C2F3560240F4000042F45A
:108330000002A0FB022000047F39140400D0401C7E
:1083400050EA124001D44000491EC2B20C0604EBB0
:10835000D010401C4008802A02D003E0002010BD4D
:1083600020F00100002900DA0020184310BD30B4CD
:1083700080EA010202F0004530F0004221F00040A6
:1083800013D090B1C30DD40DC2F31601C0F3160083
:10839000E41A41F4000140F400027D34914201D31B
:1083A000641C00E04900002C02DA30BC0020704759
:1083B0004FF400000023914201D3891A034340087F
:1083C0004FEA4101F7D151B1914202D14FF0004142
:1083D00005E002D24FF0010101E06FF0010103EB73
:1083E000C450284430BC00F06ABA2DE9FE4F8046E4
:1083F00081EA0300C00F0C46009021F0004123F0F9
:108400000045B8EB0200A94105D2404621469046FE
:108410001C460B46024623F00040104347D0270D70
:10842000C7F30A00C3F30A510290401A0190402892
:108430006BDAC3F3130040F4801B0098924620B11E
:108440000023D2EB030A63EB0B0B01985946C0F1F2
:1084500040025046FFF798FE06460D4650465946E4
:10846000019A00F01AFA10EB08006141002487EA33
:10847000115284EAE7731A4340D0009A62B3019A1A
:10848000012A4FEA075215DC001B61EB02014FF095
:10849000004202EA0752CDE90042001C41F580117A
:1084A00032462B4600F051FA03B0BDE8F08F40464B
:1084B0002146F9E7001B61EB0201001C41F5801326
:1084C00000185B412018A2F5001747EB030140EAB2
:1084D000D570B6196D4111E06D084FEA360645EAD0
:1084E000C0754FEA0752001B61EB0201001C41F509
:1084F000801149084FEA30000019514132462B469D
:1085000003B0BDE8F04F00F011BA0098012240001E
:108510000023D0EB020263EBE073009821464FEAA0
:10852000E074B8EB000061EB0401E9E783F000437D
:108530005BE781F0004158E72DE9FE4F81EA030433
:1085400004F0004421F0004100944FF0000B23F0B0
:10855000004350EA01045ED052EA03045BD0C3F347
:108560000A54C1F30A552C44A4F2F3340194A0FB3D
:108570000254C1F3130141F48011C3F3130343F414
:10858000801301FB024400FB034E840A970A44EA6D
:10859000815447EA8357A4FB076802958D0A05FBBF
:1085A00007854FEA932C04FB0C542705029D4FEAE4
:1085B000065847EA1637B5EB08056EEB070C870E31
:1085C000920E47EA811742EA8312A7FB0201B6EB3B
:1085D0000B0164EB00042B0D43EA0C335E1844EBF3
:1085E0001C50DA465146E7FB0201C5F313044FEA7B
:1085F0000B3343EA14534FEA0432019C43EA060367
:10860000A4F10C040294009CCDE900B400F09DF9A3
:1086100003B0BDE8F08F00200146F9E72DE9F04DE9
:1086200081EA030404F0004B21F0004514464FF0AA
:10863000000A23F0004150EA050220D054EA01026A
:108640001DD0C5F30A570246C5F31303C1F3130047
:10865000C1F30A5640F4801543F48013A7EB0608D3
:10866000101BD64608F2FD3873EB050002D308F163
:10867000010801E092185B41B8F1000F03DA002015
:108680000146BDE8F08D00204FF480110646844677
:108690000EE0171B73EB050705D3121B63EB0503F5
:1086A00006434CEA010C49084FEA300092185B413E
:1086B00050EA0107EDD152EA030012D082EA040029
:1086C00083EA0501084305D0101BAB4106D2012205
:1086D000002306E000224FF0004302E06FF00102A9
:1086E00053101AEB06004CEB085110EB0A0041EB5B
:1086F0000B01BDE8F04D00F019B970B521F0004351
:1087000003430CD0C1F30A550024D5EB040564EBF8
:108710000403D617AD1AB34102DB0020014670BD39
:10872000201841EB025170BDC10F80EAE07008448F
:10873000CA079623002100F0CBB8962300221146E9
:1087400000F0C6B80EB540F2334102910021CDE9E8
:1087500000110A460B4600F0F8F803B000BD20F007
:108760000040C10DC0F3160040F400007F2901DA7B
:1087700000207047962903DCC1F19601C84070477C
:1087800096398840704700F0004230F000400AD02F
:10879000C10D01F56071C0F3160042EA0151C20833
:1087A00040071143704700200146704701F0004325
:1087B00030B421F0004150EA010206D00A0DA2F5C2
:1087C0006072C1F31301002A02DC30BC0020704744
:1087D000440F44EAC104C100E01830BC00EBC250B1
:1087E00000F06DB8002801DBC0F10040002901DB7A
:1087F000C1F1004181427047002801DBC0F1004017
:10880000002901DBC1F100418842704730B50B46B9
:10881000014600202022012409E021FA02F59D42B0
:1088200005D303FA02F5491B04FA02F52844151E84
:10883000A2F10102F1DC30BD2DE9F05F0546002018
:1088400092469B4688460646814640241BE02846C1
:10885000414647462246FFF7A6FC53465A46C01AF1
:10886000914110D3114618462246FFF78DFC2D1A70
:1088700067EB01084F46224601200021FFF784FCE8
:1088800017EB00094E41201EA4F10104DFDC48462D
:1088900031462A464346BDE8F09F202A06DBCB1727
:1088A000203A41FA02F043EAE07306E041FA02F3AB
:1088B000D040C2F120029140084319467047002978
:1088C000A8BF7047401C490008BF20F00100704756
:1088D00010B4B0FA80FC00FA0CF050EA010404BFB6
:1088E00010BC704749B1CCF1200421FA04F411FA0C
:1088F0000CF118BF012121430843A3EB0C01CB1D50
:108900004FEA00614FEA102042BF002010BC7047C0
:1089100000EBC35010440029A4BF10BC7047401C9A
:10892000490008BF20F0010010BC704710B5141EAC
:1089300073F1000408DA401C41F1000192185B4118
:108940001A4301D120F0010010BD2DE9F04D9246EF
:108950009B4611B1B1FA81F202E0B0FA80F2203206
:108960009046FFF711FC04460F4640EA0A0041EA30
:108970000B0153465A46084313D0114653EA0100EF
:1089800019D0C8F140025046FFF70DFC05460E46CF
:10899000504659464246FFF7F7FB084305D00120F1
:1089A00004E020463946BDE8F08D0020054346EA44
:1089B000E0762C4337430A986305E40AA0EB0800ED
:1089C0000022FD0A44EA47540A3002D5002001463D
:1089D000E9E7010510196941DDE908450019694118
:1089E000BDE8F04DA2E7C1F30A52C1F3130140F212
:1089F000FF3341F480119A4202DA002001467047A9
:108A000040F233439A42A2F2334202DC5242FFF771
:108A1000CABBFFF7B9BB000030B5041E71F10004FA
:108A200004DB4FF00044404264EB0101141E73F17B
:108A3000000405DB1C464FF00043524263EB040385
:108A4000994208BF904230BD064C074D06E0E068F1
:108A500040F0010394E8070098471034AC42F6D385
:108A6000FFF77AFB1C7F01083C7F010870B58C186A
:108A700010F8015B15F0070301D110F8013B2A1132
:108A800006D110F8012B03E010F8016B01F8016B1F
:108A90005B1EF9D12B0705D40023521E0DD401F81B
:108AA000013BFAE710F8013BCB1A921C03E013F8E4
:108AB000015B01F8015B521EF9D5A142D8D3002019
:108AC00070BD0078704700002DE9F0411E4804F0A9
:108AD0007FFB1E4D0126002769791D4C884205D079
:108AE000207818B9042002F061FE88B1164804F01D
:108AF0006FFB6979884202D1207800B12770154850
:108B000004F066FBA97988420BD0607828B108E0B0
:108B10002670042009F0B6FDF1E7032002F046FEBE
:108B200058B10C4804F054FBA979884203D160780D
:108B3000002800D06770BDE8F0816670BDE8F041A4
:108B4000052009F09FBD00009C090020882300201B
:108B50003C070020A40900200029816802D041F0D0
:108B6000010101E021F00101816070470029816865
:108B700002D041F4807101E021F48071816070477E
:108B8000014600208968490700D501207047014649
:108B900000208968090700D50120704710B5426898
:108BA0000E4B0C791A400B6842EA042213434360CF
:108BB00083680B4A1340D1E9024222434C7943EACD
:108BC00044031A438260C26A097C22F47002491E7F
:108BD000C9B242EA0151C16210BD0000FFFEF0FFC0
:108BE000FDF7F1FF70B5072409290AD9C568A1F17D
:108BF0000A0606EB4606B440A543B3401D43C560D4
:108C000007E0056901EB4106B440A543B3401D43AD
:108C100005611F23072A09D2446B521E02EB820210
:108C200093409C4391400C43446370BD0D2A09D28C
:108C3000046BD21F02EB820293409C4391400C4391
:108C4000046370BDC46A0D3A02EB820293409C43F8
:108C500091400C43C46270BD816841F0080181609D
:108C600070470029816802D041F4A00101E021F49D
:108C7000A00181607047816841F004018160704704
:108C800038B590228DF8002001228DF801208DF852
:108C900002108DF803000B480024C0F8982103F05F
:108CA00031FE6D46285D03F06BFE0A20401E000475
:108CB000000CFBD1641CE4B2042CF3D303F044FE9B
:108CC00038BD00000080214208B50121082005F0D0
:108CD0003DFBC020ADF8000003208DF802001020FD
:108CE0008DF803006946054802F044FF044801215D
:108CF000C0F89C11C0F8981108BD0000000C01409C
:108D00000080214210B5084C207B18B1002060740F
:108D1000012010BD607C20B90120607405F0FCFBCF
:108D2000A060002010BD00002824002070B50121A3
:108D300092B0084605F0E6FA012140F2112005F054
:108D400005FB4FF4004005F0D3FA3920ADF84000A0
:108D500000248DF8434010A9334802F00BFF4FF474
:108D600060200B94CDE90D0401208DF831002F4EC9
:108D700004258DF830008DF83C500BA93046FFF7E4
:108D80000DFF052301220A213046FFF72BFF0523A3
:108D900002220D213046FFF725FF052303220E2175
:108DA0003046FFF71FFF052304220F213046FFF74F
:108DB00019FF1E4869464C300090801506901C48EB
:108DC0000190280207908020CDE9044020200890DF
:108DD000CDE90245C001CDE90904164C204602F058
:108DE00094F90121204602F085F901213046FFF770
:108DF000BDFE01213046FFF7AFFE3046FFF72CFFE6
:108E000034462046FFF7C3FE0028FAD12046FFF77C
:108E100032FF2046FFF7B4FE0028FAD10121204698
:108E2000FFF71FFF12B070BD001001400024014089
:108E3000500000200800024070B504460D460C208A
:108E40000CF010F82988018069684160216809B137
:108E5000626806E00121217260608060206070BD60
:108E600019468B689342FBD188602168816070BD90
:108E700010B50D4C0D49207851F8200080470B4962
:108E80002078203151F8200080472178074A01EBF3
:108E90004101C03A02EBC10151F82010002901D074
:108EA0008847207010BD0000602300205406002079
:108EB00000F00F01000900EB800001EB4000C0B2A0
:108EC000704710B5012005F04DFABDE810400020B4
:108ED00005F048BA00B50D48A1B041F20401A0F870
:108EE00005102021418000F5C371087C401C0874E6
:108EF00007A008F0DFFE20AA6946044802F022F924
:108F00000021084806F0C4FE21B000BD221F002049
:108F100073656E6420436861726765206461746183
:108F20000A0D0000DC01002010B50C4C94F86C0018
:108F3000642809D0206F0169884738B1206F8169A2
:108F4000884728B1012010BD062002E01C2000E067
:108F5000212002F039FC002010BD0000C8060020CE
:108F600000B50B48A1B041F20901A0F8051012218B
:108F7000418000F5C371087C401C087405A008F00E
:108F800099FE20AA6946024802F0DCF821B000BD33
:108F9000221F002053656E64204368617267696E0A
:108FA0006744617461200A0D0000000000B5A1B0A3
:108FB0000020ADF880000F4841F20301A0F8051031
:108FC0000D49097881720421418000F5C370017C4C
:108FD000491C017409A008F06DFE20AA69460548E5
:108FE00002F0B0F804480021503006F051FE21B0E4
:108FF00000BD0000221F00208801002073656E6400
:109000002073746174652064617461200A0D00002E
:1090100010B5242002F0BAFB0021044806F038FE07
:10902000BDE81040002001F01BBE0000942300208A
:1090300010B5124CA2B041F22100A4F80500A4F230
:1090400046404069E071010A2172010C6172000E14
:10905000A072042004F5C3716080087C401C087471
:1090600007A008F027FE20AA6946204602F06AF809
:109070000421E01D0AF076FE22B010BD221F002060
:109080000A0D7368656E676A6979696E6764612045
:109090000A0D000010B50F4CA2B04FF48150A4F897
:1090A00005005520E071AA202072022004F5C3714A
:1090B0006080087C401C087407A008F0FBFD20AA13
:1090C0006946204602F03EF80221E01D0AF04AFE01
:1090D00022B010BD221F00204F54412041434B209D
:1090E0000A0D000000B51848A1B041F20801A0F82F
:1090F000051016A100F2BE220B6816A1D362096802
:109100001163A0F1420242F8493F516000F2EA22A5
:109110009168C1730B0A03740B0C4374090E8174BC
:10912000117BC1740D21418000F5C371087C401C86
:1091300008740AA008F0BEFD20AA6946024802F0A1
:1091400001F821B000BD0000221F00205332303151
:1091500000000000574C494E4700000073656E64E4
:1091600020626D732076657273696F6E0A0D000060
:109170000549088A401C80B20882C82801D3AA2069
:1091800070470020704700006023002010B50121C7
:109190004FF0C05005F0C2F8BDE81040012004F0C7
:1091A000A7B9000070B5094D130AD2B205F5807653
:1091B00006E000BF10F8014B5C402B5D5340325D70
:1091C000491E89B2F6D242EA032070BDC07301087D
:1091D00070B5094DFF22134605F5807606E000BF05
:1091E00010F8014B54402A5D5A40335D491E89B244
:1091F000F6D243EA022070BDC0730108022101A02B
:1092000005F060B9415400000A2101A005F05AB9E7
:1092100041542B53544154453D3F000010B588B094
:10922000044620216846FEF7E7FF20216846FEF746
:10923000E3FF224606A1684608F04CFD6846FEF7AB
:10924000F8FF0146684605F03DF908B010BD000082
:1092500041542B4E414D453D25730000092101A08D
:1092600005F030B941542B4E414D453D3F000000C3
:109270000D2101A005F026B941542B554152545FF0
:109280004346473D3F0000000B2101A005F01AB9FD
:1092900041542B564552494F4E3D3F0070B5214D2C
:1092A000687801283DD1204C2078062830D2DFE8AC
:1092B00000F003130B2F1A2307221CA11D48FEF7F1
:1092C000BFFF28BB022015E00A221BA11948FEF7A8
:1092D000B7FFE8B901200DE01A491648FEF797FFDD
:1092E000B0B1042006E00B2217A11248FEF7A8FF38
:1092F00070B9052020700BE00E486060E88920817D
:109300000C480188A1F5B442A53A01D10BF0FCFD4F
:1093100000206870E881BDE8704080210548FEF7B4
:109320006BBF70BD88010020A820002041542B4F46
:109330004B0D0A00CC1B002041542B4F4B0D0A3023
:10934000333033003015002041542B4F4B0D0A3081
:10935000310D0A0010B5114C2078062819D2DFE82B
:1093600000F0030B07180F19BDE81040FFF746BFC8
:10937000BDE8104000F0F0B9BDE8104000F0B0B911
:1093800000F0D6F9064890F8760008B1012800D11F
:10939000A07010BDBDE8104000F004B8A820002067
:1093A000201500202DE9F041424E4348002596F853
:1093B000A810037C01290DD0404C4FF47A7132463D
:1093C0002186012792F87620142B0CD942B1012A6C
:1093D00008D008E00A2B01D386F8A850BDE8F08138
:1093E000857000E087708378052BF7D2DFE803F003
:1093F00004080B035500F1E7BDE8F04100F040B967
:1094000000F0FEF8E8E72D48403006F041FC012866
:10941000E4D1E08D401C80B2E085092800D9E585C3
:1094200026480021403006F033FCE08DA8B1012829
:1094300017D0022819D00328D0D0042819D0052825
:109440001BD006281DD007281FD0082821D00928A6
:10945000C4D1BDE8F04109F023BABDE8F04100F005
:10946000A3B8BDE8F041FFF735BDBDE8F041FFF717
:109470009DBDBDE8F04100F023B8BDE8F041FFF725
:1094800031BEBDE8F041FFF76BBDBDE8F04109F02A
:109490003BBABDE8F04109F0D9B9417C4B1C43749B
:1094A00014299BD905701AB1012A97D1877095E7C5
:1094B000857093E720150020A82000208801002057
:1094C00030B5A1B000202F4CADF8800041F207006C
:1094D000A4F805002C4842F21075818BC28BE17113
:1094E00001FB02F393FBF5F3090A21726272110A80
:1094F000A172E37290F82910217390F8281061731B
:109500002021A1735F21E173C27E2274C18C61743A
:10951000090AA174E274B0F809102175090A61758D
:10952000B0F80B10A175090AE175B0F801102176A9
:10953000090A6176B0F80510A176090AE176C179C9
:109540002177418A6177090AA17790F82A10E1779B
:1095500090F82B0084F820000CA008F0ABFB1A2038
:10956000608020AA6946204601F0ECFD04F5C37036
:10957000017C491C01740021094806F089FB21B0D7
:1095800030BD0000221F0020780C002073656E643F
:10959000204443444320646174610A0D00000000CC
:1095A000E001002004F082BF00B5A1B00020ADF8BA
:1095B00080000AA008F07EFB0E493A2020AA4880CD
:1095C00069460C4801F0BEFD0B48017C491C017442
:1095D00000210A4806F05CFB21B000BD73656E6493
:1095E00020686561727462656174206461746120D1
:1095F0000A0D0000221F0020A8200020D401002016
:1096000010B592B00020ADF8400040F6B8311348D4
:1096100006F03EFB01281FD1114C41F20100A4F8D5
:10962000050010A008F046FB1349A4F14200CA6EE1
:1096300040F8492F096F416010490A688260496803
:10964000C1601020608010AA6946204601F07AFDB2
:109650000021024806F01CFB12B010BDD001002012
:10966000221F002073656E64204C6F67696E206452
:109670006174610D0A00000020150020D0720108FD
:1096800010B592B00024ADF8404041F288310C484A
:1096900006F0FEFA012810D101030A48A0F80510CF
:1096A000448009A008F006FB10AA6946054801F0AD
:1096B00049FD0021024806F0EBFA12B010BD00008F
:1096C000CC010020221F002053656E642052656784
:1096D0006973746572656420646174610A0D0000C9
:1096E00010B54FF47A71104806F0D2FA012819D15A
:1096F0000D4C383CA07A20B1012804D0022807D0B4
:109700000AE0012007E00948FFF788FD022002E097
:10971000FFF7A4FD0020A072BDE810400021024820
:1097200006F0B6BA10BD0000C001002030150020C0
:1097300010B540F6B831074806F0AAFA012807D15B
:10974000FFF762FDBDE810400021024806F0A0BA14
:1097500010BD0000C401002010B54FF47A710D480F
:1097600006F096FA012814D10A4C343C607A10B104
:10977000012804D007E0FFF787FD012002E0FFF792
:1097800077FD00206072BDE810400021014806F01E
:109790007FBA10BDBC010020FEE7000000B585B017
:1097A0006A460021044800F089FD6946002009F05E
:1097B000D1FE05B000BD00000064004070B5174C3C
:1097C0004FF400752946204600F0B0FB01280CD16B
:1097D0001349204600F08FFB012802D1002009F038
:1097E00059FF2946204600F0D1F94FF480652946FB
:1097F000204600F09BFB01280FD109492046891C17
:1098000000F079FB012802D1002009F05BFF294616
:109810002046BDE8704000F0B9B970BD006400405A
:109820000200F01010B51A4C0021204600F0F6FDA1
:10983000022806D0012824D000220021084609F081
:10984000B5FE0121204600F0E9FD022806D00128DE
:1098500019D000220121002009F0A8FE0221204693
:1098600000F0DCFD022806D001280ED000220221E3
:10987000002009F09BFE2046BDE81040012100F0C9
:1098800085B90122D9E70122E4E70122EFE70000D0
:109890000064004070B58AB004F0FFFE0121092089
:1098A00004F054FD0121480604F038FD012188062A
:1098B00004F034FD504E0021304600F0B9FC701425
:1098C000ADF8200003208DF8220018204B4C8DF8B5
:1098D000230008A9204602F04DF9A014ADF820009D
:1098E00048208DF8230008A9204602F043F90024FF
:1098F00001258DF80A408DF80B5008208DF80800DE
:109900008DF80C408DF806408DF80D408DF807500D
:1099100006208DF80E40ADF804008DF80F508DF83C
:10992000095001A9304600F05DFB3548407BB0B1DD
:109930000E208DF81A008DF81B408DF81C50ADF8E4
:109940001040ADF81440ADF81240ADF81640ADF837
:1099500018508DF81D5004A800F0AAF903E0294919
:10996000002000F0B7FA01221021304600F032FB4F
:1099700041208DF800008DF801508DF802408DF8DF
:109980000350684603F0EEFC01221146304600F019
:1099900021FB01225102304600F01CFB0122910202
:1099A000304600F017FB0122D103304600F012FBD5
:1099B0000121304600F03CFC3F208DF800008DF87E
:1099C00001508DF802408DF80350684603F0CAFC40
:1099D00042208DF800008DF801508DF802408DF87E
:1099E0000350684603F0BEFC04F059FE06A008F0E0
:1099F00061F90AB0002070BD00680040000C014011
:109A0000282400200C05002063616E2032206F7036
:109A1000656E210A0000000000B50B4985B00120E9
:109A200088730A4804F078FE6A460121084800F06D
:109A300045FC9DF80900002803D16946012009F082
:109A400089FD05B000BD000028240020B4340020AA
:109A50000068004070B5214C4FF40075294620463F
:109A600000F064FA012810D11D4E2046314600F066
:109A700042FA012805D109F00DFE3146204600F0DA
:109A80006DF82946204600F081F84FF4806529469C
:109A9000204600F04BFA01281ED1114E2046B61C7C
:109AA000314600F028FA0F4A012807D00020107430
:109AB00029462046BDE8704000F068B8107C401C84
:109AC0001074094804F028FE012009F0FBFD31461E
:109AD000204600F043F8EBE770BD0000006800404E
:109AE0000200F01028240020BC34002010B51A4CCD
:109AF0000021204600F092FC022806D0012824D044
:109B000000220021012009F051FD0121204600F032
:109B100085FC022806D0012819D000220121084620
:109B200009F044FD0221204600F078FC022806D00E
:109B300001280ED000220221012009F037FD204625
:109B4000BDE81040012100F021B80122D9E701222F
:109B5000E4E70122EFE70000006800400A4A914272
:109B600002D1002181617047C1F313028B0101D53D
:109B7000C26070474B0101D502617047090101D5F0
:109B800082607047426070477000F03030B5082343
:109B900010240422B1F5007F1DD010DC202929D02B
:109BA00007DC012921D0042922D0082900D1C46072
:109BB00030BD402920D0B1F5807FF9D10BE00025E0
:109BC000B1F5004F06D008DCB1F5806F03D0B1F5D8
:109BD000006FEDD18561426030BDB1F5803F0DD0A1
:109BE000B1F5003FF8D1446030BD0549816030BD1A
:109BF000C36030BD036130BD046130BD436030BD22
:109C000001010100094910B588424FF0010101D15D
:109C10004C0601E04FF08064204604F08BFB2046A8
:109C2000BDE81040002104F085BB00000064004046
:109C300030B41446002819D000220272026042603B
:109C4000B1F5006F03D304250572416001E0027293
:109C5000016043B13CB142728372214630BC1A4666
:109C60000B30FEF7B0BA82720221417230BC7047ED
:109C700030B41446002819D00022027202604260FB
:109C8000B1F5006F03D304250572416001E0027253
:109C9000016043B13CB142728372214630BC1A4626
:109CA0000B30FEF790BA82720221417230BC7047CD
:109CB000F0B5827A012191402E4A136843F00103E6
:109CC00013602C4B1C331C688C431C60294D067B95
:109CD000294C0C35A6B92E688E432E604688C7885D
:109CE00046EA0746877A04EBC707C7F84066068846
:109CF000878846EA0746877A04EBC707C7F84466B1
:109D0000067B012E12D12E680E432E60867A0568DE
:109D100004EBC6064FEA3545C6F84056867A4568D4
:109D200004EBC6044FEA3545C4F84456114CC57AD5
:109D3000241D002D256806D00D4325600D4C058996
:109D4000143415B104E08D43F7E725688D43256091
:109D50000589012D02D125680D432560407B01282E
:109D600002D1186808431860106820F001001060E4
:109D7000F0BD000000660040006000402DE9FF419A
:109D8000064601250F460024284600F0DFFA012090
:109D90008DF80A508DF80B008DF80C00ADF8080016
:109DA0008DF80D0000254FF0040831E004EBD4706D
:109DB00020F00100201A401C012802D002281BD1EB
:109DC0000DE056F8351008EBC101090CADF8001094
:109DD00036F8351008EBC100ADF802000CE056F87B
:109DE000351008EBC101090CADF8041036F8351038
:109DF00008EBC100ADF80600641CE00707D1684617
:109E0000FFF756FF9DF80A00401C8DF80A006D1CF4
:109E1000BD42CBDBE00702D06846FFF749FFBDE853
:109E2000FF812DE9FF41804601250E46002428468A
:109E300000F08CFA01208DF80A5000218DF80B00FB
:109E40008DF80C10ADF808008DF80D000D464FF69A
:109E5000FF7736E0E01704EB907020F00300201A43
:109E6000401C012806D002280BD0032810D004285B
:109E70001BD114E038F8350007EA4010ADF80000B7
:109E800013E038F8350007EA4010ADF802000CE0A6
:109E900038F8350007EA4010ADF8040005E038F85E
:109EA000350007EA4010ADF80600641CA00707D192
:109EB0006846FFF7FDFE9DF80A00401C8DF80A0079
:109EC0006D1CB542C6DBA00702D06846FFF7F0FE66
:109ED000BDE8FF8110B50A46102118B1012805D050
:109EE000002010BD1046FFF79CFF02E01046FFF770
:109EF00045FF012010BD0246002011F4700F03D071
:109F0000926904E001207047CB0104D552680A40F1
:109F10001103F7D170470B0101D59268F7E78B0168
:109F200001D5D268F3E71269F1E70000024600208C
:109F300053690B424AD0B1F5807F3BD013DC08292E
:109F40002ED007DC012926D0022927D004293DD1B3
:109F5000D0682BE0102925D0202926D0402935D1E2
:109F60001069102130E0B1F5004F2BD00BDCB1F5BA
:109F7000007F22D0B1F5806F22D0B1F5006F25D1DE
:109F80009069702120E0B1F5803F11D0B1F5003F1C
:109F90001CD15068E5E790680D4915E0D06802E0F3
:109FA000D068DEE7106903210EE0106908210BE09C
:109FB0005068FBE79069012106E09069022103E007
:109FC000906900E05068042100F0C4BD70470000B3
:109FD00001010100002A426901D00A4300E08A43DE
:109FE0004261704710B50368002223F0020303604A
:109FF000036843F0010303604FF6FF7300E0521C57
:10A000004468E40701D19A42F9D14268D2073ED0B0
:10A010008A79012A02683CD022F080020260CA7963
:10A02000012A026838D022F0400202600A7A012A2E
:10A03000026834D022F0200202604A7A012A0268C3
:10A0400030D022F0100202608A7A012A02682CD0F5
:10A0500022F008020260CA7A012A026828D022F09F
:10A06000040202608A78CC78920742EA04620C7992
:10A0700042EA04424C79098842EA0452491E0A43E2
:10A08000C261016821F001010160002114E000209B
:10A0900010BD42F08002C1E742F04002C5E742F045
:10A0A0002002C9E742F01002CDE742F00802D1E7F2
:10A0B00042F00402D5E7491C4268D20701D0994218
:10A0C000F9D14068C007E2D1012010BD10460B0055
:10A0D00001D00021184770470846D1B2C0B20AF03B
:10A0E00063BA000070B58AB00121052004F02EF992
:10A0F0000121480604F012F9474E0021304600F0D5
:10A1000097F8B014ADF8200003208DF82200182035
:10A11000424C8DF8230008A9204601F02BFDE014E5
:10A12000ADF8200048208DF8230008A9204601F052
:10A1300021FD00248DF81A4001258DF81B500C20BC
:10A140008DF818008DF816408DF817400920ADF8ED
:10A15000140007948DF8195005A93046FFF742FF07
:10A160008DF80E408DF80F408DF81050ADF804407A
:10A17000ADF80840ADF80640ADF80A40ADF80C4027
:10A180008DF8115001A8FFF793FD012202213046FE
:10A19000FFF720FF14208DF800008DF801508DF896
:10A1A00002408DF80350684603F0DCF801221146A6
:10A1B0003046FFF70FFF012251023046FFF70AFF3A
:10A1C000012291023046FFF705FF0122D1033046FC
:10A1D000FFF700FF0121304600F02AF813208DF828
:10A1E00000008DF801508DF802408DF8035068464C
:10A1F00003F0B8F816208DF800008DF801508DF8A6
:10A2000002408DF80350684603F0ACF804A007F054
:10A2100051FD0AB0002070BD0064004000080140FC
:10A2200063616E2031206F70656E210A00000000AE
:10A2300000234FF6FF7221B1012917D0022924D043
:10A240003AE0016821F0020141F00101016000E003
:10A25000521E416801F00301012901D0002AF7D103
:10A26000406800F00300012823D124E0016821F0B8
:10A270000301016000E0521E4168890701D0002AF5
:10A28000F9D14068800714D115E0016821F001017F
:10A2900041F00201016000E0521E416801F003013B
:10A2A000022901D0002AF7D1406800F003000228FB
:10A2B00001D0002300E001231846704710B500EBE1
:10A2C0000113D3F8B04114F004041472D3F8B04170
:10A2D00034D0E408C2F80440D3F8B04104F00204DA
:10A2E0005472D3F8B44104F00F049472D3F8B4411B
:10A2F000240AD474D3F8B841D472D3F8B841240AEC
:10A300001473D3F8B841240C5473D3F8B841240E15
:10A310009473D3F8BC41D473D3F8BC41240A1474A9
:10A32000D3F8BC41240C5474D3F8BC311B0E937485
:10A3300039B1016941F02001016110BD640D146063
:10A34000CAE7C16841F02001C16010BD09490A682F
:10A3500042F001020A600A6843F60E739A430A60EB
:10A360000A6842EA00200860086820F001000860DE
:10A37000704700000066004030B502460020936838
:10A380005B0108D49068000101D5012003E09068CA
:10A39000C00037D5022002EB0012D2F8803103F062
:10A3A0000103C2F880310B7A73B3D2F880414D6853
:10A3B0001C434B7A43EAC5031C43C2F880418B7AA5
:10A3C00003F00F038B72D2F8843123F00F03C2F82D
:10A3D0008431D2F884318C7A2343C2F88431CB7A29
:10A3E000CC6843EA0423C2F88831CB7B096943EA8D
:10A3F0000121C2F88C11D2F8801141F00101C2F89C
:10A40000801130BD042030BDD2F880314C7A234316
:10A410000C8843EA4453C2F88031D0E7002221B1CE
:10A42000012905D0022906D112E08268114801E015
:10A430008268114802401149501A8A4214D00ADC3D
:10A44000A2B16FF0806010180FD002280CD10FE07D
:10A4500082680B48EEE7B0F5007F09D00949401843
:10A4600003D0B0F5003F03D00020704702207047B2
:10A4700001207047030000040003000800010008E9
:10A48000000003100001FFF770B512488188828830
:10A49000A0F1300400253038616AC06971B13C21F7
:10A4A000B0FBF1F0C000FEF748F90B49FDF75FFF84
:10A4B0000A4908606562E561256270BDA16A3C29B0
:10A4C00004D2491C1044A162E06170BD0120C4E9BE
:10A4D000090570BD5000002000401C46380C0020CB
:10A4E000054810B590F8210008B1012010BD2920C1
:10A4F00001F06AF9002010BDFC0C002010B50178B5
:10A50000427801EB0221144AA2F81B108178C3782B
:10A5100001EB032109B2B1F57A6F02DDA1F57A6191
:10A5200001E0C1F57A6109B20B4C8BB23D34A2F85F
:10A530001D300A2902DBA4F8073002E00021A4F84C
:10A5400007100179437901EB032122F81F1F80795D
:10A550009070012010BD0000FC0C002000B50246E8
:10A560000078FEF7A5FC134BD8725078FEF7A0FCDC
:10A5700018739078FEF79CFC5873D078FEF798FC1F
:10A5800098731079FEF794FCD8735079FEF790FC1D
:10A5900018749079FEF78CFC064958744839D1F844
:10A5A000532041F8012FB1F856208A80887101208C
:10A5B00000BD0000FC0C002010B508A007F07AFBDD
:10A5C00000F0A0F900F074F900F092F902F06CFFCD
:10A5D000044802F00EFE012010BD000054310D0AA7
:10A5E000000000008409002010B502A007F062FB03
:10A5F000022010BD5431300D0A00000010B502A039
:10A6000007F058FB062010BD5431310D0A00000040
:10A6100010B502A007F04EFB062010BD5431320DDC
:10A620000A00000010B504A007F044FB02F01CFF74
:10A6300000F068F9002010BD5431330D0A0000000D
:10A6400010B503A007F036FB00F05CF9012010BD47
:10A650005431340D0A00000010B509A007F02AFBA0
:10A6600002F002FF084C01202072084802F0C1FDF0
:10A670000020E071064802F09CFD072010BD00009C
:10A680005431350D0A000000882300207C09002089
:10A690006C09002010B509A007F00CFB094802F076
:10A6A00088FD00F025F902F0FFFE07490020087040
:10A6B000064908700649087010BD00005431360D77
:10A6C0000A00000084090020210000202000002052
:10A6D0000C0B002010B503A007F0ECFA02F0E4FE2A
:10A6E000022010BD54320D0A0000000010B502A077
:10A6F00007F0E0FA032010BD54330D0A00000000FB
:10A70000044810B50021C174018203A007F0D2FAF9
:10A71000042010BD6023002054340D0A0000000006
:10A7200010B502A007F0C6FA052010BD54350D0A79
:10A730000000000010B502A007F0BCFA062010BD12
:10A7400054360D0A0000000010B506A007F0B2FA5A
:10A7500006490020487100F0D5F802F085FE00207F
:10A7600010BD000054370D0A0000000074230020C3
:10A7700010B502A007F09EFA022010BD54380D0A51
:10A780000000000010B502A007F094FA022010BDEE
:10A7900054390D0A0000000010B5252000F0F6FF26
:10A7A0000021044805F074FABDE81040012000F0D3
:10A7B00057BA00009823002010B5154C606A002895
:10A7C00001DA14A01CE0606A400001D515A017E072
:10A7D000606A800001D518A012E0606AC00001D54F
:10A7E0001AA00DE0606A000101D51BA008E0606AB4
:10A7F000400101D51CA003E0606A800102D51DA0C4
:10A8000007F058FA606A40F08070606210BD000086
:10A8100000100240B5CDB9A6BAC4B8B4CEBB0D0A7B
:10A8200000000000B4B0BFDABFB4C3C5B9B7B8B454
:10A83000CEBB0D0A00000000B6C0C1A2BFB4C3C5A4
:10A84000B9B7B8B4CEBB0D0A00000000C8EDBCFE1D
:10A85000B8B4CEBB0D0A0000C9CFB5E72FB5F4B52B
:10A86000E7B8B4CEBB0D0A00D2FDBDC5B8B4CEBBAF
:10A870000D0A0000424F52B8B4CEBB0D0A000000D2
:10A8800010B5094802F095FC012000F0E8FC0748EB
:10A8900002F0AFFC4FF4FA7000F0E1FCBDE81040AC
:10A8A000024802F086BC0000C4090020CC09002048
:10A8B00010B502F0AFFB4FF4FA7000F0D0FC02F0DC
:10A8C000C5FB044901204871BDE8104002A007F013
:10A8D000F1B9000088230020434C4F53455F3132CB
:10A8E00056506F7765725265616C790D0A000000F1
:10A8F000024900200872024802F05BBC8823002055
:10A900007C090020024900208871024802F051BCF5
:10A91000882300205C090020024900208871024839
:10A9200002F047BC882300205C09002030B50C46AB
:10A93000054600F005F8024628190088504030BD51
:10A9400070B504464FF6FF7048F2050503460EE069
:10A9500014F8012B80EA02200022491E060403EAB3
:10A96000400000D56840521CD2B2082AF6D3002914
:10A97000EED170BD0A48026FB0F84630B0F848001A
:10A98000118801EB81014900B1FBF3F1494201EB70
:10A9900081014FF2600303EB41010844508070478E
:10A9A000C80600200120704770B5124D124C28785F
:10A9B000072811D011480069804702280CD00020D8
:10A9C00020702878801E042801D8012020700620DD
:10A9D00000F0ECFE48B901E00320F1E728780628F2
:10A9E00005D1074802F0F4FB08B902202070207856
:10A9F00070BD0000602300208C050020580000205E
:10AA0000A40900200088322801D8012070470020C6
:10AA10007047000010B506480649C08F898A8842F1
:10AA200004D2282000F0D0FE002010BD012010BD6F
:10AA3000C8060020FC0C00201D4810B5007920B18C
:10AA4000012807D002280CD108E01121194801F093
:10AA50002FF806E0174801F057F802E0112001F046
:10AA600063F8134832213038044605F011F9012803
:10AA700005D108F089F80021204605F009F90E49B2
:10AA8000886BC20612D520F0100088630848FA21AE
:10AA90002838044605F0FCF8012807D108F0CEFA62
:10AAA0002046BDE81040002105F0F2B810BD0000BE
:10AAB00074230020B52C0108FC0C002070B5204D3B
:10AAC0000026A889401C80B2A8810A2802D3AE8142
:10AAD00001F0EAFA1B491C4CA1F1FC008A88130A18
:10AAE00000F8E83F42708A790274C9794174688934
:10AAF000401C80B26881642814D36E81134D94F891
:10AB00002800297881420DD0287008212846FFF7B7
:10AB100017FF2872000A687200230A2229460C488F
:10AB200000F062FD6078012808D1A078012805D1E5
:10AB30006670A67001F016FE0120607170BD000005
:10AB4000100B0020CC350020A0440020F64400204B
:10AB500000450020024600200A4200D00120704734
:10AB6000034900200978490700D5012070470000FB
:10AB7000CC350020034900200978890700D5012041
:10AB800070470000CC350020034600201AB18B42EC
:10AB900000D0012070478B42FBD070470349002052
:10ABA000497A002900D0012070470000CC350020F0
:10ABB0000021012801D0032800D101210846704757
:10ABC0000021012805D0022803D0042801D00A283A
:10ABD00000D101210846704701460020090600D433
:10ABE00001207047024600208A4200D101207047B0
:10ABF0000120704770B517490020174E08601439BE
:10AC00000446C87004EBC40006EB40050C35102167
:10AC10002846FDF7F1FA10212846FFF791FE287427
:10AC2000000A641CE4B26874122CEBD30A494FF496
:10AC3000A2740C3122460D4601F5A270FDF7C3FA4D
:10AC4000002322462946054800F0CEFCBDE87040AE
:10AC500006F0ECB9240B0020E435002089450020E3
:10AC6000024A012110440172704700009423002021
:10AC7000044810B500698047022801D0002010BDAB
:10AC8000012010BD5800002070B58F4805210646F0
:10AC900003F030FD8D4C002518B12573304603F0CC
:10ACA0003BFD894805210830064603F023FD18B115
:10ACB000A573304603F030FD834805211030064669
:10ACC00003F018FD18B12574304603F025FD804CC3
:10ACD000E06880477F49884203DA2A2000F066FD59
:10ACE00040B3E06880477C49884206DB2A2000F0B8
:10ACF0005DFD10B12A2000F049FDE06880477749EA
:10AD0000884203DD322000F051FDB8B1E068804791
:10AD10007349884206DC322000F048FD10B1322031
:10AD200000F034FD6F4C94F84C00C0F30100032890
:10AD300008D00AE02A2000F047FDDEE7322000F0CC
:10AD400043FDEFE72E2000F03FFD606CC0F3816013
:10AD5000032802D10B2000F037FD606CC0F30170B6
:10AD6000032802D12B2000F02FFD606C800F0328F8
:10AD700002D12C2000F028FD606CC0F301400328B4
:10AD800002D12D2000F020FD606CC0F3815003281B
:10AD900002D10C2000F018FD94F84400C0F300002C
:10ADA00010B10D2000F010FDB4F84400C0F3813064
:10ADB000032802D10E2000F007FD94F84400C0F3F0
:10ADC000800010B10F2000F0FFFC94F84400C0F3A5
:10ADD000C00010B1102000F0F7FC94F84400C0F35C
:10ADE000001010B1112000F0EFFC94F84400C0F303
:10ADF000401010B1122000F0E7FC94F84400C0F3BA
:10AE00008110032802D1132000F0DEFC206CC0F377
:10AE1000806010B1142000F0D7FC206CC0F30060FB
:10AE200010B1152000F0D0FC206CC0F3406010B1D0
:10AE3000162000F0C9FC206CC0F3007010B1172080
:10AE400000F0C2FC206CC00F02D0182000F0BCFC47
:10AE5000206CC0F3404010B1192000F0B5FC206C0C
:10AE6000C0F30150032802D11A2000F0ADFCB4F861
:10AE70004000C0F3C02010B11B2000F0A5FC94F8E6
:10AE80005C00C0F3800010B11D2000F09DFC94F820
:10AE90005C00C0F3C00010B11E2000F095FC94F8D7
:10AEA0005C00C0F3401010B11F2000F08DFC94F83E
:10AEB0005C00C0F3C010002804D0BDE87040202022
:10AEC00000F082BC70BD0000AC34002028240020BB
:10AED000580000200000084100001041000094418B
:10AEE00000009041B022002070B51949194800F0C7
:10AEF00079FD0546174818490C3000F073FD1649D6
:10AF0000164C1D39B1F81D10B9B1012D05D0B1F5A0
:10AF1000A07F12D9032804D00FE0012000F054FCD8
:10AF200012E00321204603F0E5FB30B1052000F0DC
:10AF30004BFC204603F0F0FB06E0204603F0ECFB60
:10AF4000032000F033FC08B1002070BD012070BD6B
:10AF5000440C0020B8230020190D00209C34002050
:10AF600010B52A2000F022FC08B9FDF7ADFD114C08
:10AF700060688047552803DB302000F025FC06E0A0
:10AF800060688047502802DC302000F0FFFB0A4850
:10AF900090F90000552804DBBDE81040312000F096
:10AFA00013BC502804DCBDE81040312000F0EEBB9B
:10AFB00010BD000058000020882300200A4810B56A
:10AFC0000078002448B1411E032901D8012404E07F
:10AFD000052801D0072800D1022400F0C9FB00B1E8
:10AFE0000324204610BD00006023002010B541F26C
:10AFF000883421460D4804F04BFE012808D00B4848
:10B000002146001F04F044FE012806D0012010BD97
:10B01000252000F0D9FB012003E0242000F0D4FB20
:10B02000002003F0A9FD002010BD0000982300209F
:10B03000007870472DE9FE4F01A9264800F0C4FAB8
:10B04000254D264E264FDFF89C80DFF89C9000248B
:10B0500036F8140000F0A2FFFF2813D037F81000D4
:10B0600001992844029039F8140038F814B00844C3
:10B0700082465946FFF75AFC20B95A465146029873
:10B08000FDF7A1F8641CE4B2092CE1D306F0A6F99F
:10B09000104869460A3800F097FA08210098FFF72F
:10B0A00045FC124938B1002081F82900C87081F8A8
:10B0B0002800BDE8FE8F00980D4A0078107081F8D6
:10B0C00028000328F5D30A2081F829000120C87040
:10B0D000EFE700000A450020D03400203478010852
:10B0E000D47701085878010846780108A044002068
:10B0F000F64400200029016802D041F0010102E07D
:10B100004FF6FE7211400160704730B5036847F694
:10B11000F07293430C6A8A682243D1E904452C43B8
:10B1200022438C692243CC6922434C6A22438C6AB5
:10B1300022431A430260CA6842600A688260496812
:10B14000C16030BD70B50C46050033D08CB3688843
:10B15000A52121705A2161701930A070000AE07099
:10B1600020202071601D10221349FDF72CF868790A
:10B170006075B5F805001726000AA0756A88022ACE
:10B1800007D304F11700E91DFDF71DF8A878173063
:10B19000C6B231462046FEF71BF8A055761CF1B228
:10B1A000000A6054491CC9B22046FEF7FBF9012091
:10B1B00070BDFFE70020FBE720150020F8B56946C9
:10B1C000214800F001FA1226204F0024009804EBD9
:10B1D000C40500EB4500B11EFFF7A8FB88B9009835
:10B1E000324600EB450107EB45000C30FCF7EBFF66
:10B1F0000098324600EB4501154800EB4500FCF78E
:10B20000E2FF07EB4500007B092805D11148012129
:10B21000A14002680A430260641CE4B2122CD5D338
:10B2200006F0F2F80B494FF4FA701439888018319F
:10B230004FF0FF30A1F1150208600749A1F5227017
:10B2400003F078FDF8BD000089450020E4350020BA
:10B2500034370020240B002078380020704710B5C8
:10B26000044606E0142006F0DDFC01F0ABFC641E91
:10B27000A4B2002CF6D110BD70B5044600F0A2FEB9
:10B280000646FF2822D0204600F088FEFF281DD069
:10B290000F49114A0C5C0F4932F81000451821463D
:10B2A0002846FFF74DFB2855641C000A28550B481B
:10B2B000621C30F816100A48081803D000232946EB
:10B2C00000F092F9BDE8704006F088B870BD00004B
:10B2D000FA770108D0340020D477010846780108B5
:10B2E0000A4500202DE9F8411C46002688468DF8C5
:10B2F0000060217815464A1C592322706B5421782E
:10B30000194F4A1C227068546A463946404603F079
:10B3100011FD22E037F816002178020A13484B1C71
:10B3200050F8220023704FEA104C05F801C0217834
:10B330004FEA102C4B1C237005F801C021784B1CE0
:10B340002370685402EBC20108EB41004278207878
:10B35000411C2170761C2A54F6B29DF800008642EA
:10B36000D8D30020BDE8F881783800206477010840
:10B370002DE9F0434FF05908DDE90754002694F811
:10B3800000C04FF001090CF10107277005F80C808F
:10B39000277807F1010C84F800C0E855224F21F00E
:10B3A0007F4000BF57F826C0604536D120784FEA6D
:10B3B000114C471C277005F800C020784FEA112C6B
:10B3C000471C277005F800C02078471C27702954B7
:10B3D00006EBC601267813F81170701C2070AF556B
:10B3E000012A01D0FF2A1CD103EB41014FF00009D3
:10B3F000487BB0B120780123421C22702B54227864
:10B400000823501C2070AB542078891C284403F07A
:10B410004DFC21780844207003E0761CF6B2122E11
:10B42000C0D34846BDE8F08364770108524B10B59D
:10B43000524A18781168C40602D541F0200101E093
:10B4400021F0200111608106116802D541F0400110
:10B4500001E021F0400111604106116802D541F080
:10B46000800101E021F080011160000602D541F465
:10B47000807001E021F4807010605878C107116875
:10B4800002D041F4007101E021F4007111608107E4
:10B49000116802D541F4806101E021F480611160FE
:10B4A0004107116802D541F4006101E021F4006117
:10B4B00011600107116802D541F4805101E021F4C7
:10B4C00080511160C106116802D541F4005101E0BC
:10B4D00021F4005111608106116802D541F48041C8
:10B4E00001E021F4804111604106116802D541F468
:10B4F000004101E021F400411160000602D541F451
:10B50000803001E021F4803010609878C007106826
:10B5100002D040F4003001E020F400301060FFF76A
:10B520003DFB28B3587A082803D3106840F0100078
:10B530001060FFF733FB002819D110481438C18878
:10B54000491C8BB20021C380C82B04D9136843F077
:10B5500001031360C18003895B1C9BB20381B3F5B7
:10B56000967F04D9136843F002031360018110BD74
:10B57000106820F01000DBE7CC350020240B002001
:10B5800030B50C460F4A00EBC00102EB41030C4DF5
:10B590000C33122813D21878A0420FD0092C0DD1E9
:10B5A000184603F0B9FB587818B92878401C287061
:10B5B0005870587BFF2801D0401C58731C7030BD58
:10B5C000130B0020E4350020064A824205D07F3A62
:10B5D000824202D00A3A824202D101200A607047B8
:10B5E000002070478945002010B50BF02FFB01208B
:10B5F00010BD000001A006F05DBB00004556454EA1
:10B60000545F410D0A00000070B515A006F052FB12
:10B61000164D00244FF4FA766879D0B101F024FF7A
:10B620003046FFF71CFE6879B0B101F01DFF3046CF
:10B63000FFF715FE0E4801F0CBFD697988420ED068
:10B64000641CE4B2052CE7D3BDE87040042000F090
:10B65000BBB8FFF72DF9E3E7FFF72AF9E7E770BD7D
:10B660004556454E545F41430D0A00008823002093
:10B670009C09002001A006F01DBB00004556454E68
:10B68000545F420D0A00000001A006F013BB000049
:10B690004556454E545F430D0A00000070B516A094
:10B6A00006F008FB174D00244FF4FA76A87901281C
:10B6B0001BD001F00DFF3046FFF7D1FDA87901281E
:10B6C00016D001F005FF3046FFF7C9FD0E4801F026
:10B6D0007FFDA97988420ED0641CE4B2052CE5D325
:10B6E000BDE87040032000F06FB8FFF715F9E2E7FE
:10B6F000FFF712F9E7E770BD4556454E545F4443E6
:10B700000D0A000088230020A409002010B5102194
:10B710000548FCF771FD05490020086008710839EB
:10B720000860486010BD0000182400202C0800208C
:10B7300070B50A4C052604F1080520686168884246
:10B740000BD0295C06A006F0B5FA2068401C90FBDF
:10B75000F6F106FB11002060F0E770BD2408002020
:10B76000457272204E554D2069732025640D0A00E4
:10B77000054900200A5C0AB101207047401CC0B294
:10B780001028F7D3002070471824002010B5034676
:10B7900000F00CF830B1DC08184600F079F90249E5
:10B7A00000200855012010BD18240020C20800F018
:10B7B00007010448805C01228A40104000D001202B
:10B7C000704700001824002010B50346FFF7EEFF75
:10B7D000A0B90B4AA2F10801486813540522401C85
:10B7E00090FBF2F402FB140048600649D80803F00D
:10B7F00007030A5C01249C4022430A54012010BD27
:10B800002C080020182400200149C860704700005F
:10B810000020024070B50D4E0546304600F088F815
:10B82000042811D10A4C206940F0020020616561B2
:10B83000206940F040002061304600F079F821692D
:10B8400041F6FD721140216170BD0000FFFF0F0045
:10B850000020024008490420CA68D20701D0012014
:10B860007047CA68520701D502207047C968C906E7
:10B87000FBD5032070470000002002400248016908
:10B8800041F080010161704700200240F0B506469A
:10B890004FF6FF770D46384600F04AF804280DD1E0
:10B8A000074C206940F0010020613580384600F0E7
:10B8B0003FF8216941F6FE7211402161F0BD0000A0
:10B8C000002002402DE9F841064600204FF6FF77A0
:10B8D00000900D46384600F02BF8042817D10D4C87
:10B8E000206940F0010020613580B846384600F0FC
:10B8F0001FF841F6FE77042806D1B61C280C0096E6
:10B900003080404600F014F8216939402161BDE8DB
:10B91000F8810000002002400348024941600349C9
:10B92000416070472301674500200240AB89EFCD9D
:10B9300000B50346FFF78EFF03E000BFFFF78AFF65
:10B940005B1E012803D0002B00D1052000BD002B79
:10B95000F4D1FAE70A290FD801EB4102074903881D
:10B9600021F8223001EB820183788B70C278CA7093
:10B9700002790A718068886070470000A023002067
:10B9800000B501211648FFF7E5FF154802210C30EC
:10B99000FFF7E0FF124803211830FFF7DBFF1048E4
:10B9A00004212430FFF7D6FF0D4805213030FFF782
:10B9B000D1FF0B4806213C30FFF7CCFF0848072198
:10B9C0004830FFF7C7FF064808215430FFF7C2FF91
:10B9D0000348092160305DF804EBFFF7BBBF0000AE
:10B9E000B807002010B504468268084690472179C0
:10B9F0000022814202D0A27020710CE0E3788342E1
:10BA000001D1A27007E0A078401CC0B2A0702288CB
:10BA1000904200D3E170E07810BD00002DE9F047BE
:10BA200081461A48184C00278088401E86B204EBD5
:10BA3000C60041684846FCF7D5FE04D34846616815
:10BA4000FCF7DAFE18D240F6FF70BDE8F087B819AF
:10BA5000450804EBC5084846D8F80410FCF7CCFEAE
:10BA600002D26D1EAEB207E04846D8F80410FCF7CB
:10BA7000B9FE06D26D1CAFB2B742E8D934F937002F
:10BA8000E3E734F93500E0E7546D010820000020B9
:10BA9000064A0021535C834202D100205054704773
:10BAA000491CC9B20529F5D3704700002C080020B5
:10BAB0002DE9F041074612480E466421804604F005
:10BAC000E7F800250F4C012806D1B847E5720021A0
:10BAD0004046656004F0DCF8E07A11280ED1607C05
:10BAE000B0420BD1606841F6EC41B1EB104F05D18B
:10BAF00003490120E572403165600871BDE8F081BD
:10BB0000342300204C0D002010B501460220884748
:10BB100004490220087103480021BDE810403C3868
:10BB200004F0B6B87423002070B50F4900240F4DFF
:10BB3000CA7A0F4E132A0CD14A7C824209D1486836
:10BB400041F6EC42B2EB104F03D1CC724C602C7139
:10BB5000B463064832213C3804F09AF8012801D138
:10BB60002C71B46370BD00004C0D002074230020C4
:10BB7000FC0C0020F0B5CA78002502F00F03D206B5
:10BB800001D58A7813430A784FF00F0E12F0FF0F99
:10BB90004FF001021CD004680F8802FA05F6374006
:10BBA000B74211D14FEA850C0EFA0CF724EA0707C9
:10BBB00003FA0CF43C43CF78282F02D0482F02D050
:10BBC00002E0466100E006616D1C082DE4D30460CC
:10BBD0000C88FF2C1ED944685FF0000606F10807A8
:10BBE00002FA07F50F882F40AF420FD14FEA860CBB
:10BBF0000EFA0CF7BC4303FA0CF73C43CF78282F1E
:10BC000000D14561CF78482F00D10561761C082E00
:10BC1000E4D34460F0BD0000F0B5144C002801DA14
:10BC2000E36900E06368420D120185B2C0F3015779
:10BC30009540C0F30346032F05D0C2020AD5032264
:10BC4000B240934307E023F07062636823F07063AF
:10BC5000636002E0AB4343F0706201B12A43002805
:10BC600001DAE261F0BD6260F0BD00000000014059
:10BC70000246002092680A4200D0012070474161CC
:10BC800070470161704700787047000070B50C4C38
:10BC9000206980470B4D02280BD10B480321064633
:10BCA00002F028FD28B1304602F036FDA06880473A
:10BCB00004E020698047022801D00020287070BD70
:10BCC0005800002088230020A43400200C4810B520
:10BCD00040880B4A01211C3A05F04AFF08483038D9
:10BCE0004069FCF750FD02460B4606480649FCF742
:10BCF00095FCFCF75BFDFFF791FE0449488110BD00
:10BD0000500000209A99999999991340380C002075
:10BD10007CB5002328A40093246801946D4601ACEF
:10BD2000012825D0C85CE65C7040E8545B1CDBB29F
:10BD3000042BF7D39DF800109DF8010001F00F04CB
:10BD4000034664F31F13137003099DF8020043EACE
:10BD5000001353709DF8033003F0F00444EA101010
:10BD6000907003F00F0040EA1110D07000207CBDED
:10BD7000C85CE65C7040E8545B1CDBB2042BF7D374
:10BD80009DF801109DF8000001F0F00343EA001354
:10BD900013700B019DF8021043EA1113537001F068
:10BDA000F0039DF8031043EA111301F00F019370A3
:10BDB00061F31F10D9E700009023B02170B505464C
:10BDC00005F01AF94443601C01D01CB105E06FF086
:10BDD000A90402E005F010F904462C70200C6870EC
:10BDE000200AA870EC70002070BD0000FEB500268F
:10BDF00004468DF8086053783D480D460B2974D2EF
:10BE0000DFE801F0730606596073717373730600FF
:10BE10000A4602A9204600F0F9F802004FF0590046
:10BE20004FF0090115D18DF8086020709DF80820A9
:10BE3000521CD2B28DF80820A5549DF80820521C3F
:10BE4000D2B28DF80820A1549DF80820521C8DF81C
:10BE50000820012D49D18DF8086020709DF8080058
:10BE6000401CC0B28DF8080025549DF80800401C05
:10BE7000C0B28DF8080021549DF80800401CC0B2E3
:10BE80008DF8080026549DF80800401CC1B21848DF
:10BE90008DF808100C38C27A62549DF80810491CBD
:10BEA000C9B28DF80810807A60549DF80800401CD3
:10BEB0008DF8080019E0014602AB22462846FFF73C
:10BEC00011FA12E063F31741937863F30F21D378EB
:10BED000127963F3070102ABCDE90043034628461C
:10BEE000FFF746FA08B18DF808609DF80800FEBD1E
:10BEF000F035002070B516490324164B91F82C201C
:10BF000091F82B10144D02EB01218AB262210170CD
:10BF1000110A41708270002135F81160964203D0F9
:10BF2000491CC9B21329F7D313290ED0022C0AD009
:10BF30000A4A2044555C0A4A32F811102A4619442C
:10BF4000FCF741F92C44204670BD0224FBE70000B9
:10BF5000A0440020D03400200E780108FA770108B0
:10BF6000D477010800B5FEF7FBFD0B4A00281068E6
:10BF700002D040F0080001E020F008001060FEF759
:10BF8000F9FD0028106802D040F0040001E020F024
:10BF90000400106000BD0000240B0020024610B514
:10BFA000FF20074B002100BF33F81140944201D11C
:10BFB000084610BD491CC9B21329F5D310BD0000B5
:10BFC0000E780108024610B5FF20074B002100BF84
:10BFD00033F81140944201D1084610BD491CC9B242
:10BFE0000929F5D310BD000034780108007A7047A4
:10BFF000007970470148B0F90A007047380C0020FA
:10C00000533530385F444355323430312DE9F043F5
:10C01000224C002759256781057042700925894601
:10C02000857039465FF0030501EBC10604EB460C51
:10C030009CF80C601E4203D19E4201D00A2A23D1F3
:10C04000174E3668CE40F6071ED066890127761C4B
:10C050006681144E56F821804FEA184800F8058092
:10C060006D1C36F82180EDB24FEA182800F80580E3
:10C070006D1CEDB216F8216046556D1CEDB29CF8B2
:10C080000C6046556D1CEDB2491CC9B21229CBD3C8
:10C0900089F800503846BDE8F0830000E435002000
:10C0A000280B0020647701082DE9F0412F4DA88866
:10C0B00018B1401EA880BDE8F081FFF753FFFFF7DD
:10C0C000B5F92B4890F827000028F4D12748294FCC
:10C0D00014300024D0F8006026FA04F0C00701D024
:10C0E000092106E004EBC40007EB4000007B20F0D0
:10C0F00001012046FFF744FA641CE4B2122CEBD392
:10C100002878122600EBC00007EB40041A4F14F801
:10C110000C1F17F81000814214D010212046FEF7A2
:10C120000FFC2074000A60742878217800EBC002AC
:10C13000002307F812101149324606FB0010214671
:10C14000FFF752FA2878401CC1B20020297012294A
:10C1500000D328706978491CC9B269706429AAD3D0
:10C160006870BDE8F04105F04FB90000100B0020E9
:10C17000A0440020E4350020343700208945002009
:10C1800000210D4A0CE0834206D101EB410000EB97
:10C19000C10002EB00107047491CC9B2022908D245
:10C1A00001EB410303EBC10302EB03131B78FF2BED
:10C1B000E9D10020704700003C1300202DE9F04732
:10C1C0000026DFF80C81DFF80C91DFF80CA1434C5E
:10C1D0004FF400474FF6FF75012804D0022817D00E
:10C1E000032854D070E0EB21822008F0DDFBA0F59D
:10C1F0000041E080B94202D2281AE08002E0A84261
:10C2000000D3E680E088FCF79DFA42464B4652E0B8
:10C21000E321B22008F0C8FBE080B84204D301213A
:10C220006180281AE08000E0668080B2FCF78AFA1C
:10C2300042464B46FCF780F900225346FCF7EEF9E4
:10C24000FCF7B4FAFCF79FFA4FF03332244BFCF7BB
:10C2500073F9244A244BFCF7E1F9FCF7A7FAA06133
:10C260006088012830D11D484FF4FA61143003F082
:10C270000FFD012807D11DA005F01CFD1748002166
:10C28000143003F005FDA06980F000401BE0E321BD
:10C29000B42008F089FBA0F50041E080B94202D249
:10C2A000281AE08002E0A84200D3E680E088FCF78C
:10C2B00049FA4246164BFCF73FF900225346FCF779
:10C2C000ADF9FCF773FAA061A069BDE8F087000042
:10C2D000FCA9F1D24D622040E0FFEF407C0000203D
:10C2E000F308CA40F6285C8FC2F513404E656761BB
:10C2F0007469766520766F6C746167652073616D13
:10C30000706C65206661756C74210D0A0000000078
:10C310004D621040C079032801D0002070470120F1
:10C3200070478079012802D0002800D00020704793
:10C330000148406870470000380C00202DE9F84F94
:10C3400005462D4800248DF80040006F016B88479A
:10C35000DFF8A89003462A4999F8008001260220B8
:10C360000322284F6FF0814CDFF89CA02944AC4495
:10C37000B8F1000F0AD0B8F1010F1ED0234BB8F16D
:10C38000020F1FD0B8F1030F2CD120E0DFF880801E
:10C39000B94203D298F80F10022910D31D4929443D
:10C3A0001D4DA94203D298F80F10022911D2D4458D
:10C3B00015D3BBB188F80F4014E0B94212D28DF802
:10C3C000006011E0994204D3D44508D30AE09942B1
:10C3D00002D28DF8002007E010498C4502D28DF87A
:10C3E000000001E08DF8004069460D48FFF7FAFAB9
:10C3F00089F80000BDE8F88FC80600200C0B00206B
:10C40000F528DCC3285C4F04FFFF3F00F5289C03A0
:10C4100060230020CCCCCCC0CCCC8C00FFFF5F00D4
:10C42000AC2300202DE9F04114480468144821464B
:10C43000FBF765FF054613492046FBF766FF2946D3
:10C44000FBF795FFFCF79FF90F4D88460446002245
:10C450002B46FCF76EF806460F4620464146002262
:10C460002B46FCF769F832463B46FCF7D7F8FCF759
:10C470009DF906490860BDE8F0810000380C0020F5
:10C480000000A0403333A3400000244058000020A7
:10C490000148B0F908007047380C002040790128A5
:10C4A00002D0002800D000207047000001484078EA
:10C4B000704700002000002070B53F4E7088401C7F
:10C4C00080B270800A286FD33C4C00257580B4F888
:10C4D00040004FF4FA71884224D2401C80B2A4F884
:10C4E000400088421ED12572607F032801D00228B7
:10C4F00018D125770120607784F82250A5716574E2
:10C50000A4F8405084F824502C4884F8255084F82E
:10C5100027503838E5730179012901D1856105710A
:10C5200000F04EFB94F8241025480029017802D031
:10C5300021F0030101E041F00301017094F825109E
:10C540000029017802D021F00C0101E041F00C013A
:10C550000170B4F8541031B1491E0904090CA4F853
:10C56000541000D1E5733188491C89B231806429A7
:10C570001AD3358094F8291079B1491E11F0FF01C2
:10C5800084F8291009D1E178012906D1E57094F8E1
:10C59000281011B1491E84F82810217A0029017849
:10C5A00003D021F01001017070BD41F01001017045
:10C5B000BDE8704000F004BBB00B0020A044002098
:10C5C0002C0B002000F00F00092801D937307047EC
:10C5D000303070470009092801D9373070473030B2
:10C5E0007047704770470000074A30B45170064BDF
:10C5F0000022083303E0845C9C54521CD2B28A426D
:10C60000F9D330BC02F0B4BDF00B0020064A10B5DF
:10C61000054B00215278083303E05C5C4454491C0C
:10C62000C9B29142F9D310BDF00B002070B50C4691
:10C63000054602F053FE024621462846BDE87040FA
:10C6400004F07CBA074A30B45170064B002208331C
:10C6500003E0845C9C54521CD2B28A42F9D330BCB1
:10C6600002F0DEBDF00B002002F08EBE10B504F02B
:10C67000E1FA02490020087010BD0000F00B002014
:10C680000148407870470000F00B00207FB50D494D
:10C690006B464A6800928A788DF80420002104E0F5
:10C6A000445C5D18491C6C71C9B29142F8D30649CB
:10C6B00001208DF80D0048709DE80F0003F07EFB0F
:10C6C0007FBD0000F00B0020A044002001498870CD
:10C6D00070470000F00B0020024A40F2B471516034
:10C6E00070470000F00B00207047000070B50D4649
:10C6F000064602F0F3FD0A4C217800290ED17F2175
:10C7000001704670857003250020FFF7E5FF03F0F8
:10C7100071F8284602F008FE0120207070BD00006C
:10C72000F00B002070B50E46044602F0D7FD0C4D0C
:10C730002978002913D1002C11D0002203E0B15C2C
:10C740008154521C92B2A242F9D30020FFF7C4FFD9
:10C7500003F050F8204602F0E7FD0120287070BD7C
:10C76000F00B002002F0CABC0078704700787047D8
:10C77000FEE700002DE9F0410427044600F17006B1
:10C780004FF001085FF0000594F89100062876D27A
:10C79000DFE800F0031975424E5C94F8540003285A
:10C7A0006DD330460AF00CF9002868D104F19401E9
:10C7B00030460AF021F970B384F8918084F89050E3
:10C7C00084F8AC5050E0D4F808C094F89930207840
:10C7D00004F19A02D4F89410E04784F8980094F891
:10C7E0009010491C84F89010FF280CD0022084F887
:10C7F000910084F8AC5094F854008128C4D10320EF
:10C8000084F85400C0E794F84400C9B2814236D39A
:10C8100084F891702CE027E094F8900094F844108C
:10C82000884202D384F891701EE084F891801BE066
:10C8300084F89150D4F8A82022B10121D4F8A400A2
:10C84000904711E0226D002AF7D10DE084F8915055
:10C85000D4F8A81029B10220D4F8A42006F0E8FFEB
:10C8600002E0216D0029F6D194F8910004288BD1C3
:10C870002278BDE8F0410421012006F0D9BFBDE8CF
:10C88000F081000030B500201D4902460446012514
:10C89000C1F8985105235B1E1B041B0CFBD14006FD
:10C8A000D1F81C31000E0BB140F00100C1F89841E5
:10C8B00005235B1E1B041B0CFBD1521CD2B2082AA1
:10C8C000E6D3C1F898410522521E1204120CFBD186
:10C8D000C1F89C410522521E1204120CFBD1C1F872
:10C8E00098510522521E1204120CFBD1C1F8984136
:10C8F0000522521E1204120CFBD1C1F89C5130BD0E
:10C90000008021420F480122C0F89C210521491EC8
:10C910000904090CFBD1C0F898210521491E09041E
:10C92000090CFBD10022C0F89C210521491E0904F5
:10C93000090CFBD1C0F898210520401E0004000C12
:10C94000FBD17047008021420C480021C0F89C11A7
:10C950000521491E0904090CFBD10122C0F89821C8
:10C960000521491E0904090CFBD1C0F89C210520B2
:10C97000401E0004000CFBD17047000000802142E3
:10C9800030B516490024C1F8984122460123050616
:10C9900002D5C1F89C3101E0C1F89C41C1F8983141
:10C9A00005256D1E2D042D0CFBD1C1F898410525E0
:10C9B0006D1E2D042D0CFBD14006521C000ED2B270
:10C9C000082AE4D3C1F89C31C1F898310520401EF3
:10C9D0000004000CFBD1C1F8984130BD0080214219
:10C9E0002DE9F041084D4FF400642C6007F0E9FE9A
:10C9F0002F1F66103E6007F0E4FE2E6007F0E1FE98
:10CA00003C60BDE8F0810000140C014070B5084C9A
:10CA10004FF40060206007F0D4FE2515256007F074
:10CA2000D0FE201D0560BDE8704007F0CABE0000C2
:10CA3000100C01402DE9F047144F0024DFF84C8022
:10CA400082462546A8F108083E1507F1040960064C
:10CA5000040E3E6007F0B5FED8F80000000501D5D1
:10CA6000641CE4B2C9F8006007F0ABFE6D1CEDB2C7
:10CA7000082DECD3BAF1000F04D0FFF7B1FF204628
:10CA8000BDE8F087FFF7C2FFF9E70000100C014096
:10CA90002DE9F047DFF84890054600244FF4806701
:10CAA0004FF40068A9F104062806404601D530601D
:10CAB00001E0C9F8000007F084FE376007F081FE4E
:10CAC000C9F80070072C01D1C6F800806806050E71
:10CAD00007F077FE641CE4B2082CE5D3BDE8F087CC
:10CAE000140C014070B509484FF400650560041549
:10CAF000046007F066FE054E361D356007F061FEE6
:10CB00003460BDE8704007F05CBE0000100C0140CE
:10CB100070B507484FF400640460054D00152D1FE3
:10CB2000286007F04EFE2C60BDE8704007F049BE5B
:10CB3000140C014070B50C4C4FF40060206007F0FD
:10CB400040FE2515256007F03CFE074808380068C0
:10CB5000000501D5012400E000240348001D056004
:10CB600007F02FFE204670BD100C0140064A0188D8
:10CB70000020B2F835308B4204D3B2F8432014328F
:10CB80008A4200D803207047C806002070B50B4DBC
:10CB900006680024B5F83900FBF7CFFD3146FBF7F6
:10CBA00021FE01D2012407E0E88FFBF7C6FD3146E4
:10CBB000FBF722FE00D20224204670BDC8060020EA
:10CBC0007047000003497F20086003490020087077
:10CBD00070470000002C0040740100200C48C1691F
:10CBE00041F40061C1610B4940F2FF30086009481F
:10CBF0007F21001F0160016841F0800101604FF05A
:10CC0000E020002180F800140121C0F800117047D5
:10CC100000100240042C00402DE9FE4342F20F7840
:10CC2000224CADF80080694621480194FCF704F9D4
:10CC300040F6C315ADF8005069461D480194FCF755
:10CC4000FBF841F64B561B4FADF80060694618489B
:10CC50000197FCF7F1F842F22730ADF80000694681
:10CC600013480194FCF7E8F840F2E730ADF8000013
:10CC70001148019069460E48FCF7DEF8ADF80060F7
:10CC800069460B480194FCF7D7F8ADF800506946A7
:10CC900007480197FCF7D0F8ADF8008069460448D2
:10CCA0000194FCF7C9F8BDE8FE83000025D8000810
:10CCB000C434002035D90008F9EA00082DE9F04114
:10CCC0000024154E5FF0FF0704EB440000EBC400A6
:10CCD00006EB00100546B021FBF78EFA641CE4B2A7
:10CCE0002F70022CF0D30D4C206818B90C4806F0B8
:10CCF00019FE206006F075FE18B90A21206806F0BA
:10CD000069FE0849012006F0ABFDBDE8F041064987
:10CD1000022006F0A5BD00003C130020D00000203A
:10CD2000F16C0108D9A00008CDA0000810B5482179
:10CD30000F48FBF761FA0E4828214830FBF75CFAF0
:10CD40000C4801F06DFC010004D009481422483061
:10CD5000FBF739FA0748203001F062FC010006D0E9
:10CD600003481422BDE810405C30FBF72CBA10BD1C
:10CD7000440F00208472010810B5284800F0B3F970
:10CD80002648083000F0AFF92448103000F0ABF925
:10CD90002248183000F0A7F92048203000F0A3F90D
:10CDA0001E48283000F09FF91C48303000F09BF9F5
:10CDB0001A48383000F097F91848403000F093F9DD
:10CDC0001648483000F08FF91448503000F08BF9C5
:10CDD0001248583000F087F91048603000F083F9AD
:10CDE0000E48683000F07FF90C48703000F07BF995
:10CDF0000A48783000F077F90848803000F073F97D
:10CE00000648883000F06FF90448903000F06BF964
:10CE10000248BDE81040983000F065B95C09002078
:10CE200070B51A4C1B491C486278194D0978006985
:10CE3000052A18D2DFE802F003091E101800E87B6B
:10CE400008B103200EE001200CE0072902D0804742
:10CE50000228F8D1022005E00729F2D080470228F5
:10CE6000EFD00420607070BD0729F3D080470228FE
:10CE7000F7D1EFE700F022FB00266E606E7301F041
:10CE80004BFBA8606670267070BD0000340800205F
:10CE90002824002060230020580000202DE9F041C4
:10CEA00016460D46FFF76CF9040007D035B12EB1D8
:10CEB000287818B194F85400012802D00020BDE869
:10CEC000F08195F82000C00702D0A86A0028F6D0AB
:10CED00095F8250084F8450010B9322084F8450003
:10CEE000C0B200EB4000C00004F036FFC4F88C0074
:10CEF000011EE4D094F84530182204F1700009F0C6
:10CF00006FFD95F82000C0070FD194F8450000018F
:10CF100004F022FFC4F88800011E2ED094F845309A
:10CF2000102204F1580009F05BFD286A206404F126
:10CF3000200007462021FBF75FF91F2229463846CB
:10CF4000FBF741F9E86AF862A86AB86295F824002C
:10CF500087F82400286B38630B4830610B48F06079
:10CF60000B48B0600B4870600B4830600B48706134
:10CF7000022084F854000120A1E754F88C0F04F03B
:10CF8000BDFE0020206099E7C14D0108314C010829
:10CF9000A34C0108B34C0108274D01089D4B010823
:10CFA00038B5044601213C2001F0D0F901210846A2
:10CFB00001F0CCF901211248FEF72EFEA468B4B1AD
:10CFC0002088ADF8000010208DF8030002208DF8B5
:10CFD000020069466068FEF7CDFD207A01280AD07C
:10CFE000002803D121886068FEF749FE38BD05A0FE
:10CFF00004F060FE38BD21886068FEF742FE38BD4F
:10D00000000230004F5053206973204E554C4C0D98
:10D010000A00000010B5044800F0CBF8BDE810404D
:10D02000024800F0E6B80000C4090020CC09002046
:10D0300010B5044800F0BDF8BDE81040024800F00B
:10D04000D8B80000CC090020C409002010B504485D
:10D0500000F0AFF8BDE81040024800F0AAB80000A8
:10D06000C4090020CC09002010B5054800F0A1F843
:10D07000044800F09EF8BDE8104003A004F01ABE7A
:10D08000C4090020CC090020414320C8ABB5CD0025
:10D0900010B5054800F0ADF8044800F0AAF8BDE866
:10D0A000104003A004F006BEC4090020CC090020F3
:10D0B000414320C8ABB8DF0038B504460121102039
:10D0C00001F044F9A06800280CD00188ADF80010E8
:10D0D00004218DF8031003218DF802104068694681
:10D0E000FEF748FD38BD00680168002900D00847F8
:10D0F0007047000038B5044601213C2001F026F9B4
:10D10000A468B4B12088ADF8000010208DF80300A9
:10D1100002208DF8020069466068FEF72BFD207A38
:10D1200001280AD0002803D121886068FEF7A7FDF6
:10D1300038BD04A004F0BEFD38BD21886068FEF74C
:10D14000A0FD38BD4F5053206973204E554C4C0DF7
:10D150000A00000038B504460121042001F0F6F869
:10D16000A468002C15D02088ADF8000010208DF8A0
:10D17000030003208DF8020069466068FEF7FAFCA0
:10D18000207A012806D0002803D121886068FEF7A4
:10D1900076FD38BD21886068FEF773FD38BD10B597
:10D1A000044601884068FEF76AFD002020720120D5
:10D1B00010BD10B500684168496819B1806888479A
:10D1C000012010BD002010BD01884068FEF750BD51
:10D1D00000684168896809B1806808470320704782
:10D1E00010B5044601884068FEF74BFD012020720F
:10D1F00010BD10B500684168096819B1806888479A
:10D20000012010BD002010BD38B5044601211020BA
:10D2100001F09CF8A06800280CD00188ADF800103F
:10D2200048218DF8031003218DF8021040686946EB
:10D23000FEF7A0FC38BD00000A4810B5C088094AB6
:10D240000221203A04F094FC06480749303800696E
:10D25000FBF75BF84FF07A51FAF7FFFF034948609C
:10D2600010BD00005000002000003041380C0020AC
:10D2700030B504465FF0000014F8015B8D4203D125
:10D28000012A08D0521ED2B2002B04D0401C5B1ED3
:10D2900080B29BB2F0E730BD124810B5C07E124C90
:10D2A000012813D04FF47A700146A0600E4802F0B6
:10D2B000EFFC012814D1606810F0010F00F10100AB
:10D2C00060600A4804D0FFF774FF03E06420EBE7D6
:10D2D000FFF78FFFBDE810400021034802F0D8BCE3
:10D2E00010BD0000780C00200000002094090020F0
:10D2F000094B9A7A72B1094841780B44DB7A03B141
:10D300008380491CC9B241708A4201D80021417012
:10D3100000797047002070472C0B00208C050020FE
:10D3200003A004F0C7FC04F05DFC00F003FC000067
:10D33000476F20746F20536C6565700D0A00000004
:10D34000FEE770474FF4A06000F03EB800F01F0207
:10D35000012191404009800000F1E020C0F88011D7
:10D360007047000070B50F23C47801780122F4B132
:10D37000144C2468457804F4E064C4F5E064240A9D
:10D38000C4F10406E3408478B5401C402C4301F10D
:10D39000E021230181F80034007800F01F018A4069
:10D3A0004009800000F1E020C0F8002170BD01F0CC
:10D3B0001F0082404809800000F1E020C0F8802171
:10D3C00070BD00000CED00E002490843024908600E
:10D3D000704700000000FA050CED00E0024A114021
:10D3E000014302480160704780FFFF1F08ED00E025
:10D3F00004480168044A01F4E06111430160BFF38D
:10D400004F8FFEE70CED00E00400FA0504480168C8
:10D41000044A01F4E06111430160BFF34F8FFEE75E
:10D420000CED00E00400FA054FF400720021014801
:10D4300003F0DEBD0045002010B50948FFF7D9FE16
:10D440000120FDF70CFF0748FFF7D3FE4FF4FA70F9
:10D45000FDF705FFBDE810400248FFF7AABE000037
:10D46000C4090020CC09002010B5FFF7E1FD4FF4FE
:10D47000FA70FDF7F4FEFFF7E9FD0449002048715A
:10D48000BDE8104002A004F015BC00008823002075
:10D490004F50454E5F313256506F7765725265611D
:10D4A0006C790D0A0000000002490120C871024891
:10D4B000FFF79FBE882300206C090020024901204D
:10D4C000C8710248FFF795BE882300206C09002030
:10D4D0000249012088710248FFF78BBE8823002093
:10D4E0005C090020007808B10020704701207047D7
:10D4F000014908627047000000000E4202490A68B4
:10D5000042EA8000086070470070004000B50B30B0
:10D51000034609F0D1FA18680D49C0F309300A2210
:10D5200021F83C0F1868C0F3093090FBF2F081F845
:10D5300030005868800C48805868800C4881186812
:10D540001A79800D62F38D208881012000BD0000D2
:10D55000C806002070B50B30044609F0ADFA0A4D3C
:10D560006068296FC0F3C260496A8847296F2068E4
:10D57000C96AC0F3026088472068C0F3407085F82C
:10D580005900012070BD0000C806002000B50B3016
:10D59000034609F091FA98880A2280B290FBF2F0D3
:10D5A0000A49A1F866005868000C90FBF2F0A1F857
:10D5B00068005868000C90FBF2F040F4805021F8AD
:10D5C0004A0F1868000C4871012000BDC8060020F1
:10D5D00000B50B30034609F06FFA98880B49000A32
:10D5E0000A3081F86A005868000E0A3081F86B0032
:10D5F0009888000A01F8500F5868000E8870586823
:10D60000000C48701879C870012000BDC8060020C1
:10D6100010B50446FBF7FCFC0B34204609F04CFA2D
:10D6200060684FF6FF71C0F3892000EB800001EACB
:10D630004000044921F8410F6068000D4880012036
:10D6400010BD0000C806002000B500F10B0318460D
:10D6500009F032FA034819680163596841630120EF
:10D6600000BD0000B022002000B500F10B031846F9
:10D6700009F022FA0348196881635968C1630120DF
:10D6800000BD0000B022002000B500F10B031846D9
:10D6900009F012FA034819680164596841640120CD
:10D6A00000BD0000B022002070B500F10B04204640
:10D6B00009F002FA2068154DC0F340400A2185F8B0
:10D6C00045006068000C90FBF1F0A5F83300A088DD
:10D6D000C0F38D002880207868712088000A85F8C2
:10D6E0003B00A088C0F38D00A5F83900296F2068A1
:10D6F000C968C0F3004088472068C0F3004085F83F
:10D700005A002068800C2881012070BDC8060020C6
:10D7100000B50B30034609F0CFF998880549C0F3EE
:10D720008D00C8805868000DC0F57A60A1F83500FA
:10D73000012000BDC806002000B50B30034609F0EB
:10D74000BBF918680549C0F38930A1F837000448CF
:10D75000196881655968C165012000BDC8060020AF
:10D76000B02200202DE9F0472348244F0122868A69
:10D7700007F2FA2500206F602870334620213846D2
:10D78000FFF776FD687004461DA0696804F092FA00
:10D79000B4422AD0022025E0385D202828D02978FC
:10D7A000A14605EB810107EB09008860334642463C
:10D7B00020211248FFF75CFD2A7815490446A0EBAA
:10D7C00009005054297805EB8100826811A004F00B
:10D7D00071FA2878401CC0B22870042805D208F1DC
:10D7E0000100C0B28046B442D6D10120BDE8F08726
:10D7F000641CA4B2F7E7000088010020921D0020FD
:10D80000696E6F757420636D643A25730A000000B9
:10D81000A4200020256420706172616D3A25730A8E
:10D82000000000002DE9FC4100203E4C00904FF428
:10D830004571019021606160207260720820A072C1
:10D84000E84600F093FF054600F0A4FF019A65F357
:10D85000196265F39B6260F31D72334D60F39F7232
:10D860000192287A10B3002060F311420192E87906
:10D87000F0B1002060F393420192FDF79FFB009905
:10D8800060F38B210091FDF78FF8DDE9006760F30D
:10D89000155726480197C068FAF761FF80B20A2140
:10D8A000B0FBF1F0C82805D2002004E00120DBE73E
:10D8B0000120DFE7C83860F35D561D48CDE90067F9
:10D8C000006FB0F9020090FBF1F000F5FA7060F320
:10D8D00014360096FDF7CCF9009960F3DF7124202F
:10D8E0000091FDF763FFDDE9001260F39E71687A35
:10D8F00060F34F32CDE90012687808B9A87800B11A
:10D90000012060F3D7524046019209F0DCF80098FC
:10D9100044F80B0F01986060024806F08BF8BDE8F0
:10D92000FC8100001823002088230020380C0020F0
:10D93000C80600202DE9FC410024374E00944FF426
:10D940007A70019430607060347274720820B07222
:10D95000E8462820FDF72AFF58B92620FDF726FFC4
:10D9600038B91C20FDF722FF18B92120FDF71EFF52
:10D9700008B1012200E00022019962F38E31274AAA
:10D98000019113781B1F022B05D8D27C1AB10122FA
:10D9900062F3CF310191FDF707F8022803D0FDF7BC
:10D9A00003F8032803D1019864F3CF3001901C4F92
:10D9B00078688047DDE90054283060F31F64194817
:10D9C00019490078283060F3174401943868FAF751
:10D9D0009CFCFAF7C4FE42F21071884200D9084656
:10D9E00060F30D041148807A60F30B25CDE90054F3
:10D9F000FFF77EFC009960F307014046009109F0B3
:10DA000062F8009846F80B0F01987060024806F023
:10DA100011F8BDE8FC8100001823002060230020DD
:10DA2000580000208823002000007A442C0B00209E
:10DA30007CB50021144B009140F23F4001911860E9
:10DA400058601972114C597208209872A278684671
:10DA5000521CD2B2A270102A00D3A17000990125E5
:10DA6000A47865F3CF3164F30B21641C64F30701E0
:10DA7000009109F028F8009843F80B0F01985860BE
:10DA8000014805F0D7FF7CBD182300208C0500203D
:10DA90001FB5104A012010720020A2F84000009B20
:10DAA0009DF80410A3F5E0636846343B09D0AB2B26
:10DAB00006D140F2DF73A2F84E30401DFEF794FD10
:10DAC0001FBD40F23473A2F84E30401DFEF7BAFD80
:10DAD0001FBD0000A044002000B50B30034608F035
:10DAE000EBFF0648196801615968416104495868AB
:10DAF000096F000C0880012000BD0000B02200204A
:10DB0000C806002070B50B30044608F0D5FF074D5D
:10DB10002068296FC0F30360C9698847296F60686E
:10DB20004969800F8847012070BD0000C8060020A9
:10DB3000704700004FF0E020016921F0020101610F
:10DB40000220FFF703FC0320FFF700FC0420FFF78F
:10DB5000FDFB0520FFF7FAFB0620FFF7F7FB072088
:10DB6000FFF7F4FB0820FFF7F1FB0920FFF7EEFBBE
:10DB70000A20FFF7EBFB0B20FFF7E8FB0C20FFF779
:10DB8000E5FB0D20FFF7E2FB0E20FFF7DFFB0F2088
:10DB9000FFF7DCFB1020FFF7D9FB1120FFF7D6FBC6
:10DBA0001320FFF7D3FB1420FFF7D0FB1520FFF75E
:10DBB000CDFB1620FFF7CAFB1720FFF7C7FB182085
:10DBC000FFF7C4FB1920FFF7C1FB1A20FFF7BEFBCC
:10DBD0001B20FFF7BBFB1C20FFF7B8FB1D20FFF746
:10DBE000B5FB1E20FFF7B2FB1F20FFF7AFFB202085
:10DBF000FFF7ACFB2120FFF7A9FB2220FFF7A6FBD4
:10DC00002320FFF7A3FB2420FFF7A0FB2520FFF72D
:10DC10009DFB2620FFF79AFB2720FFF797FBFEF7D7
:10DC2000D1FF2820FFF792FB2920FFF78FFB2A2046
:10DC3000FFF78CFB3220FFF789FB3320FFF786FBD1
:10DC40003420FFF783FB3520FFF780FB3620FFF7FA
:10DC50007DFB3720FFF77AFB3820FFF777FB392071
:10DC6000FFF774FB3A20FFF771FB3B20FFF76EFBD9
:10DC70003C20FFF76BFB3D20FFF768FB3E20FFF7E2
:10DC800065FB3F20FFF762FB4020FFF75FFB412071
:10DC9000FFF75CFB4220FFF759FB4320FFF756FBE1
:10DCA0000020411E820002F1E022C2F88011401CD7
:10DCB0000828F7DB0120FFF721FCFEF783FF094866
:10DCC000FFF797FA0848C07B0028084802D0FFF702
:10DCD00090FA01E0FFF76DFA41F28830FDF7BFFAE4
:10DCE000FFF794FBF409002028240020EC09002011
:10DCF00070B56249624E634C4868634D401C486091
:10DD00000521B0FBF1F201FB120005287AD2DFE811
:10DD100000F0033347728F005CA003F0CBFF287A3A
:10DD200008B165A105E0306980475449083151F8D0
:10DD3000201064A003F0BEFF206F016A88474F499E
:10DD40004C3151F8201066A003F0B4FF6A484B49EB
:10DD500094F86C200078143151F8201067A003F07B
:10DD6000A9FF94F8450008B16CA100E06FA173A071
:10DD7000BDE8704003F09EBFB4F84320B4F84110F2
:10DD800074A003F097FF7E48B0F81D20B0F81B1078
:10DD90007CA003F08FFF206FB0F9021084A0E7E7AA
:10DDA000B06880470446706880470146224686A0D6
:10DDB00003F080FF8C48FFF70BFA08B18BA400E05A
:10DDC0008DA48F48FFF704FA08B18BA100E087A16A
:10DDD00022468CA003F06EFF287A08B191A200E0E1
:10DDE00091A2E87908B191A100E091A1BDE870404D
:10DDF00090A003F05FBF974C6068FAF7C4FC02463E
:10DE00000B4600E038E094A003F054FFE068FAF716
:10DE1000BAFC02460B4695A003F04CFF3068FAF7B7
:10DE2000B2FCBDE8704002460B4696A003F042BF2C
:10DE3000206F016B88471149343151F8201097A0A9
:10DE400003F038FFA87808B19AA200E09BA2687896
:10DE500008B198A100E099A19AA003F02BFFFAF76E
:10DE600051FF28B99D48D0E900219DA003F022FF71
:10DE7000BDE8704000F04AB970BD00003C070020CA
:10DE800058000020C8060020882300200D0AA1AAFF
:10DE9000A1AAA1AAA1AAA1AAA1AAA1AAA1AAA1AA2A
:10DEA000A1AAA1AAA1AAA1AAA1AAA1AAA1AAA1AA1A
:10DEB000A1AAA1AA0D0A000041435F4368617267ED
:10DEC000696E67000D0A4443555F576F726B696E48
:10DED000674D6F6465203C25733E0D0A000000000D
:10DEE0005643555F576F726B696E674D6F6465205F
:10DEF0003C25733E0D0A00006023002043686172D8
:10DF000067696E675F5374616765203C25733E09DE
:10DF1000534F43203C25643E0D0A0000436F6E734F
:10DF200074616E74566F6C7461676500436F6E73D5
:10DF300074616E7443757272656E740043686172C9
:10DF400067696E675F4D6F646520203C25733E0DE9
:10DF50000A00000044656D616E645F766F6C7461E9
:10DF60006765203C25643E0944656D616E645F63AE
:10DF7000757272656E74203C25643E0D0A000000C7
:10DF8000FC0C00204F75747075745F766F6C746153
:10DF90006765203C25643E094F75747075745F6336
:10DFA000757272656E74203C25643E0D0A00000097
:10DFB0004368617267696E6743757272656E74203B
:10DFC0003C25643E0D0A000054656D703120202010
:10DFD000203C25643E092047554E5F54454D502056
:10DFE0003C25643E0D0A00009C09002044697363CF
:10DFF0006F6E6E65637400004F70656E0000000008
:10E00000A409002044435F52656C6179203C25736C
:10E010003E202041435F52656C6179203C25733E70
:10E020000D0A0000434300004343320043433100E4
:10E030004350000043502D4343312020203C2573A2
:10E040003E092043432D4343322020203C25733E8C
:10E050000D0A0000380C00204B4C33305F566F6CBB
:10E0600074203C25663E0D0A0000000053616D706F
:10E070006C5F766F6C74616765202020203C25669C
:10E080003E0D0A0043435F52206973202020202068
:10E0900020202020203C25663E0D0A004F42435F91
:10E0A00047756E436F6E6E6563742020203C257348
:10E0B0003E0D0A004E4F5F4C6F636B004C6F636BFD
:10E0C000000000004856494C203C25733E2048562D
:10E0D000494C5F32203C25733E0D0A002824002065
:10E0E000456E7465722046616C7365536C6565702E
:10E0F0002049646C6520636F756E74202564204D23
:10E1000041582069732025640D0A00002DE9F0476D
:10E11000DFF84880DFF848900025464618F80500EB
:10E12000B0B1FDF705FB3327B04600244FEA0906DE
:10E1300018F8052016F83410914205D106EBC400FA
:10E14000416808A003F0B6FD641CE4B2BC42EFD302
:10E150006D1CEDB2052DE0D3BDE8F0872C08002042
:10E16000C07501084572726F7220436F6465204963
:10E170006E466F2069732025732D25640D0A0000FB
:10E180002DE9F041264C207860B10026254D01286C
:10E190000DD0022827D003283FD0BDE8F04122A0AF
:10E1A00003F088BDFAF7AEFD80F0010014E008F03E
:10E1B0005BFC012798B1012813D002280DD11D481E
:10E1C00006721D48FEF7F5FFFFF72CFB4FF4FA70BF
:10E1D000FDF745F86F7302202070BDE8F0812770CD
:10E1E000FBE72670F9E76068401C6060A97B0129A5
:10E1F00005D0052803D303206660207003E00128C2
:10E2000001D1FBF747FBFEF70BFE287B0028E4D08B
:10E21000FFF754F96E606E73E3E7FFF781F80000D3
:10E22000340800202824002045525220536C656594
:10E23000700D0A00882300207C090020F0B52948D1
:10E24000807A00EB80004200B2F5AF7F43D32649CD
:10E25000264B00240878012703EBC0060546B6F8D4
:10E2600002C094450CD316E033F830C0944505D273
:10E2700003EBC00CBCF802C0944504D8401CC0B2EB
:10E280000528F1D301E0052800D30420CC708B7859
:10E29000EBB98F7016E033F830C094450CD814E019
:10E2A00033F830C0944505D203EBC00CBCF802C073
:10E2B000944503D8401EC0B20028F1D18C70CB78B1
:10E2C0002BB9CF70F3888B8001E0CC708C708B8879
:10E2D00013B15B1E8B80F0BD8542FCD0322AFAD987
:10E2E0000870F0BDCC350020900B0020AC77010801
:10E2F000034A516821F440410143516070470000D6
:10E3000000100240044A0029516901D0014300E095
:10E31000814351617047000000100240044A002907
:10E32000D16901D0014300E08143D1617047000011
:10E3300000100240044A0029116901D0014300E0A5
:10E34000814311617047000000100240044A002917
:10E35000916901D0014300E0814391617047000061
:10E36000001002400149086070470000400442422A
:10E37000F0B52A4A51682A4B11F00C014FF00F05F5
:10E3800003D0042901D0082901D0036026E0516898
:10E39000546805EA914104F480340D2901D0891CA8
:10E3A00000E00621BCB1D46A14F4803FD46A04F0C2
:10E3B0000F0404F101040AD0D66AD76AC6F3031623
:10E3C000761CB3FBF6F3C7F30327BF1C7B43B3FBF9
:10E3D000F4F34B43D9E7134B594301605168124C96
:10E3E00005EA1111635C0168D94041605368072553
:10E3F00005EA1323E35C21FA03F38360536805EA1B
:10E40000D323E35CD940C1605268032303EA92320C
:10E41000231F9A5CB1FBF2F10161F0BD00100240D4
:10E4200000127A0000093D00F80400200246002096
:10E4300053090949012B0BD0022B0BD0D1F8241022
:10E4400002F01F02012393400B4200D001207047CD
:10E450000968F5E7096AF3E700100240014908601E
:10E460007047000080044242014908607047000084
:10E470003C04424202490A6A02430A6270470000B1
:10E480000010024010B5084C44F22001A06B084275
:10E4900001D1400605D52F20FDF796F90020A06395
:10E4A00010BD012010BD0000FC0C002070B50D4611
:10E4B0000646002403E0305D02F0F4FB641CAC422D
:10E4C000F9DB70BD70B50D460646002403E0305DF3
:10E4D00002F0E8FB641CAC42F9DB0D2002F0E2FB29
:10E4E0000A2002F0DFFB002403E0305D01F0B6FCFF
:10E4F000641CAC42F9DB70BD0248018841F0100198
:10E5000001807047042800400248018821F0100172
:10E510000180704704280040034800880249091F11
:10E52000098840EA014070471C28004010B50121CD
:10E530004FF0C050FFF7F2FE4FF400742046FFF793
:10E5400099FF0120FFF790FF0120FEF7D1FFFAF7B6
:10E55000B8FC0120FFF782FF6120FFF767FF00286A
:10E56000FAD02046FFF786FF0120FFF77DFF00F07D
:10E5700023F800F019F849F63F4000F005F8BDE82F
:10E58000104000F011B8000000B50246FFF7B4FFDC
:10E590000449C2F303400880081D02805DF804EBC3
:10E5A000FFF7B2BF08280040024801888906FCD561
:10E5B00070470000042800400448018821F0080149
:10E5C000018001880907FCD570470000042800403D
:10E5D000114910B50120C1F89801FEF793F9902078
:10E5E000FEF7CEF90020FEF7CBF9FEF7ADF9FEF706
:10E5F00089F99120FEF7C4F9FEF744F9074C208011
:10E60000FEF740F96080FEF79FF96088218840EAB4
:10E6100001202080208810BD00802142840000203D
:10E6200010B510B3416801B38168F1B1037818499E
:10E63000002200BF02EB420404EBC20401EB04140D
:10E6400024789C4211D0521CD2B2022AF2D300226A
:10E6500002EB420303EBC20301EB03131B78FF2B16
:10E6600005D0521CD2B2022AF2D3002010BD02EB18
:10E67000420303EBC20201EB0214014620222046B2
:10E68000F9F7A1FD012084F85400024810BD0000F4
:10E690003C130020D4000020704772B6704762B669
:10E6A0007047000070B5FDF7BDFEFDF747FE002284
:10E6B000012804D0022804D0032802D002E001225D
:10E6C00000E002220A4900230C78A24202D08B61AA
:10E6D0000A7070BD4D78AA4201D18B6170BD8A6904
:10E6E000521C8A61022AF9D34C708870F5E7000049
:10E6F0002000002070B50D460446FFF70DFF21688D
:10E7000009B1616802E04119C4E90001814201D800
:10E71000012070BD002070BD00210160416001201A
:10E720007047000070B50F4D0224B5F8410028B1C4
:10E73000B5F8430010B10024204670BD0A483C21C2
:10E740000646FFF7D7FF0028F6D03046FFF7E4FF74
:10E75000B5F8410020B10A20FDF736F80124EBE7B7
:10E760000920F9E7C806002094340020084810B5B5
:10E77000C0780324012807D040B10420FDF716F823
:10E7800000B10224204610BD0124FBE70024F9E774
:10E7900088230020084810B500790324012807D0F9
:10E7A00040B10320FDF702F800B10224204610BD5D
:10E7B0000024FBE70124F9E7882300202DE9F0413C
:10E7C00042780378284E02EB032295B2284A378A12
:10E7D0000024264B92F82220AF4207D11B7A8B42AD
:10E7E0003CD1C2B30A46811C22482EE0778AAF4250
:10E7F00008D15B7A8B4231D16AB30A46811C1D482D
:10E80000133022E0F78BAF4208D1DB7B8B4225D15E
:10E810000AB30A46811C1748773016E0378CAF429E
:10E8200008D11B7C8B4219D1AAB10A46811C114820
:10E830007B300AE0768CAE4212D15B7C8B420DD1EC
:10E840004AB10A46811C0B487F30F9F7BCFC2846C8
:10E85000FCF712FD05E0FFE7332402E0132400E09B
:10E8600031242046BDE8F0810E780108FA770108CE
:10E87000A0440020453500202DE9FF4F8046604828
:10E8800000248DB0B0F842201F46A146042A03D2CE
:10E89000132011B0BDE8F08FB8F8013098F80010DF
:10E8A0005DBA71238DF8003098F800308DF8013092
:10E8B00098F801308DF8023098F8023004268DF86F
:10E8C00003304FF0050B4FF4017A012907D00329DB
:10E8D0005ED002297AD00179012974D03BE0B8F8E2
:10E8E000011083464DBA04211046FCF77BF918B19C
:10E8F000A5F50070033812D0BBF842000421FCF7E4
:10E9000071F908B155450AD0BBF842000521FCF762
:10E9100069F9010040F207202ED085422CD19BF8E6
:10E920002210584631B3A5F50075033D1BD0012DCB
:10E930000AD0042D0BD198F80300012802D83149E0
:10E94000887001E04FF001098DF8049005262D49EB
:10E9500001201C3988703E80324669460F98F9F7CD
:10E9600032FC204695E70121C1734FF4FA71ABF8F0
:10E970005410E9E7332441E0A5F50071033903D0D1
:10E98000554501D0854201D1132437E0312435E0CB
:10E99000B8F8011080464DBA04211046FCF722F960
:10E9A00030B35545F2D198F822000028E2D015483E
:10E9B0001C38817841B1002181701348007A8DF8AC
:10E9C000040011E002E016E0242417E08046042150
:10E9D0001046FCF707F958B15545D7D198F82200F1
:10E9E0000028C7D08DF804900526A7F800B0B3E73B
:10E9F0005545CBD1C8E70021017112243E80B0E714
:10EA0000A04400202C0B0020CC35002004494BF6FC
:10EA10005C200880091D4AF65520088070470000D8
:10EA2000B06C00400CB500212E48019100910268A5
:10EA300042F4803202604FF6FF72036803F4003341
:10EA40000093019B5B1C0193009B13B9019B9342B4
:10EA5000F3D10268920342D50121009122490A684C
:10EA600042F010020A600A6822F003020A600A6893
:10EA700042F002020A6041684160416841604168B9
:10EA800041F480614160C16A184A1140C162C16AA3
:10EA9000174A1143C162016841F080610160016859
:10EAA0000901FCD5416821F47C114160416841F4C1
:10EAB000E8114160016841F08071016001688901DD
:10EAC000FCD5416821F003014160416841F0020139
:10EAD00041604168C1F381010229FAD10CBD009166
:10EAE0000CBD0000001002400020024000F0FEFFBC
:10EAF00014080100FFF78ABF0A4810B500780728FC
:10EB000004D0094800698047022809D10748D0E9A4
:10EB100001100A30814203D2BDE81040FEF788BFE1
:10EB200010BD000060230020580000202824002091
:10EB300001490872012070479406002001490871BC
:10EB40000120704794060020032803D0042801D038
:10EB5000002070470149C8710120704794060020C9
:10EB6000012802D008B100207047024988710120B5
:10EB70007047000094060020024A002110440172F0
:10EB80007047000094230020012802D008B1002023
:10EB90007047024948710120704700009406002028
:10EBA00070B5FEF7DFFD002818D0124C0020124D82
:10EBB000124E608380B200EB400005EB800041689C
:10EBC0007068F9F724FB0028608B08D000EB400048
:10EBD00005EB8000806800B18047012070BD401CBB
:10EBE00080B260831328E5D305A003F063F800200A
:10EBF00070BD000088010020DC7201088C2000201C
:10EC0000416E20756E7265636F676E697A65642008
:10EC1000434D4420210A00001FB51E48FEF7D8FAD4
:10EC200000B101208DF800001B48FEF7D1FA00B1B9
:10EC300001208DF804001948FEF7CAFA00B101203E
:10EC40008DF808001648FEF7C3FA00B101208DF8D0
:10EC50000C0069461348FCF7C5FE00B10120124CB8
:10EC600001A9E0700F480C38FCF7BCFE00B1012090
:10EC700020710C4802A90C30FCF7B4FE00B1012051
:10EC80006070084803A91830FCF7ACFE00B1012001
:10EC9000A0701FBD9C090020A4090020DC090020F1
:10ECA000E4090020DC23002088230020F0B5CF22D7
:10ECB0000270002343700C7884700126C2700671C4
:10ECC0004F78477191F802C080F806C00223C271E4
:10ECD0000372CB7843720B7983720324C27204737C
:10ECE0004B79437304258273C5738B7903740526AE
:10ECF00042748674CB79C3740627027547750B7A04
:10ED000083754B7AC3754FF0070C027680F819C0F3
:10ED1000897A81761B20F0BD054951F8062F40F80D
:10ED2000022F4A6842600A890281897A817270479B
:10ED3000D0350020F0B5002382F8003003EBC30487
:10ED400000EB4404647834B144EA03251478660087
:10ED5000641C14708D535B1CDBB2122BEED3107845
:10ED600000281DD0002317E000200EE001EB400535
:10ED700031F810606C88F7B204F0FF0C674502D9D7
:10ED80006E8021F81040401CC0B21478E41A641E52
:10ED90008442EBDC5B1CDBB21078401E9842E3DC63
:10EDA000F0BD000010B5FAF7BFF888B1FCF71EF906
:10EDB00000280CD0FCF798F8002808D0084890F8F4
:10EDC0003800C00602D5FBF78BFB18B1012010BD3F
:10EDD00004A000E00EA002F06DFF002010BD0000B6
:10EDE000FC0C0020424D532054686520436861723A
:10EDF00067696E672050686173652053746F707324
:10EE00002041626E6F726D616C6C790A0D000000BA
:10EE1000434353204E6F204368617267696E6720D9
:10EE2000416C6C6F7765646E0D0000000C48816862
:10EE3000491C81604168491C416081684FF47A72C5
:10EE4000B1FBF2F302FB1311012902D1C168491C85
:10EE5000C1600178002901D10121017070470000D3
:10EE6000780100200C484FF47A710068B0FBF1F093
:10EE7000B0F1807F0ED220F07F414FF0E020491E9C
:10EE80004161064AF02182F8141D002181610721A9
:10EE900001617047FEE700000C0000200FE000E079
:10EEA00010B5FDF78FFEBDE810404FF41F72024908
:10EEB000024804F0EFBA00002015002000F001081D
:10EEC000124810B5016841F0010101604168104A23
:10EED0001140416001680F4A11400160016821F44E
:10EEE00080210160416821F4FE014160016821F048
:10EEF000A05101604FF47F0181600021C162FFF7E2
:10EF000091FD05494FF00060086010BD00100240FF
:10EF10000000FFF0FFFFF6FE08ED00E00C4810B522
:10EF200000880B4A0021243A02F022FE08483038BB
:10EF3000C068F9F728FC02460B4606480649F9F76F
:10EF40006DFBF9F733FCFCF769FD0449088110BD3E
:10EF5000500000209A99999999991340380C0020F3
:10EF600010B5084C0121204600F04BF8002807D0CE
:10EF700000F0A4FE2046BDE81040012100F034B8A6
:10EF800010BD0000000400407FB50C46054601217D
:10EF90000220FFF7C3F9ADF800400020ADF804509F
:10EFA000104CADF80600ADF802006946204600F0AE
:10EFB0003FF801221146204600F02FF81D208DF861
:10EFC0000C0001218DF80D1003208DF80E008DF836
:10EFD0000F1003A8FEF7C6F90121204600F007F83C
:10EFE0007FBD000000040040C94301827047002932
:10EFF000018802D041F0010101E021F0010101800E
:10F00000704702460020138A92890B4202EA0102ED
:10F0100002D0002A00D001207047002A828901D046
:10F020000A4300E08A43828170478185704700006F
:10F0300030B502881B4B1C4C98420DD0A0420BD01F
:10F04000B0F1804F08D0194DA84205D0184DA84204
:10F0500002D0184DA84203D122F070054A882A43F5
:10F06000154DA84206D0154DA84203D022F4407594
:10F07000CA882A4302808A8882850A880285984243
:10F080000AD0A04208D00E4A904205D00D4A9042C4
:10F0900002D00D4A904201D1097A01860121818274
:10F0A00030BD0000002C014000340140000400404D
:10F0B00000080040000C0040001000400014004018
:10F0C0000040014000440140004801400A4800213E
:10F0D000428D4AB10722C273027B521CD2B2027324
:10F0E000102A00D1017370470177C173C172017694
:10F0F0004174808CFDF79ABA500B002070B51B4C00
:10F100000125002025756076E07B01280AD1607A10
:10F11000102807D1FDF765FAE07B012802D1607A5B
:10F12000102807D0207908B1E07818B1A07801281C
:10F1300006D007E096202086E5760220A07001E048
:10F14000607930B1607A20B1E07B042803D1E08B94
:10F1500008B900F0F3FAE07A012806D1E07B06282E
:10F1600003D1BDE8704000F0E9BA70BD500B00203B
:10F170002DE9F041274CA078012849D0264F387955
:10F18000012802D1E07A012842D0FDF779FA2085E2
:10F1900020483830FDF73AFA1E4E002538363078D0
:10F1A00000F0F001A173E584A18CA7F842103D7135
:10F1B000A178012700F00F00022901D100B9A77042
:10F1C000E07A012801D100F0B9FAA07B00281FD114
:10F1D0003078124B00F00F01A184012009E000BF3C
:10F1E000E28C16F800C003F802C0521C401CE284F6
:10F1F000C0B28842F4D900F06BF938B1E7742946FF
:10F200006174A08CBDE8F041FDF710BA0921F7E761
:10F21000BDE8F081500B0020A04400209C38002065
:10F2200070B5194C0026A07801281CD00125657501
:10F23000FDF726FA208504F13800FDF7E7F904F11F
:10F240003800A1780078022900F00F0001D100B940
:10F25000A570E07A012801D100F070FA0B486677BA
:10F260006570057170BD607F401CC0B26077022878
:10F27000F8D301F02BFC00F035F866770448A6704F
:10F28000E673067070BD0000500B0020A044002003
:10F29000F00B002010B5104C207868B104F1380054
:10F2A00041782171807828B17F2800D97F20401CC7
:10F2B000C0B200E0012060712079E0706079A07137
:10F2C0000020207200F09CFA207A10B10320E07335
:10F2D00010BD0420FBE70000500B002000487047E1
:10F2E0009C38002007480021C1738170C172C1752C
:10F2F00001760175417541768176C1760177017499
:10F3000081757047500B002010B5064CA07AFDF7B0
:10F31000DDF904F13800FDF7B9F94620A085012098
:10F32000607610BD500B002070B5164C00260728E3
:10F33000E08301D8667201E0102060720125A5709B
:10F340002684E07D012805D00C206074FDF78EF93D
:10F35000A67070BD607A10B1102803D004E000F0F0
:10F36000B9FA01E000F06CFAE571A07AFDF7AEF9A8
:10F3700004483830FDF78AF9E5734620A0856576A4
:10F3800070BD0000500B002010B500F0D3FBBDE8AD
:10F39000104000F0D3B900000B48417B29B101298E
:10F3A0000FD002290FD100F0A7B9C18CA1F602013C
:10F3B00049428186408D072801D300F0A9B800F0AA
:10F3C0002DB900F079B97047500B002070B51F4D72
:10F3D000A5F138042978687801F00F0140EA01208E
:10F3E000A08440F60201608588420BD90D2161742A
:10F3F000FDF71CF90220207400F042FA002020746E
:10F40000E07370BD0828FCD300F062F8B8B1104B6F
:10F410000220E18C2A5C401C5A54628D491C521E09
:10F420006285C0B2E1840728F3D901252573A08C39
:10F43000FDF7D8F8E572BDE8704000F021BA092167
:10F440006174A08CBDE87040FDF7F0B8880B002017
:10F450009C38002070B50F4B0F4DA3F1380418787D
:10F4600000F00F01A184012006E0E28C1E5CAE5486
:10F47000521C401CE284C0B28842F6D900F028F841
:10F4800030B100216174A08CBDE87040FDF7CEB8AA
:10F490000921F7E7880B00209C3800200A480A4918
:10F4A0004FF000020078A1F1380110F0F0008873ED
:10F4B000CA84CA740549C87603D0102803D1FFF75F
:10F4C00085BFFFF7C7BF7047880B0020A04400200E
:10F4D0000E4A00201146937B098D43B1102B0ED0AC
:10F4E000202B0FD0302B09D1032907D305E0928CB4
:10F4F000002A03D0521C914200D3012070470829F2
:10F50000FCD3FAE7528D072AF9D2F3E7500B00201B
:10F51000F0B51E481E4E0121838E1E4C00F1380CA2
:10F52000072B1ED2C18601220EE000BFC58C1CF83D
:10F53000027067556D1CC584458D6D1E4585C58E51
:10F540006D1C521CC586D2B29A42EFD9428D0AB9BF
:10F5500086F8211041730822C27301760021C1840C
:10F56000F0BD0122C38C1CF80250521CE5545B1CF8
:10F57000C384438DD2B25B1E4385072AF2D9180497
:10F58000000CEDD186F82110F0BD0000500B0020DA
:10F59000A04400209C38002070B51F4C608E38B30A
:10F5A000607D002836D00025657504F13806257782
:10F5B000307810F0F000A0731CD010281AD020284A
:10F5C00028D1FFF785FFE8B13078217B00F00F00EC
:10F5D000884219D16573FFF7DFFE9620608601200F
:10F5E0002077607B002815D1BDE87040FFF76EBD25
:10F5F00003200AE00620607400F050F8BDE8704077
:10F60000FFF74CBF092000E004206074BDE87040A3
:10F6100000F044B870BD0000500B0020F0B51C484D
:10F6200001231C4D868E418D00F138048E4215D386
:10F63000CEB2012109E0C28C675CAF54521CC28477
:10F64000428D521E491C4285C9B2B142F3D9408D48
:10F65000002802D1104880F82130F0BDC386012176
:10F660000CE0C28C675CAF54521CC284428D521EA7
:10F670004285C28E521C491CC286C9B2B142F0D921
:10F68000022141730821C17303760021C184F0BDBA
:10F69000500B00209C380020A044002010B5054CE1
:10F6A0000146A08CFCF7C2FF0020E073E0722076D8
:10F6B00010BD0000500B002030B50D48017E002920
:10F6C00014D10C4C00F13803C18E07290AD8C28C22
:10F6D0005D5CA554521CC284428D521E4285491C59
:10F6E000C186F1E7002141730721C17330BD0000DD
:10F6F000500B00209C38002070B50E48017E002978
:10F7000017D190F82A1000F138040B4D491C09E07C
:10F71000C28CE65CAE54521CC284428D521E42859D
:10F720005B1CC386C38E8B42F2D900214173072133
:10F73000C17370BD500B00209C38002070B52C4C5C
:10F7400000212246E37B0320527D092B1CD2DFE8F7
:10F7500003F0050C10141C202A383C00002A13D09A
:10F760006175BDE87040FFF799BEBDE8704000F0DC
:10F7700075BABDE8704000F037BA00F041F8207A61
:10F78000002801D10420E07370BDBDE8704000F096
:10F79000F3B9A179491EC9B2A1710129F4D8E07366
:10F7A0006079A07170BD227D01203AB12175A176EA
:10F7B0000721E17396216186207770BDE18D49B103
:10F7C00070BDBDE87040FFF7E7BE638E13B132B184
:10F7D00061750B206074BDE87040FFF75FBFFFF7F5
:10F7E000DBFD607B0028EBD1BDE87040FFF76EBC0D
:10F7F000500B002001490120C8757047500B0020B4
:10F800000E48017A29B1012915D0022915D100F03D
:10F810003DB90A4AC179383241F020011170018C9A
:10F82000A1F6020149428186C08B072801D300F06E
:10F8300079B800F0B7B800F001B97047500B00205C
:10F8400030B50D480D4CC18BC1F3032242F01003BB
:10F8500000F13802137051700221038CE55C55549D
:10F860005B1C0384C38B491C5B1EC9B2C38307297D
:10F87000F3D90821817230BD500B00209C38002044
:10F8800010B5134C142204F13801207C40F03000F4
:10F890000870002048708A7060840320A072CC2217
:10F8A0000A54401CC0B20728FAD90820A0720020D0
:10F8B000FCF712FFA07AFCF709FF05483830FCF787
:10F8C000E5FE0620E0734620E0850120A07610BD0D
:10F8D000500B0020F0B51149012001F13804CA8B0A
:10F8E000227003460E4F08E00D8C401CC0B27E5DB6
:10F8F000E6546D1C5B1C0D84DBB215469342F3D9B4
:10F900006A1C8A72072807D8CC222254401CC0B235
:10F910000728FAD908208872F0BD0000500B00209B
:10F920009C3800202DE9F0411C4C1D4904F138029F
:10F93000A38E072B1AD20125E58628460CE0268CDB
:10F940008F5D1754761C2684E68B761EE683E68E42
:10F95000761C401CE686C0B29842F0D9257200257C
:10F96000E575FCF7C1FE2584BDE8F0810120238CFC
:10F97000CD5C15545B1C2384E38B401C5B1EC0B222
:10F98000E3830728F3D90820A072FFF7BDFC042009
:10F99000E073BDE8F04100F0BBB80000500B002060
:10F9A0009C3800202DE9F041224C234B04F1380112
:10F9B000A28EE58B4FF00100AA4220D3EDB20122C6
:10F9C0000BE0268C401CC0B29F5D8F54761C2684B1
:10F9D000E68B761E521CE683D2B2AA42F1D9A572FA
:10F9E000CC2202E00A54401CC0B20728FAD90820F1
:10F9F000A072FFF789FC0420E073BDE8F081E08687
:10FA000001200CE0258C5E5D0E546D1C2584E58B79
:10FA10006D1EE583E58E6D1C401CE586C0B29042EC
:10FA2000F0D9022020720025E575FCF75DFE2584E3
:10FA3000E3E70000500B00209C38002070B5114C0B
:10FA4000E07D01281CD1104A04F13803E08E07281C
:10FA50000AD8218C555C1D54491C2184E18B491E18
:10FA6000E183401CE086F1E70820A072FFF74CFC20
:10FA7000002020720420E073BDE8704000F048B818
:10FA800070BD0000500B00209C3800202DE9F04193
:10FA9000174CE07D012828D194F83600A17FC2B22E
:10FAA0000844C1B2A17204F13803124E0BE0258C58
:10FAB000521CD2B2775D1F546D1C2584E58B6D1EE0
:10FAC000E583401CE086E08E8842F0D3CC20072AF4
:10FAD00003D89854521CD2B2F9E70820A072FFF75D
:10FAE00013FC002020720420E073BDE8F0810000C8
:10FAF000500B00209C38002010B5FCF7B7FD0348E0
:10FB00000021C1738170C175017510BD500B0020BB
:10FB10000748C179491CC9B2C171102901D100211E
:10FB2000C1710179002902D0C178491EC1707047A6
:10FB3000500B00200F48417E012903D1818D09B16E
:10FB4000491E8185817E012903D1C18D09B1491EDC
:10FB5000C185C17E012903D1018E09B1491E0186EB
:10FB6000017F012904D1418E002901D0491E41861F
:10FB700070470000500B002070B51A4C0126A08D74
:10FB8000D0B1207DA17D084326D00025657625755E
:10FB9000E08B98B1207908B1E078A8B16079B0B174
:10FBA000012814D002281AD016D9A079A0F101009A
:10FBB000A0714FF0050013E0304600E02846607465
:10FBC000BDE87040FFF798BF2570022008E0FFF7FE
:10FBD00017FE207A08B1A67570BDA57570BD03200B
:10FBE000E07370BD500B002070B51B4C208EB0B17F
:10FBF000607D00282FD0002004F13801607509785D
:10FC000001F0F002A273302A25D1E07601F00F0551
:10FC1000FFF75EFC28B1032D05D305200EE002207E
:10FC20000CE009200AE0022D07D0012D0BD0002D99
:10FC300011D1BDE87040FFF72DBB08206074BDE80E
:10FC40007040FFF759BF07206074FFF755FF9520FC
:10FC500020860120E07670BD500B00200B49012268
:10FC6000888D68B1087D002809D000200875487685
:10FC70004B7A43B1102B02D10A700220C87370472F
:10FC80004A74104600E04874FFF736BF500B00205E
:10FC9000094A29B192680068904204D8101A04E019
:10FCA0009168016003E0C0431044884201D3012001
:10FCB0007047002070470000780100200D4810B503
:10FCC000407B012815D03220FBF770FD002810D1B1
:10FCD0002A20FBF76BFD00280BD1074C2068018818
:10FCE0000648FFF7A2F920684068804720688068CE
:10FCF000206010BD28240020C434002000040040EF
:10FD000030B52C4C2078012852D12B490122C868EB
:10FD1000401CC8600A70002323700524B0FBF4F572
:10FD200004FB1504002C43D1002841D00A24B0FB69
:10FD3000F4F504FB15044A7004B98A701424B0FB6E
:10FD4000F4F504FB150404B9CA703224B0FBF4F5D1
:10FD500004FB150404B90A716424B0FBF4F504FB38
:10FD6000150404B94A714FF4FA74B0FBF4F504FBBE
:10FD7000150404B98A714FF47A74B0FBF4F504FBEE
:10FD8000150404B9CA7140F2DC54B0FBF4F504FB6D
:10FD9000150404B90A724FF4FA64B0FBF4F504FBDD
:10FDA000150404B94A7241F27072904200D3CB60DC
:10FDB00030BD000078010020101500200FB512485A
:10FDC00001880A2901D3002101800288009900EBF3
:10FDD0000212516002889DF8041000EB02121172A9
:10FDE00002889DF80D1000EB021251740188DDF8B5
:10FDF000052000EB011141F8092FDDF809204A60C8
:10FE00000188491C01800FBDA040002070B510483A
:10FE1000006800281BD1FAF7C5FD002817D00D4C4B
:10FE200021886088814212D000250A2800D365808D
:10FE3000608804EB0010001D0FC801F02AF9064885
:10FE40000121817080F82A506088401C608070BD5C
:10FE50004C0B0020A0400020A044002010B5044C12
:10FE60000146204601F0A8F820880006FCD510BD08
:10FE7000004C00402DE9F041384C40F225573946FE
:10FE8000204601F007F8364D002690B1204601F0DB
:10FE90008FF8C1B2A88AC82804D2324A1154401C33
:10FEA000A88200E0AE820A292FD03946204600F011
:10FEB000DAFF40F224473946204600F0EBFF38B124
:10FEC000AE82204601F074F83946204600F0CBFFA0
:10FED00040F227752946204600F0DCFF18B129467C
:10FEE000204600F0C0FF40F226652946204600F07B
:10FEF000D1FF18B12946204600F0B5FF0821204661
:10FF000000F0C1FF012805D00BE0FEF749FEAE82EC
:10FF1000BDE8F0810821204600F0A2FF204601F054
:10FF200047F80421204600F0AEFF012806D1042145
:10FF3000204600F095FF204601F03AF802212046C5
:10FF400000F0A1FF0128E3D10221204600F088FF44
:10FF50002046BDE8F04101F02BB80000004C004005
:10FF600088010020921D002070B5314D40F22556C9
:10FF70003146284600F08EFF2E4C98B1284601F0FD
:10FF800017F8C2B2208B0021C82804D22A4B1A5479
:10FF9000401C208300E02183E182E1703146284645
:10FFA00000F061FF40F224463146284600F072FF1F
:10FFB00040B1284600F0FCFF0120E07031462846A1
:10FFC00000F051FF40F2266631462C46284600F0EC
:10FFD00061FF18B13146204600F045FF0821204658
:10FFE00000F051FF012806D10821204600F038FF1B
:10FFF000204600F0DDFF0421204600F044FF0128E8
:020000040801F1
:1000000006D10421204600F02BFF204600F0D0FF4F
:100010000221204600F037FF012808D102212046A6
:1000200000F01EFF2046BDE8704000F0C1BF70BD6B
:1000300000500040880100205A1E002010B5094CD5
:10004000207F00280DD0E07F10280AD1A07F00F08B
:1000500037FA00202077BDE81040FF210248F8F76A
:10006000CBB810BDA04400209C38002010B5074C30
:10007000207F002808D0E07F112805D104F12B0053
:1000800000F0AAFA0020207710BD0000A044002054
:1000900010B50A4C207F00280FD0E07F14280CD127
:1000A000032104F12B0000F0E7FA00202077BDE8DF
:1000B0001040FF210248F8F79FB810BDA04400206F
:1000C0009C38002010B5064C207F002806D0E07F29
:1000D000192803D100F0F6F80020207710BD0000A9
:1000E000A044002010B5064C207F002806D0E07FF9
:1000F000222803D100F04CF90020207710BD000029
:10010000A044002070B5104C207F00280ED0E07F66
:1001100027280BD194F82B0000250C4A04F12B0161
:10012000022804D0012000F0E1FA257770BD0220FA
:1001300000F0DCFA05482577801F84F8215040F84C
:10014000065F456070BD0000A0440020B60B002093
:1001500010B50A4C207F00280FD0E07F28280CD152
:10016000022104F12B0000F0B7FB00202077BDE84E
:100170001040FF210248F8F73FB810BDA04400200E
:100180009C38002010B5094C207F00280DD0E07F5E
:100190002E280AD106480088401E81B2054800F08A
:1001A00021F9002084F82100207710BDA044002010
:1001B000760B00209D38002010B50A4C207F0028C7
:1001C0000FD0E07F31280CD1032104F12B0000F087
:1001D000F3FB00202077BDE81040FF210248F8F72C
:1001E0000BB810BDA04400209C38002010B5074C6F
:1001F000207F002808D0E07F3E2805D104F12B00A5
:1002000000F028F90020207710BD0000A044002055
:1002100010B50A4C207F00280FD0E07F85280CD134
:10022000012104F12B0000F0FDFB00202077BDE848
:100230001040FF210248F7F7DFBF10BDA0440020A7
:100240009C380020044A81781170C078491C1170D4
:10025000801C507070470000B60B002006480178E3
:10026000012908D141780C2903D20C3050F8210023
:100270000047002101707047B40B002002490120A3
:10028000087000F023BC0000B40B002002490020DD
:10029000087000F01BBC0000B40B00207047000089
:1002A000074801214177002180F8221000F8061F3D
:1002B000C17241878177C17780F8211070470000B3
:1002C000A044002070B52F484178012959D919213F
:1002D00001702D4C00214170B4F8420002281BD35C
:1002E00094F82B0004F12B0600F07F050B2D3DD276
:1002F000DFE805F03C060627143C143C3C3C270094
:100300002846FAF75DFC80B3B4F8420003211FE0F1
:100310001E49FCF707FA31E013212CE02846FAF7D2
:100320004FFC10B3B4F842000621FAF75BFC00283A
:10033000F2D0324629461548FBF758FD0328E7D886
:1003400011E02846FAF73CFC78B1B4F842000221EB
:10035000FAF748FC0028DFD0324629460B48FBF765
:1003600045FD0028D4D1312101E0FFE71221207999
:10037000012803D111B11920FCF7B8F90A20A4F81B
:10038000460070BD0A0C0020A04400200047002059
:10039000114810B5407801281DD9104C0321B4F83C
:1003A0004200FAF71FFC78B10D48FBF7A3FD0328C4
:1003B00003D30B49FCF7B6F90AE02079012807D1ED
:1003C00000202071312100E013212220FCF78EF95A
:1003D0001E20A4F8460010BD0A0C0020A0440020F6
:1003E0000047002070B5064617480D4640780128A2
:1003F00028D9164C2079012824D1607F00220321BE
:10040000FAF7C2FBB8B1032D01D2132114E0AD1EDF
:10041000A9B23046FEF7D2F908B101460CE00C480B
:100420006E2101703178417071788170014603202E
:10043000FCF778F903E07F212E20FCF757F92820FC
:10044000A4F8460070BD00000A0C0020A044002063
:100450000047002070B5054616484078012827D986
:10046000154C0221B4F84200FAF7BCFBC8B1297858
:1004700011F07F0F03D0207901280ED015E0084637
:10048000FAF7AAFB88B10D487E21017029784170E6
:1004900001460220FCF746F907E0002020711221F6
:1004A00000E013213E20FCF721F90A20A4F84600C1
:1004B00070BD00000A0C0020A0440020004700206E
:1004C0002DE9F04707464148417801297BD91021A1
:1004D00001703F4C002580464570B4F8420002216F
:1004E000FAF780FB002865D007F07F06012E07D0C1
:1004F000022E05D0032E03D02079012856D05DE0CE
:10050000607F4FF00109032804D001281AD0022887
:100510001FD019E0022E17D1207901284ED1FAF709
:1005200067FB68B1E07B58B16677FEF7E3FA84F8C1
:100530000C90C82084F8009084F8200078213AE0DC
:10054000222138E0022E06D0032E0CD0012E07D037
:1005500009E0032EFAD1207901282FD17E212AE04B
:10056000FCF72EFBE5736677A4F8405084F8225020
:10057000A5716574032E05D084F8245084F82550A5
:1005800084F827503846FAF727FBB8B111485021B4
:100590000170477085703221C17080F80490F42199
:1005A000417106200B49FCF7BDF807E025711221C7
:1005B00001E008E013211020FCF798F80A20A8F8C1
:1005C0000400A4F84600BDE8F08700000A0C0020F3
:1005D000A0440020004700202DE9F04107462248B2
:1005E000417801293ED911210170002545701E2155
:1005F0001E4C81800221B4F84200FAF7F3FA50B39E
:10060000387800F07F00FAF7D3FAF0B1FAF7F0FA91
:10061000C8B13878FAF7E0FA154E38B15120307089
:100620003878707031460220FCF77CF81148017967
:10063000012902D105713570757001202070C82024
:1006400084F820000BE0222106E02079012806D161
:100650002571122100E013211120FCF747F80A2030
:10066000A4F84600BDE8F0810A0C0020A044002058
:10067000004700206844002070B519494A78012AD3
:100680002CD914220A701E228A800178427809042B
:10069000807801EB0221134C0D180421B4F84200BC
:1006A000FAF7A0FA98B16FF07F40854208D1FAF7C7
:1006B000A1FA0D49542008700120FCF733F80AE034
:1006C0002079012807D100202071312100E0132179
:1006D0001420FCF70BF80A20A4F8460070BD0000B7
:1006E0000A0C0020A0440020004700202DE9F05F04
:1006F000DFF8D8A1002490469AF801000E460128A0
:1007000076D973480179012972D181460122407F4F
:100710001146FAF739FA00287ED0307800254FF0DC
:10072000010BAAF10A07012807D002283FD0B9F827
:100730004200022871D2132451E03D70A8464C4675
:10074000B9F842000221FAF74DFA0028F3D0E07818
:10075000012809D05F4D672028703078687094F8C0
:100760002200012802D004E0372438E0A0790128D3
:1007700002D0607C18B10CE0C5F8028009E0534853
:100780000938FBF71BFB84F811B0D7F80100C5F856
:10079000020087F800B084F806B067218AF80010DC
:1007A0008AF801804B490620FBF7BCFF1BE089F863
:1007B0001150B9F842000621FAF714FA0028BAD00D
:1007C00099F82810032906D8387810B1012813D0D9
:1007D00013E0032900D33624387858B11CB12146E0
:1007E0002720FBF783FF1E20AAF80400A9F8460083
:1007F000BDE8F09F2424F2E73D70364C33490422D3
:100800002560A58009392046F7F71AFD88B33078AE
:100810002E4A401EC0B201E056E053E0521F111FA5
:10082000FBF776FA20B1122447F8015FBD80D6E7C6
:10083000717888F80010B17888F80110F17888F89C
:100840000210317988F80310204940460422491FDC
:10085000F7F7F6FC002848460CD090F82810FF293E
:1008600002D2491C80F82810C9B202291BD83524AD
:10087000DAE725E080F8285067212170327862702D
:100880003278022A0DD0022280F823208AF8001044
:100890008AF8015089F822B00E490220FBF742FF86
:1008A00003E00122F0E7032903D047F8015FBD8090
:1008B00099E736240A2180F8291089F803B0B3E7B4
:1008C0002424B1E712248AE77F2488E70A0C002059
:1008D000A0440020004700202DE9F041334F064698
:1008E000682038703248417801295CD9282101708C
:1008F0001E21304C81800122607F1146FAF744F9B5
:100900000025C0B3B4F842000321FAF76BF998B39D
:10091000FAF76EF988B3307810F07F01707805D05F
:10092000032903D0207901282BD039E0012805D0F4
:10093000032803D02079012820D031E011B1032908
:1009400007D00DE0012884F8245009D084F8255000
:1009500006E00121012884F8241001D084F8251034
:100960003078FAF739F9D8B1307878700F49022029
:10097000FBF7D8FE14E00BE008E005E0257131211B
:100980000BE02571122108E0222106E0132104E08A
:100990002079012804D125717F212820FBF7A6FEAC
:1009A0000A20A4F84600BDE8F081000000470020BE
:1009B0000A0C0020A0440020F8B50646164A002084
:1009C000ADF8000050780D46012823D93120107071
:1009D000124C1E209080207901281BD10122607FBB
:1009E0001146FAF7D1F840B16B460D4A2946304618
:1009F000FDF742FF010001D104E07F213120FBF728
:100A000075FE04E00649BDF80000FBF78BFE0A20E6
:100A1000A4F84600F8BD00000A0C0020A044002005
:100A20000047002070B5054625484178012946D980
:100A3000852101701E21234C81800122607F114697
:100A4000FAF7A2F8002670B3B4F842000221FAF7D0
:100A5000C9F830B3FAF7CCF850B1287800F07F002D
:100A600001280BD0022805D02079012816D023E0D8
:100A700022211EE0012084F8270001E084F827608D
:100A80002878FAF7A9F8B8B10F48C521017029787C
:100A9000417001460220FBF745FE0DE02671122150
:100AA00007E0132105E0FFE72079012804D1267132
:100AB0007F218520FBF71AFE0A20A4F8460070BDAE
:100AC0000A0C0020A0440020004700200448002118
:100AD0000222017042700122827081807047000002
:100AE0000A0C002010B5084C207F00280BD0E07FB6
:100AF00000F00EF800202077E077BDE81040FF21DD
:100B00000248F7F779BB10BDA04400209C380020B4
:100B1000084910B5497801290BD9074C21790129D9
:100B200004D1002121711121FBF7E0FD0A20A4F876
:100B3000460010BD0A0C0020A04400202DE9F04121
:100B40001446054669B1092927D13348017800299F
:100B500023D000210170BDE8F041FF212F48F7F7B5
:100B60004BBB2F4802274178012906D0022914D116
:100B700021782C4E102923D025E0054601782078D5
:100B800001F1400282420AD12046272904D141784E
:100B9000012901D1FFF756FB6F70BDE8F0817F2876
:100BA000FBD160788142F8D1A078782804D0FFF793
:100BB0006DFB03206870F0E71E20A8800420F9E791
:100BC00047706078B0772178174B184AF17700208A
:100BD0001F5C8F4208D1342901D0362902D1144933
:100BE000098829B9507003E0401CC0B20C28EFD32B
:100BF0000C2801D10B2050700A4814212B300746D5
:100C0000F7F7FAFA1422611C3846F7F7DCFA0120EC
:100C10003077A6F84250C0E7510B00209C380020E6
:100C20000A0C0020A04400206A780108B40B0020C0
:100C30007A0B002001490120487070470A0C0020FF
:100C400070B5154C40F22551204600F023F90028DC
:100C50000ED0204600F0ACF9C2B2104881890B04D6
:100C600006D44C044FF0000306D50A2A01D0838134
:100C700070BD41F400410DE00D2A09D0C1F30D040F
:100C8000074D491C89B22A558181C729EFD870BD0B
:100C900041F48041818170BD00380140880100200D
:100CA000041B002010B5044C0146204600F084F9D6
:100CB00020880006FCD510BD0044004070B5304CC3
:100CC00040F225563146204600F0E4F82D4D88B11B
:100CD000204600F06DF9EA89C0B2FE2A04D22A4902
:100CE0008854521CEA8101E00020E8813146204608
:100CF00000F0B9F840F224463146204600F0CAF828
:100D000040B1204600F054F9012068703146204679
:100D100000F0A9F840F226652946204600F0BAF80E
:100D200018B12946204600F09EF80821204600F020
:100D3000AAF8012806D10821204600F091F82046A3
:100D400000F036F90421204600F09DF8012806D174
:100D50000421204600F084F8204600F029F9022101
:100D6000204600F090F8012808D10221204600F02A
:100D700077F82046BDE8704000F01AB970BD000059
:100D80000044004088010020CC1B002070B5314D8C
:100D900040F225563146284600F07CF82E4C98B19A
:100DA000284600F005F9C2B2608A0021C82804D2A2
:100DB0002A4B1A54401C608200E061822182A1709B
:100DC0003146284600F04FF840F224463146284686
:100DD00000F060F840B1284600F0EAF80120A07069
:100DE0003146284600F03FF840F2266631462C4650
:100DF000284600F04FF818B13146204600F033F88D
:100E00000821204600F03FF8012806D1082120469D
:100E100000F026F8204600F0CBF80421204600F030
:100E200032F8012806D10421204600F019F82046A6
:100E300000F0BEF80221204600F025F8012808D174
:100E40000221204600F00CF82046BDE8704000F07A
:100E5000AFB870BD0048004088010020CA1C0020C7
:100E6000C943018070470A0A01219140C9430180AA
:100E700070470029818902D041F4005101E021F43A
:100E80000051818170470246002012880A4200D03A
:100E90000120704730B501F01F0201240025C1F385
:100EA000421304FA02F2012B0FD0022B0FD0838AD7
:100EB0004FEA11210088134204FA01F400EA040009
:100EC00001D000B10125284630BD8389F0E7038AAF
:100ED000EEE710B5C1F3421301F01F040121A14058
:100EE000012B07D0022B07D01430002A026805D04E
:100EF0000A4304E00C30F8E71030F6E78A4302605A
:100F000010BD000030B50446008A85B00D464CF691
:100F1000FF710840E98801432182A1894EF6F31050
:100F20000140A8882A8910436A890A431043A08196
:100F3000A08A4FF6FF410840A9890143A182684673
:100F4000FDF716FA1948844201D1039800E002988F
:100F5000A189090400EBC00101EB0010296801D54B
:100F6000490000E08900B0FBF1F06422B0FBF2F12F
:100F700009010B096FF018056B4300EB8300A3898F
:100F80001D044FF0320306D503EBC000B0FBF2F0B6
:100F900000F0070005E003EB0010B0FBF2F000F0FA
:100FA0000F000843208105B030BD0000003801402B
:100FB0008088C0F308007047C1F308018180704742
:100FC00010B500F02BF9BDE81040FDF737B900F07F
:100FD0004DBA000004480088034A0449121F1288D1
:100FE00042EA0040C8607047BC6C0040900B002093
:100FF00002F0EDBE02F024BF0A484FF0E022816803
:1010000019B99169084B594381609169826843F22B
:10101000856311441A44826088B202EB820140EA7F
:1010200001407047900B00200DE37A0570470000E7
:10103000034900200978C90700D00120704700004B
:101040002C0B0020034900200978890700D50120D6
:10105000704700002C0B002001460020A1F5E06243
:10106000B43A00D1012070470FB41FB50DF1230130
:10107000069800909DF822208DF804200DF10500BF
:10108000F7F7A1F89DE80F0000F03EFA1FBC5DF8ED
:1010900014FB0FB585B000208DF808009DF81820CE
:1010A00005998DF80A2000918DF809000DF11901BC
:1010B0000DF10B00F7F787F8684602F0BBFC09B0AA
:1010C00000BD0000074810B54178002909D1012171
:1010D0004170FCF7A9F9F9F7ADFFBDE81040FAF748
:1010E0006DB810BD900B002010B52A48284CC1687F
:1010F000E2792948F7F767F82748227827A16B3863
:10110000F7F761F82448627828A15D38F7F75BF8B3
:101110002148A27828A15138F7F755F81E482279BE
:1011200028A12B38F7F74FF81B48E27828A145385B
:10113000F7F749F8184862792CA12138F7F743F8F6
:101140001548A2792CA11738F7F73DF81248A27A72
:101150002FA15F30F7F737F80F48217A0A30F7F7F9
:101160004BF80D4800216B3800F8E81F41708C21C6
:101170000171A0214171142101725021417213218A
:1011800001738821417319210174417410BD00005D
:10119000FA770108900B00203B35002032313039BE
:1011A0003134302D535A3031000000003839323696
:1011B00020202020202000004443552020202020F3
:1011C0002020000048573A312E302E430000000006
:1011D00053573A312E30302E435F32343032303470
:1011E0005F383932365F3030000000007878787828
:1011F000787878780000000078787878787878784F
:1012000078787878787878787878787878000000C6
:101210005232583030303031000000002DE9F05F9C
:10122000644CDFF894B1654920785D4640F00100D8
:101230002070DBF80400F7F768F8F7F790FADFF8AA
:1012400080A1A0729AF8100060725E48808F010A37
:10125000E1722073E868F7F782FA010A6173A073FC
:1012600059480126022700780025DFF860910728F9
:1012700066D0D9F810008047022863D0E573DFF804
:10128000508198F8030001285ED000285ED0042029
:10129000FAF78CFA00B1677498F80400012857D067
:1012A000002857D00320FAF781FA00B127744F467F
:1012B0004849D9F80000F7F728F8F7F750FA010A7B
:1012C000A174E0749AF80E00C8B3002020750120C4
:1012D000FAF76CFA217860F3041121F0E000207035
:1012E0003020FAF763FA617860F300016170312011
:1012F000FAF75CFA617860F3410161700320FAF754
:1013000055FA617860F3820161700320FAF74EFAB2
:10131000617860F3C30161700420FAF747FA6178DD
:1013200060F3041161700420FAF740FA61784646D0
:1013300060F34511617098F8010088B90EE00BE088
:10134000E6739CE7E7739AE76574A5E76674A3E71D
:101350002674ACE72574AAE70120B7E7B07810B18E
:1013600041F0400001E021F0400020F0800060707A
:10137000A570DBF80C00F7F7F2F9A0803078A071C7
:1013800078688047E0711448257200780228207838
:1013900003D240F00200207006E020F0020020702E
:1013A00002D940F0040001E000F0FB002070BDE82D
:1013B000F09F0000CC350020380C002000002041B8
:1013C00028240020C80600206023002058000020A8
:1013D0008823002000401C46900B00200848094943
:1013E00010F8EC2FCA7042780A714279037902EB47
:1013F0000322CA80427A007A02EB002008817047FB
:10140000D03400202C0B002030B5164885B0016880
:10141000001D0068814223D01249134A103900246C
:10142000086120464FEA0D0300EBC00102EB4101C9
:10143000097B092903D1411C1955641CE4B2401CE5
:10144000C0B21228F0D3074812210C3084720B303E
:101450000546F6F7D1FE224669462846F6F7B3FE62
:1014600005B030BD200B0020E43500202DE9F0410F
:10147000214C0127207820B9FFF736FEFEF710FF38
:1014800027701E4D0026287890B195F8200020B1D5
:10149000401E85F82000BDE8F08119482E700168D3
:1014A000184A01F4E06111430160BFF34F8FFEE77A
:1014B0006088401C80B26080022807D36680FEF7F7
:1014C000DDFEEF71EE7600F055F8E680A088401C56
:1014D0000004000CA08004D0A680FEF7BFFEFBF73E
:1014E000C3F8FEF793FCFAF7E7FFF9F7E7FABDE870
:1014F000F041FEF7D3BE0000A80B0020A04400205E
:101500000CED00E00400FA050FB40098A0F5E061CE
:10151000DF3907D0A0F5E061343903D080B204B0E0
:1015200000F04CB812480188322901D30021018013
:101530000288009900EB0212516002889DF80410A5
:1015400000EB0212117202889DF80D1000EB0212DE
:1015500051740188DDF8052000EB011141F8092FD5
:10156000DDF809204A600188491C018004B07047F9
:10157000444100202DE9F0410D4C00270D4E0E4D49
:1015800010E0322800D367806088307004EB0010D0
:10159000001D0FC8FCF77CFA6088401C608028683A
:1015A000401C2860218860888142EAD1BDE8F08132
:1015B00044410020A00B0020A40B00200D4910B5D1
:1015C0000978C90710D00B4900230839A1F1140488
:1015D0000A68B0F5827F08D0A0F58070113803D179
:1015E00022F002000860238110BD22F00100086093
:1015F000E38010BD2C0B00202DE9FE4F15460E4652
:101600000746FBF7DFFADFF894C2A54C002F5ED047
:10161000012F7DD19CF80800E246002878D130786F
:10162000D6F8011040EA01206061F7F701FDFBF7F1
:10163000C9FA2A469BA0616900F03CFBD4E9050188
:10164000814266D0A061A5F10D00E16981460B18C9
:10165000C3F30A02D90A99A0E36100F02BFBFAF761
:101660005BF9218CE069DFF884B2B1EBD02F0BD0AD
:10167000C10A5844C70A2184FF0239469CA000F0E1
:1016800019FB3846FAF7C6F84FEAE97109EB917091
:10169000C0F38708371DA807B0F1804F0CD09BA07E
:1016A00000F008FB70190322FF210938F6F79DFDB1
:1016B00008F1010000F0FF0879480024426A02EBBB
:1016C0000B010091C1694FF0010B416275E0357962
:1016D000257072796270D6F806004FF6FF7800BA6E
:1016E00020F0FF03707A0343636071892181307BAE
:1016F000D6F80D7040EA0720E060378A27824FF065
:10170000FF36A6610026E6616662A4F8208001E04B
:101710004AE0BEE08CF80860CDE900100297294647
:1017200080A000F0C7FA2089228AE1688DE80700CE
:10173000627821788A48636800F0BCFABDE8FE4F01
:10174000F7F7A8BC5FF0000557F824100098FAF7E7
:10175000B9F8042808D06D1CEDB2032DF4D381A094
:10176000009900F0A7FA1DE00098006801901CB1F4
:10177000A8F10100844206DBDDE9001357F82420BC
:1017800081A000F097FA57F82410019881420DD0FB
:1017900085A000F08FFADDE9001357F824207AA025
:1017A00000F088FA8AF808B0BDE8FE8F0098001DA6
:1017B0000090032D03D2641CE4B24445C2D3FBF76E
:1017C00001FA1FFA89F15546BAF82C20301DF7F7B7
:1017D000E9FC334CA885024621897CA000F06AFA16
:1017E000FBF7F0F9E1686069884250D12089AA8D41
:1017F000904204D0BDE8FE4F7DA000F05BBA002708
:1018000085A000F057FA8D4E3046FAF703F8DFF85E
:10181000308230464146FAF755F8042807D07F1C3D
:10182000FFB2032FF5D3314686A000F043FA3768A4
:1018300031463B46424654A000F03CFA47451AD197
:101840007E4F00263F1D38466168FAF73BF80428B2
:1018500007D0761CF6B2032EF5D3394682A000F0ED
:1018600029FA3E683946334689A0626800F022FAB8
:101870006068B04202D085F808B095E7FBF7A2F99E
:10188000F7F7D6FB8BA000F015FAFBF7B1FDF9F7DF
:10189000F5FFBDE8FE4FFBF795B900008801002079
:1018A000DC1A00200A0D43757272204261673A25E6
:1018B000642C206C656E2025640A0D0057726974D3
:1018C000652D616464723A20736563746F722025BC
:1018D000642C2C6F6666736574202564202C7265F9
:1018E000636C656E202530640D0A000000600208FC
:1018F0003434437572722045726173652D2D6164B5
:1019000064723A202530780D0A0000000A0D6C61DF
:1019100073742D2D2D2D2D6261672121212121210F
:10192000210A0D000D0A3636365570642D2D747956
:1019300070653A2564202C7665723A25642C5462D1
:101940007974653A25642C204372633A25642C50DF
:1019500061673A25642C506C656E3A25640D0A0067
:1019600078780108213232212121212121212121D0
:1019700057726974652D4661696C2D616464723AB1
:10198000202530780D0A00006164647220253078CB
:101990002C2C5772697465202530782C2C72656167
:1019A00064202530780D0A000A0D20726561647686
:1019B000616C20213D20557064646174615B695DD8
:1019C0002921212121210A0D000000003132325548
:1019D0007064486561642E46696C654372633D2599
:1019E00030782C544372633D2530780D0A00000096
:1019F000557064486561642E46696C654372632066
:101A0000213D205443726320212121207265747589
:101A1000726E210D0A0000002121217570642D696C
:101A20006E666F21212057726974652D746F747012
:101A30006167202564200D0A00000000005802089C
:101A40004433221155706444617461466C616721AE
:101A50002057726974652D4661696C2D61646472EA
:101A60003A202530780D0A002121217570642D69F6
:101A70006E666F21212057726974652D4661696C0D
:101A80002D616464723A202530780D0A0000000050
:101A90003161646472202530782C2C57726974652A
:101AA000202530782C2C72656164202530780D0A51
:101AB0000000000032327570642D616C6C2077720A
:101AC000697465204F4F4B4B2121726573746172AD
:101AD0007421212121212121212121210D0A000010
:101AE00030B50D46094CC1B041F20D01A4F8051006
:101AF00001462A46E01DF6F766FB658040AA694666
:101B00002046F9F71FFB41B030BD0000221F002026
:101B1000FEE7000070B50E4D0224286F816A8847E9
:101B200030B1286F816A884700B10024204670BD1B
:101B3000084805210546FCF7DDFD0028F6D02620E3
:101B4000F9F742FE2846FCF7E7FD0124EEE7000026
:101B5000C80600206434002010B50C46801AF6F741
:101B6000E3FD2146F6F703FCF6F7F9FD80B210BD60
:101B70002DE9F041194D01EB4106294601EB8604A0
:101B8000904615F8262061880027CAB199B1142023
:101B9000B1FBF0F06080F6F7D5FD4FF06632104BE8
:101BA000F6F7CAFC6FF00B02F6F7A7FDF6F7FEFD9D
:101BB000A060C8F80000678005F82670BDE8F081D5
:101BC00022790844521CD2B222716080142AF5D1C5
:101BD000012005F826002771F0E70000480C0020DE
:101BE00066660A4010B50121CC022046FCF7A2FB34
:101BF0002046BDE810400021FCF79CBB07490020AF
:101C0000086007490878401CC0B208701E2803D835
:101C100002497F200839086070470000082C004006
:101C20007401002043E0322100BF00BF00BF00BFAD
:101C300000BF00BF00BF00BF00BF00BF00BF00BFAC
:101C400000BF00BF00BF00BF00BF00BF00BF00BF9C
:101C500000BF00BF00BF00BF00BF00BF00BF00BF8C
:101C600000BF00BF00BF00BF00BF00BF00BF00BF7C
:101C700000BF00BF00BF00BF00BF00BF00BF00BF6C
:101C800000BF00BF00BF00BF00BF00BF00BF00BF5C
:101C900000BF00BF00BF00BF00BF00BF00BF00BF4C
:101CA00000BF491E11F0FF01BED1401EC0B2002886
:101CB000B9D170470FB4054B10B503A9044A029877
:101CC00000F044F910BC5DF814FB0000313F01083E
:101CD000F00400200FB4084B10B504A902AA039821
:101CE00000F034F9044602A9002000F0C6FC2046AA
:101CF00010BC5DF814FB00007B26010830B528B14C
:101D0000144C031F002021680A4605E0084630BD38
:101D10009A4203D810465268002AF9D1002800D010
:101D200041680BD00468A3EB0005A54204D11B68F1
:101D30001C440346046002E0436000E023603AB1C3
:101D40001C68D51AA54203D115682C441C60526842
:101D50005A6030BD100C00202DE9F04782460F4C30
:101D600010480D4E0E4F001B4FF0000820F00705E5
:101D70004FF0010900221146504602F0E1FD002813
:101D800002D1306810B10020BDE8F0873C60C4E9A2
:101D90000058C6F80090EDE7140C0020844700209E
:101DA000100C00208067002002E008C8121F08C144
:101DB000002AFAD170477047002001E001C1121FCC
:101DC000002AFBD1704700002DE9FF5F82B000219F
:101DD000DDE90430020DDDF840B0034318D044F6CD
:101DE0001050A2F2FF3242431514119801281FD05F
:101DF000A5EB0B00401C5FEA000A4FF000064E4FB7
:101E0000DFF83891B046504615D5CAF1000413E00A
:101E1000119801244AA3012801D16FEA0B0102980D
:101E2000119AC0E90031C0E9024206B0BDE8F09F56
:101E3000CBF10000DFE704460021404A491842EB9D
:101E40000450CDE9001012E0E00707D032463B46CF
:101E500040464946F6F770FB8046894632463B4687
:101E600010461946F6F768FB06460F466410002C2C
:101E7000EAD1DDE90401DDE90023BAF1000F06DA59
:101E8000F6F75AFB42464B46F6F756FB05E0F6F7E7
:101E9000C5FB42464B46F6F7C1FB04460E46002200
:101EA000284BF6F7B9FD03D84FF0FF30014607E0A5
:101EB0000022254B20463146F6F797FAF6F793FDB8
:101EC000102409E0002C0ADB0A220023F6F7B4FCF8
:101ED000039B30321A55641E50EA0102F2D1641C91
:101EE000039AC4F111031444119A012A03D0012268
:101EF00008430DD10AE0084304D000204FF0110B35
:101F0000119072E7A3EB0B056D1E0DE05B4504DD40
:101F10004FF0000205F1010504E003DA4FF0000282
:101F2000A5F10105002AECD002981199C0E902310F
:101F3000C0E9004579E70000000014400000F03FD0
:101F4000300000000000F0430000E03F2DE9FF4FAB
:101F500095B09B468946064600250FE2252877D195
:101F600000242746F84A0121059400E0044316F8AE
:101F7000013F203B01FA03F01042F7D130782A28C4
:101F800011D06FF02F033078A0F13002092A16D853
:101F9000059A44F0020402EB820203EB4202104471
:101FA000761C0590EFE759F8042B0592002A03DA16
:101FB000504244F40054059044F00204761C3078FA
:101FC0002E2816D116F8010F44F004042A280DD04B
:101FD0006FF02F023078A0F13003092B09D807EBFE
:101FE000870302EB4303C718761CF3E759F8047B19
:101FF000761C30786C280FD006DC4C2817D0682867
:102000000DD06A2814D104E0742810D07A280FD19A
:102010000DE044F400140AE044F4801401E044F4B8
:1020200040147278824202D104F58014761C761C2A
:10203000307866280BD013DC582877D009DC0028CC
:1020400075D04528F6D04628F4D047281AD19DE10E
:1020500018E0632835D0642879D0652812D195E13D
:10206000702873D008DC6728F1D069286FD06E28FB
:102070000DD06F2806D1B5E073282CD0752875D007
:10208000782874D05A46179990476D1C75E1C4F3AF
:102090000250022809D003280DD0D9F800100428D6
:1020A0000DD00D6009F1040967E1D9F80010EA17B5
:1020B000C1E90052F6E7D9F800100D80F2E70D7083
:1020C000F0E719F8041B8DF8001000208DF80100CE
:1020D000EA46012003E059F804AB4FF0FF306107F6
:1020E0004FF0000102D40DE008F101018846B94229
:1020F0000FDA8045F8DB1AF808100029F4D108E05F
:1021000008F1010188468142FADB1AF8081000291B
:10211000F6D105985B46A0EB080721463846179A8A
:1021200000F094FA284400EB080507E04DE029E1AF
:102130000DE01AF8010B5A4617999047B8F10108BB
:10214000F7D25B4621463846179A13E142E00A224D
:102150000092C4F302524FF0000A022A08D059F844
:1021600004CB032A4FEAEC710AD00DE029E02AE003
:1021700009F1070121F00702F2E802C1914609E0E6
:102180000FFA8CFC4FEAEC71042A03D14FFA8CFC55
:102190004FEAEC71002907DA0A460021DCF1000C55
:1021A00061EB02012D2202E0220504D52B228DF8DD
:1021B0000420012203E0E20701D02022F7E7904645
:1021C00059E00A2102E010220DE010214FF0000A30
:1021D00000910BE010224FF0000A44F0040408279D
:1021E000009203E008224FF0000A0092C4F302526A
:1021F000022A05D059F804CB0021032A08D009E0AF
:1022000009F1070121F00702F2E802C1914605E059
:102210001FFA8CFC042A01D10CF0FF0C4FF00008CF
:10222000220728D5702806D0009B83F0100353EABC
:102230000A0305D00EE040228DF80420012208E0B8
:102240005CEA010206D030228DF804208DF80500EA
:1022500002229046009B83F0080353EA0A030AD146
:102260005CEA010201D1620705D530228DF8042015
:102270004FF001087F1E582804D034A003900EA808
:1022800002900DE036A0F9E753466046009AF6F753
:10229000D3FA84460398825C0298401E0290027032
:1022A0005CEA0100F0D1029806A9081A00F1200AA0
:1022B000600702D524F4803400E00127574502DD91
:1022C000A7EB0A0000E0002000EB0A01009005984F
:1022D0004144401A0590E00306D45B462146179A14
:1022E000059800F0B3F90544002706E001A85A4616
:1022F000C05D179990476D1C7F1C4745F6DBE003D6
:102300000CD55B462146179A059800F09FF90544C5
:1023100004E030205A46179990476D1C0099481EDA
:1023200000900029F5DC08E0029802995A460078EE
:10233000491C0291179990476D1CBAF10001AAF14E
:10234000010AF1DC65E10000092801003031323377
:1023500034353637383961626364656600000000E1
:1023600030313233343536373839414243444546CB
:102370000000000000F058F90544761C3078002871
:102380007FF4ECAD19B02846BDE8F08F620700D4A9
:10239000062709F1070222F0070CFCE80223E146B8
:1023A00003F000485FEA080C02D00FF2702C0DE039
:1023B0005FEA045C02D50FF2682C07E05FEAC47C98
:1023C00002D00FF2602C01E0AFF2700C4FF0FF383A
:1023D00023F00043CDF850C065280CD006DC45281A
:1023E00009D046281DD047283DD13DE0662818D0A9
:1023F00067287ED138E00021112F01DB112000E099
:10240000781CCDE9000106A90EA8FFF7DDFCDDE987
:102410000F010E9A03910021009207F1010A049125
:102420004DE04FF000400097CDE9011006A90EA83D
:10243000FFF7CAFCDDE90F0203920E9B11990022FF
:10244000DDF80CA00093049211B9791C00EB010A8D
:10245000B7EB0A0004D4C0F1FF3007F1010A049081
:10246000AAEB0700019044E0012F00DA01270021C8
:10247000112F01DD112000E03846CDE9000106A949
:102480000EA8FFF7A1FCDDE90F010E9A03910021D0
:1024900004910092BA4621070CD40399514500DA01
:1024A0008A46BAF1010F05DD009AAAF10101515CDB
:1024B000302908D0B84202DA10F1040F06DA0121FF
:1024C000CDE9011015E0AAF10101E9E7002805DCDA
:1024D000049901440491AAEB000102E0411C51451A
:1024E00000DD8A460499401A401C01904FF00040DC
:1024F0000290200704D40198504501DBCDF80480F8
:1025000000208DF84F0002980DF14F07B0F1004FF9
:1025100025D02B200E9002984FF0020800280CDAEC
:10252000404202902D200E9007E00A210298F6F713
:102530006DF93031029007F8011DB8F10001A8F1E2
:102540000108F2DC02980028EFD1791E0E9808707D
:10255000307800F0200040F0450007F8020D12A886
:10256000C01B00F107081498007800B1012000EBAF
:102570000A01019801EBE07105984144401A401EA0
:102580000590E00306D45B462146179A059800F0B3
:102590005DF805441498007818B15A461799904789
:1025A0006D1CE00324D55B462146179A059800F080
:1025B0004DF805441CE00498002807DBDDE9030121
:1025C000884203DD0098405C179901E0179930209C
:1025D0005A469047049805F10105401C0490019863
:1025E000401E019004D12E205A46179990476D1C29
:1025F000BAF10001AAF1010ADDDC05E017F8010BD0
:102600005A46179990476D1CB8F10001A8F10108CE
:10261000F4DC5B462146179A0598ABE62D000000D6
:102620002B000000200000002DE9F04104460025A9
:102630001E461746880404D405E039462020B047DA
:102640006D1C641EF9D52846BDE8F0812DE9F041E6
:10265000044600251E469046C80301D5302700E0F9
:102660002027880404D505E041463846B0476D1C54
:10267000641EF9D52846BDE8F0810A68531C0B603A
:1026800010707047F0B40C4905244A680E68531C5A
:1026900093FBF4F504FB1535B54203D1F0BC07A05C
:1026A000FFF708BB044D0835A85493FBF4F004FB76
:1026B00010304860F0BC7047E00A00204576656E37
:1026C000742071756575652069732066756C6C0A78
:1026D00000000000F0B58DB001F0BBF82E4E0025D3
:1026E0002E4C24E09DF824300AAA03A80899F7F795
:1026F000BFFA8DF81F5001203070079803AF00908B
:1027000097E80F0000F0D4F901280ED123481422D5
:1027100003A91438F5F757FD2048CDE901561438C0
:10272000016900910FC800F079F9FAF74BFA676870
:1027300027B309AB0AAA08A90020B8470028D1D1BD
:102740001CE000BF9DF824300AAA03A80899F7F7F7
:102750008FFA8DF81F50FEF76BFC30B1079803AE6F
:10276000009096E80F0000F033F9079803AE009050
:1027700096E80F00FEF778FCFAF724FAE66936B11E
:1027800009AB0AAA08A90120B0470028DAD100F055
:10279000B9FF0DB0F0BD0000E8000020C01400201B
:1027A00070B520211B48F5F727FD1A483021303835
:1027B000F5F722FD01F046F8FAF780FAFAF7B6FAD3
:1027C000144A1549303A0020FAF768FB10B113A0FB
:1027D000FFF770FA0F4A1049183A34390120FAF716
:1027E0005DFB10B113A0FFF765FA0A4C303CE568B9
:1027F00025B100231A4619461846A847646A002CDA
:1028000007D0A4460023BDE870401A4619460120AF
:10281000604770BDF01400204001002063616E31FC
:1028200020D0ADD2E9B3F5CABCBBAFB3C9B9A60DD0
:102830000A00000063616E3220D0ADD2E9B3F5CA60
:10284000BCBBAFB3C9B9A60D0A00000000B50D4965
:10285000A1B041F20B020020A1F80520401C80B27B
:102860002828FBD3502048800749087C401C087466
:1028700006A0FFF71FFA20AA69460248F8F762FC93
:1028800021B000BD221F0020A820002053656E64E7
:102890002063656C6C2074656D70200A0D0000006B
:1028A00010B51149A2B041F20C02A1F80520002098
:1028B00001F2EA2213180C18401C93F8973080B2EA
:1028C000E3710828F6D3082048800849087C401C9A
:1028D000087407A0FFF7EEF920AA69460248F8F746
:1028E00031FC22B010BD0000221F0020A8200020D3
:1028F00073656E6420626D735F73746174655F6984
:102900006E666F0A0D00000010B51249A2B041F2C8
:102910000A02A1F80520002001F2EA2200EB4003A0
:102920000C181344401C93F8213080B2E37128281E
:10293000F4D3282048800849087C401C087407A06C
:10294000FFF7B8F920AA69460248F8F7FBFB22B066
:1029500010BD0000221F0020A820002053656E64D7
:102960002063656C6C2074656D70200A0D0000009A
:102970002DE9F05F0024134EDFF84CB0DFF84CA0D7
:10298000054640F227474FF00109A04656F834109B
:10299000286888420FD106EBC400416809B1284677
:1029A00088472868B84204D15846FBF7B5FE8AF834
:1029B0000C90C5F80080641C64B2102CE6D3BDE80E
:1029C000F09F00000C050020AC34002028240020DB
:1029D0000FB4142210B502A90D48F5F7F4FB0C4C06
:1029E0001422214601F51270F5F7EDFB802109480C
:1029F000F9F747F90848016820468847142120461E
:102A0000F5F7FAFB0020206010BC5DF814FB000015
:102A1000E80C002000100140080500200FB470B53C
:102A2000214C0A9D607814280BD200EB800004EB47
:102A30008000142204A9001DF5F7C5FB6078401C36
:102A40006070059941F6EC4218480024B2EB114F32
:102A500010D19DF81B10102904D0132902D0112980
:102A600003D005E09DF81E1001E09DF81C10817058
:102A70000A210EE041F6EB42B2EB114F0AD19DF86C
:102A80001B108278914203D114210161847001E00E
:102A900032210161054800210C30FDF7F9F82C7056
:102AA00070BC5DF814FB00009C0D00209800002015
:102AB0000FB4142270B504A92748F5F784FB264DFE
:102AC00026484FF0FF366C68C461A0B2A0F574418F
:102AD000563903D0304670BC5DF814FB41F6EC412A
:102AE000B1EB144F03D0491EB1EB144F06D11A4974
:102AF000142201F17800F5F766FBEBE718498C42E8
:102B00001AD018498C4217D017498C4214D0174953
:102B10008C4211D016498C420ED016498C420BD0F3
:102B200015498C4208D015498C4205D014498C4275
:102B300002D014498C420CD10749142201F1B4008F
:102B4000F5F741FB0449AA7A00230B31204600F037
:102B500091FB0020BFE70000D40C0020980000206B
:102B600056F4261856F4011856F4071856F40818A7
:102B700056F40A1056F4121856F41D1856F41F088D
:102B800056F41A1056F41A1810B5134C13490020B5
:102B9000C4E900010421217260720520A072FF22A5
:102BA000082104F10B00F5F720FB0D4A32F8411F14
:102BB0005088E172090AC0F57A6021736073000AD7
:102BC000A073107908B1022000E00120E073BDE895
:102BD0001040014800F00CBF600D0020F4561018A2
:102BE000C80600202DE9F04101462E4C00250422A4
:102BF0000823022604F10B0001293CD002294FD101
:102C00002949C4E9005122726572A372FF2208218A
:102C1000F5F7EBFA254F0120E07237F8330F2073F8
:102C2000000A60737888C0F57A60A073000AE073C8
:102C3000B8882074000A6074B879A074204600F047
:102C4000D7FE0320F8F70BFBE672F888000A207322
:102C5000387A0A306073B7F80900A073000AE0738D
:102C6000B7F80B002074000A6074A574BDE8F04149
:102C70000C4800F0BDBE0E49C4E9005122726572D5
:102C8000A372FF220821F5F7B0FA1020E0720D20A0
:102C900020736573A673FF20E07325740620E3E7B5
:102CA000BDE8F081600D0020F456EB1CC806002042
:102CB000F456EC1C2DE9F04101462D4C0025042270
:102CC0000823022604F10B00012938D002294CD137
:102CD0002849C4E9005122726572A372FF220821BB
:102CE000F5F783FA244F0120E07237F8460F20737E
:102CF000000A60737888A073000AE073B8882074B3
:102D0000000A607497F82600A074204600F070FE58
:102D10000320F8F7A4FA97F82600C0F16400A7F89A
:102D20000700E6722073000A6073A573E5732574CB
:102D30006574A574BDE8F0410D4800F059BE0F4917
:102D4000C4E9005122726572A372FF220821F5F7CF
:102D50004CFA1020E072092020736573A673FF20DF
:102D6000E073257411206074E3E7BDE8F081000092
:102D7000600D0020F456EB1CC8060020F456EC1C35
:102D800070B50C4C05460C490020C4E90001042133
:102D9000217260720220A072FF22082104F10B0050
:102DA000F5F723FAE572280A20732046BDE8704043
:102DB00000F01EBE600D0020F45627182DE9F04FDC
:102DC00085B0054614216846F5F716FA714C0821BE
:102DD0000026042204F10B004FF0100B4FF00709FE
:102DE0004FF00208012D7CD0022D7BD16A4B924618
:102DF000C4E9006322726672A172FF22F5F7F5F949
:102E0000664D0127E772A8782073E8786073287907
:102E1000A0736879E073E8882074000A6074287AE7
:102E2000A074204600F0E4FD0320F8F718FA84F8B7
:102E30000B802889000A2073A87A6073E87AA0734F
:102E4000287BE073687B20746674A674204600F0CB
:102E5000CFFD0320F8F703FA0320E072277384F80C
:102E60000D80A87CA073E87CE073287D2074687DC9
:102E70006074A87DA074204600F0BAFD0320F8F726
:102E8000EEF94748FF22112180F887616846F5F77F
:102E9000ACF984F80BA0E87D2073287E6073A673DC
:102EA0009DF80000E0739DF8010020749DF8020079
:102EB00060749DF80300A074204600F099FD032083
:102EC000F8F7CDF90520E0729DF8040020739DF815
:102ED000050060739DF80600A0739DF80700E0737D
:102EE00001E03FE03BE09DF8080020749DF80900F8
:102EF00060749DF80A00A074204600F079FD03205C
:102F0000F8F7ADF90620E0729DF80B0020739DF8EC
:102F10000C0060739DF80D00A0739DF80E00E07327
:102F20009DF80F0020749DF81000607484F812B0B2
:102F3000204600F05DFD0320F8F791F984F80B902E
:102F40000A2121730B21617384F80E90E020E07355
:102F5000FF2020746074A0740E4800F049FD05B095
:102F6000BDE8F08F0F4BC4E9006322726672A17254
:102F7000FF220821F5F739F984F80BB031202073CE
:102F8000667384F80E90FF20E073267484F8118035
:102F9000A674E1E7600D0020F456EB1CC806002083
:102FA00020150020F456EC1C70B50B4C05460B495F
:102FB0000020C4E900010421217260720120A07286
:102FC000FF22082104F10B00F5F70FF9E572204606
:102FD000BDE8704000F00CBD600D0020F4560910F3
:102FE00010B5134C13490020C4E9000104212172DB
:102FF00060720720A072FF22082104F10B00F5F790
:10300000F4F80D4890F86C10E17230F8661F2173E7
:10301000090A61734188A173090AE1730179217476
:10302000407960742046BDE8104000F0E1BC00002B
:10303000600D0020F4561C18C806002070B5484DDD
:1030400048490020C5E9000104212972687207205F
:10305000A872FF22082105F10B00F5F7C6F82B2016
:10306000F8F7A4FB404C18B92C20F8F79FFB28B1C7
:1030700094F85B0020F00300401C03E094F85B0030
:1030800020F0030084F85B002D20F8F78FFB18B9BF
:103090000C20F8F78BFB28B194F85B0020F00C00B3
:1030A000001D03E094F85B0020F00C0084F85B0046
:1030B0002E20F8F77BFB002894F85B0020F030000E
:1030C00000D0103084F85B000B20F8F76FFB00286D
:1030D00094F85B0020F0C00000D0403084F85B0022
:1030E0000E20F8F763FB18B91A20F8F75FFB28B138
:1030F00094F85C0020F00300401C03E094F85C00AE
:1031000020F0030084F85C0094F85900012894F83A
:103110005C0020F00C0000D1001D84F85C0094F8E5
:103120005A00012894F85C0020F0300000D11030E3
:1031300084F85C0014F84F0FE87260780A30287346
:10314000A0786873E0780A30A8732079E873207B50
:103150002874607B6874BDE87040014800F048BC8A
:10316000600D0020F4561318C806002070B53E4DBF
:103170003E490020C5E900010421297268723C4CD7
:10318000A972204694F86C1090F86100642920F030
:10319000030000D1401C84F861002F20F8F706FBE3
:1031A000002894F8610020F0C00000D0403084F87E
:1031B00061001A20F8F7FAFA18B90E20F8F7F6FAB3
:1031C00028B194F8620020F00300401C03E094F85A
:1031D000620020F0030084F862000B20F8F7E6FAA2
:1031E000002894F8630020F0030000D0401C84F80D
:1031F00063000320F8F7DAFA18B90420F8F7D6FAD2
:1032000028B194F8630020F00C00001D03E094F84E
:10321000630020F00C0084F863002E20F8F7C6FA53
:10322000002894F8640020F0030000D0401C84F8CB
:1032300064000120F8F7BAFA002894F8640020F03E
:103240000C0000D0001D84F8640014F8610FE872CF
:1032500060782873A0786873E078A873BDE8704040
:10326000014800F0C5BB0000600D0020F4561910A5
:10327000C80600202DE9F0411F4616460C460546BB
:10328000F7F78AFA574A2846A91A574D90424FD065
:1032900022DC564AA0EB0201904276D00BDC544966
:1032A000401871D05349C8426BD12078A876A86BDA
:1032B00040F0080064E05048081825D0B0F5C02F51
:1032C0005FD13A4631462046F7F748F9002858D0F2
:1032D000A86B40F0020053E0B1F5202F46D0B1F5C5
:1032E000901F52D0B1F5A81F5ED0B1F5F01F48D1A4
:1032F00021463246032E00DD03223B48F4F763FFEC
:10330000A86B40F480403BE02078E870607828713A
:10331000A0786871E078A8712079E87160792872E6
:10332000A0796872E079A872A86B40F0010027E0EC
:10333000208868826088A882B4F904004FF47A611A
:10334000884202DDA0F57A6001E0C0F57A60E8828B
:10335000B4F90600884202DDA0F57A6001E0C0F50C
:103360007A602883A86B40F0040009E03A463146B1
:103370002046F7F7C3F8002803D0A86B40F01000F0
:10338000A863BDE8F08100E01CE0207885F8230008
:10339000607805F8240FA0786870E078A8706869F4
:1033A00040F020006861ECE7207905F8340F60797F
:1033B0006870A079A870E079E870686840F0400013
:1033C0006860DEE7207885F82700607805F8280F28
:1033D000A0786870E078A870286940F080002861C3
:1033E000CFE7000056F40818FC0C002056F41A1021
:1033F000AA0BE0F7000015F8000019F870B50F4CA3
:103400008318A34201D9032070BDA2B10124002377
:103410000BE005780E78AE4204D0FF2D01D00220DB
:1034200070BD0024401C491C5B1C9342F1D3012C4D
:1034300001D0012070BD002070BD00000000020816
:10344000F8B501210820FAF781FF03248DF8024026
:1034500014250F4F8DF803504FF48066ADF80060CF
:1034600069463846F8F786FB8DF802407400ADF8DF
:1034700000408DF8035069463846F8F77BFB31462B
:103480003846F8F7FEFB21463846F8F7FAFBF8BD58
:10349000000C01402DE9F0418846054614462249BA
:1034A0002044884202D90120BDE8F081CCB3E00776
:1034B00000D0541C224641462846FFF79FFF0028B3
:1034C000F2D0012080F31088F8F726FA3520F8F7BB
:1034D0009BF9E80AC002F8F79DF9074640F2E73089
:1034E000401E80B2FCD200260FE000BF08EB460170
:1034F00018F81600497840EA01212846F8F7C6F97D
:103500000746042804D1AD1C761CB6EB540FEDD34E
:10351000F8F7B4F9002080F31088042F02D00220BD
:10352000C2E7FFE70020BFE70000020810B54FF038
:10353000000140B1054C2046F6F77AFE2046F6F72A
:1035400061FB012010BD024CF5E70000006800405F
:103550000064004030B4022814D20B4A00EB800310
:1035600002EB83021569002D0CD00A7A8B7A042AAB
:1035700006D00C6801F10B022146AC4630BC604716
:103580004C68F7E730BC70478C0F002010B538B19D
:10359000044800BFF6F7F0FE042800D1FF2010BD5C
:1035A0000148F7E7006800400064004030B402289A
:1035B00015D20C4A00EBC00302EB83040122E3683E
:1035C0008A4013420BD09343064AE36000EB80032A
:1035D000483252F82320002A01D030BC104730BCBA
:1035E00070470000440F002010B518B1F6F752F9EB
:1035F000012010BDF6F776FDFAE7000010B583282C
:1036000012D10A4C207C01280ED0A4F13000C16AEE
:1036100009B1012088470120207404480021BDE839
:1036200010401430FCF734BB10BD0000F014002033
:1036300070B500291DD10F4E0546002406EB04107D
:103640000168A94203D100210C30FCF721FB641C66
:10365000A4B2022CF2D30848817F002909D0017C52
:10366000022906D100218177BDE870401830FCF7AF
:103670000FBB70BDEC000020F0140020044B00EBE9
:10368000C00203EB820200219160FFF74FBF0000F0
:10369000440F0020022811D2094900EB800201EBFF
:1036A00082018A68002A09D0054B00EBC001483B23
:1036B00003EB8101C96801B1012110477047000087
:1036C0008C0F002010B50446022817D2FAF7E5FF48
:1036D0000B4804EB840100EB8100C16809B120466E
:1036E0008847FAF7DCFF064804EBC401483800EBD2
:1036F0008100C168002901D00021C16010BD000017
:103700008C0F00202DE9F047254F4FF0000845466B
:1037100007F1300606EB05142078012802D00228B4
:103720002DD036E0A089062803D21E4931F81010AA
:1037300000E0C621201DFCF7ABFAF8B1FAF7ADFFA7
:10374000A089401CA08105EB450007EBC000D0F824
:103750000CC0BCF1000F04D000231A4619462846BD
:10376000E047022020704FF00109FAF798FF04F1BA
:1037700008000021FCF78CFA84F80E9009E004F1AF
:1037800008006721FCF784FA18B1A4F80C8084F8CB
:1037900000806D1CEDB2022DBCD3BDE8F0870000A7
:1037A000C0140020C47201082DE9F041022802D3A0
:1037B0000020BDE8F0810C4E00EBC00706EB87044B
:1037C0000125A560002565712371E27026F8271098
:1037D0002146E560FFF708FF18B10220A060012034
:1037E000E7E7A560E4E70000440F002070B5064657
:1037F000022807D20D4806EBC60400EB8405A86832
:10380000022801D0002070BD05F110000446F6F733
:103810000FFA21463046FFF7B9FEFF28F3D0012208
:10382000E96882401143E96070BD0000440F002048
:103830000EB58DE807006946014803F0F8F80EBDA3
:103840003412002010B500F089F8BDE8104000F0F7
:1038500033B810B500F042F8BDE8104000F088B869
:1038600030B54FF0FF34E8B1124A002352F833501C
:10387000854208D102EBC300416011B9002042F833
:103880003300002030BD5B1C142BEFD351B100235B
:1038900052F8335045B102EBC3056D6825B15B1C8E
:1038A000142BF5D3204630BD42F8330002EBC300A1
:1038B0004160E6E7B40F002010B54FF426710648CA
:1038C000F4F79AFC04492823A0310C2201F5F0708A
:1038D00003F086F8002010BDB40F00203EB5104C58
:1038E00004F5207514E06946284603F085F80021A8
:1038F000009A54F83100904207D104EBC1004368AC
:1039000033B19DE80700984702E0491C1429EFD322
:10391000284603F055F80028E5D000203EBD000001
:10392000B40F002000280CD00B4A002101EB41030A
:1039300002EB83039B682BB1491C89B21429F5D390
:103940000020704701EB410302EB830188600020F7
:1039500042F82300084670474C12002010B5F021B1
:103960000248F4F749FC002010BD00004C12002072
:103970002DE9F84300216846FCF78AF9009818B34E
:10398000012821D0DFF84880002500BF05EB450164
:1039900008EB810458F82160A76896B18FB1201D0B
:1039A0003146FCF775F901280BD1A06838B1606881
:1039B0000099091AB1FBF6F101FB06006060204690
:1039C000B8476D1C142DE1D30020BDE8F88300003A
:1039D0004C120020002803D002C00021FCF758B987
:1039E0007047002803D00068002800D001207047ED
:1039F0001CB50F490C68C4B1017A002304290ED00C
:103A0000D0F80020CDE90023427A52B100230429E6
:103A100009D0016800F10B020020A0471CBD4268DC
:103A2000F0E7837AF3E74168F4E700201CBD00006B
:103A3000C01400207CB50446FDF704FB38B9207A99
:103A4000042830D0D4F80000FDF706FB68B31C480A
:103A5000856935B3207A0022042828D0D4F80010D4
:103A6000CDE90012617A21B30023042823D0216814
:103A700004F10B020120A84798B1207A04281CD039
:103A80002568104E002400BF06EB04100168A9420F
:103A900003D100210830FCF7FBF8641CA4B2022C0F
:103AA000F2D300207CBD6068CEE701207CBD616858
:103AB000D6E7A37AD9E76168DAE76568E1E700004D
:103AC000C0140020EC0000200A4810B5418D49B117
:103AD000002141850848F9F78CFB08A0BDE810409B
:103AE000FEF7E8B8012141850348F9F762FB09A018
:103AF000F4E700008801002084090020BFAAC6F472
:103B00004143BDBBC1F7CEC2B6C8BCCCB5E7C6F712
:103B10000D0A0000B9D8B1D54143BDBBC1F7CEC233
:103B2000B6C8BCCCB5E7C6F70D0A0000094810B509
:103B3000418C41B100214184F9F796FC06A0BDE813
:103B40001040FEF7B7B801214184F6F7B1FE07A097
:103B5000F5E7000088010020BFAAC6F4BDBBC1F78D
:103B6000BCCCB5E7C6F70D0A00000000B9D8B1D546
:103B7000BDBBC1F7BCCCB5E7C6F70D0A000000001D
:103B8000704700000B4810B5C48C00210A4A01237D
:103B90004CB1C184D3710948F9F72BFB08A0BDE8EB
:103BA0001040FEF787B8C384D1710448F9F701FBD0
:103BB00006A0F4E788010020882300206C0900207B
:103BC000BFAAC6F443433143500D0A00B9D8B1D55A
:103BD00043433143500D0A000B4810B5048D0021BA
:103BE0000A4A01234CB1018513720948F9F701FB18
:103BF00008A0BDE81040FEF75DB8038511720448C7
:103C0000F9F7D7FA07A0F4E78801002088230020FD
:103C10007C090020BFAAC6F44343325F43430D0A28
:103C200000000000B9D8B1D54343325F43430D0AC9
:103C300000000000F9F7DCFB0B4810B5048C0021F4
:103C40000A4A01234CB1018493710948F9F7D1FA6A
:103C500008A0BDE81040FEF72DB803849171044818
:103C6000F9F7A7FA08A0F4E78801002088230020CC
:103C70005C090020BFAAC6F4D6B1C1F7BCCCB5E739
:103C8000C6F70D0A00000000B9D8B1D5D6B1C1F70A
:103C9000BCCCB5E7C6F70D0A0000000070477047BE
:103CA000704700000A4810B5818C49B10021818419
:103CB0000848F9F79EFA08A0BDE81040FDF7FABFE2
:103CC000012181840348F9F774FA07A0F4E70000A2
:103CD0008801002074090020BFAAC6F4C9FDD1B92B
:103CE000C4A3BFE90D0A0000B9D8B1D5C9FDD1B947
:103CF000C4A3BFE90D0A0000704770477047000079
:103D00000D4810B5C18B61B10021C1830B48F9F793
:103D100070FA0B48F9F76DFA0AA0BDE81040FDF7FC
:103D2000C9BF0121C1830548F9F743FA0448F9F7EF
:103D300040FA08A0F1E70000880100207409002083
:103D400064090020BFAAC6F4B8DFD1B9C4A3BFE993
:103D50000D0A0000B9D8B1D5B8DFD1B9C4A3BFE905
:103D60000D0A00002DE9F04104460E460D20FCF737
:103D700075F80A20FCF772F8002510E02078F8F7B3
:103D800029FC01462078F8F71DFC07460846FCF799
:103D900065F83846FCF762F86D1CADB2641CB5429C
:103DA000ECD30D20FCF75AF8BDE8F0410A20FCF7EF
:103DB00055B8002142F6DE6304E01A46521EFDD1DA
:103DC000491C89B28142F8D37047FFF739BB2DE90E
:103DD000F04115460C460646F8F784FEA020F8F799
:103DE00057FEF8F7A7FE98B9200AF8F751FEF8F742
:103DF000A1FE68B9E0B2F8F74BFEF8F79BFE38B9C0
:103E0000F8F770FEA120F8F743FEF8F793FE20B113
:103E1000F8F77EFE0020BDE8F08100246F1E09E067
:103E2000BC4201D0012000E00020F8F703FE30552D
:103E3000641CA4B2AC42F3D3F8F76AFE0120EAE7AF
:103E40002DE9F041164607460C4600252AE035B11B
:103E5000E00618D1F8F75CFE0620F7F700FAF8F74D
:103E600041FEA020F8F714FEF8F764FE88B9200A96
:103E7000F8F70EFEF8F75EFE58B9E0B2F8F708FE64
:103E8000F8F758FE28B9785DF8F702FEF8F752FE09
:103E900020B1F8F73DFE0020BDE8F081641C6D1CE8
:103EA000A4B2ADB2B542D2D3F8F732FE0120F3E7A7
:103EB00070B5174D0526A5F1080423E000F068FD54
:103EC000E8B92168685C491C91FBF6F206FB121107
:103ED0002160062813D2DFE800F0120306090C0F58
:103EE000F7F788FB0EE0F7F7C5FB0BE0F7F7CCFB25
:103EF00008E0F7F789FB05E0F7F7D0FB02E005A043
:103F0000FDF7D8FE00F044FD0028D7D070BD0000BA
:103F1000E80A0020556E6B6E6F776E206576656ED1
:103F2000742069732069676E6F7265640A0000000F
:103F30002DE9F041134C0546C1B22046FDF73CF88F
:103F400020880006FCD5104890F8A810012906D159
:103F50000E4E0027B178022904D080F8A8702846B8
:103F6000BDE8F0810A4C0B48E179962903D245540B
:103F7000491CE171F3E7FDF7B3FD307C401C307460
:103F8000E771ECE7004C004020150020A82000203D
:103F900088010020E019002038B51248006F016B3D
:103FA00088478DF8000069460F48F7F71BFD0F4C56
:103FB0000F4D012801D068B111E002212846FAF71F
:103FC00099FB60B1E07B401CE0732846FAF7A4FB44
:103FD000012038BD0020E0732846FAF79DFB002041
:103FE00038BD0000C80600200C24002060230020FB
:103FF00084340020134810B590F83800C0070DD065
:1040000011484179012907D0022141710FA000BF59
:10401000FDF750FE012010BD12A0F9E71748006916
:104020008047022801D0022010BD15480A2104460D
:10403000FAF760FB0028F7D02046FAF76DFB032063
:1040400010BD0000FC0C002074230020424D535F83
:1040500050524F544F43414C5F4742323031310A46
:104060000D000000424D535F50524F544F43414C9E
:104070005F4742323031350A0D0000005800002001
:1040800044340020104810B500698047022802D04F
:10409000012810D008E00D490020C8730C48006FBB
:1040A000016A8847042801D0002010BD09A0FDF74F
:1040B00001FE012010BD88210B48F4F79DF80BA0EC
:1040C000FDF7F8FD022010BD5800002060230020FD
:1040D000C8060020BDF8C8EBD6B1C1F7B3E4B5E718
:1040E000C1F7B3CC0D0A00003C340020BDF8C8EB8A
:1040F000BDBBC1F7B3E4B5E7C1F7B3CC0D0A00000F
:104100000D4810B5806B44F2010108420BD0F7F75F
:10411000FDFA3D210848F4F76FF888210748F4F7C5
:104120006BF8012010BD064800698047022801D0C5
:10413000022010BD002010BDFC0C00203C340020EB
:10414000580000200D4810B5C078AA2809D0FAF709
:1041500099F958B10A480069804702280BD003201A
:1041600010BD08A0FDF7A6FD012010BD0CA0FDF7B5
:10417000A1FD022010BD002010BD0000FC0C00209D
:104180005800002052455620445F43445A5F48413E
:104190004E44494E475F43524D2041410A0D0000B5
:1041A00052656164792D537461746520526563654D
:1041B0006976656420546865204368617267696E3A
:1041C000672050696C652041626F7274204D657381
:1041D000736167650A0D000010B5FAF753F948B12D
:1041E000FAF7E0FD50B1074800698047022807D080
:1041F000032010BD04A0FDF75DFDF9E7012010BD0F
:10420000002010BD5800002052756E6E696E672D3B
:1042100053746174652052656365697665642054E2
:104220006865204368617267696E672050696C65D4
:104230002041626F7274204D6573736167650A0D6A
:1042400000000000214810B5807EAA2808D0FAF7A7
:1042500019F950B12820F7F7A9FA002821D108E070
:104260001BA0FDF727FD012010BD20A0FDF722FDBA
:1042700017E00620F7F79AFA98B91C20F7F796FA94
:1042800078B92120F7F792FA58B90920F7F78EFA92
:1042900038B90A20F7F78AFA18B92620F7F786FA0C
:1042A00008B1032010BD1F4800698047022801D0D3
:1042B000052010BD1C483C210446FAF71BFA0028D3
:1042C000F7D02046FAF728FA042010BDFC0C002095
:1042D00043445A5F5F43524F20414120746F204353
:1042E00068617267696E670A0D000000537461723D
:1042F000742D5374617465205265636569766564D5
:1043000020546865204368617267696E6720506950
:104310006C652041626F7274204D657373616765CF
:104320000A0D0000580000205C34002010B506483B
:1043300005210446FAF7DEF9002803D02046FAF7F3
:10434000EBF9012010BD00007434002000B5F4F733
:1043500097FC0520FFF72DFD5DF804EBFAF738B95F
:10436000072070477047022070470000124810B5C0
:10437000018F49040DD50021816310490120487146
:104380000F480088FEF7FCFCBDE810400DA0FDF7CB
:1043900091BC0A4840F6B83108300446FBF778FC77
:1043A000002808D00CA0FDF785FC2046BDE8104091
:1043B0000021FBF76DBC10BDFC0C00207423002015
:1043C000C8060020445F43445A5F48414E44494E6A
:1043D000475F43484D0D0A004E4F2048616E64739D
:1043E00068616B65205369676E616C0A0D0000009F
:1043F00000207047704701207047704703207047C6
:104400000848007928B1012807D0022808D1F7F719
:104410008BBB02210448F7F74BBB0348F7F774BB8B
:104420007047000074230020BD2D0108052070474F
:10443000F6F702BB042070472DE9F041304E00250D
:1044400006F12807F07C012811D1F6F7E3FA70B1E4
:10445000FDF760FB58B9F4F767FD40B1FAF762F970
:1044600028B93879012802D1F4F782FE0546254C97
:10447000284694F83810490707D4F17C012901D067
:10448000B9B12BE0A17EAA2928D0FEF78DFD1E48E8
:10449000006F816A8847012528B1387918B9BD7144
:1044A0001A48F8F7A6FEF574A06B20F00400A0638C
:1044B00014E013481430007920B1012807D00228F5
:1044C0000CD108E006211248F7F7F2FA06E010488E
:1044D000F7F71AFB02E00620F7F726FBA06B81072F
:1044E00002D520F0020007E0000706D509A0FDF77D
:1044F000E1FBA06B20F00800A063BDE8F0810000A4
:1045000060230020FC0C0020C80600205C0900206D
:10451000E52B010843445A5F48414E44494E475FEA
:1045200043524D2041410A0D000000000620704713
:1045300038B51A48006FB0F90200002800DA40428E
:10454000ADF8000069461648F7F74CFA00B10120B3
:1045500014490979012902D108B1F6F7D3F91148B4
:10456000322144380446FBF793FB012806D1002092
:10457000FEF7FCFD00212046FBF78AFB0948FA21E3
:1045800034380446FBF784FB012806D10020FEF7EF
:1045900027FD00212046FBF77BFB38BDC806002025
:1045A000002400208823002070B505460846F7F750
:1045B000E7FD040062D00420812D2CD00CDC042DFA
:1045C00017D0802D5AD194F85400032856D3E16CAB
:1045D000002953D0802043E0822D13D0832D4DD16C
:1045E00094F85410032949D394F8911002292DD03E
:1045F00033E094F85400032840D32046BDE87040CF
:10460000F8F7B8B894F85400032837D3E16C0029C0
:1046100034D0822024E094F8541003292ED394F847
:10462000911002290DD194F8901094F844209142F1
:1046300000D2032084F89100227804210120FFF7A2
:10464000F7F8E16C002919D0812009E084F8910085
:10465000227804210120FFF7EBF8E16C19B18320E7
:10466000BDE870400847207800F098FA2078BDE84F
:10467000704000231A46194600F0DABA70BD70B5D2
:104680000C460546F7F77CFD00281ED090F8541024
:10469000022906D8C168002917D02846BDE8704015
:1046A000084781290AD0002C0FD1802180F85410AE
:1046B0002A46BDE870400120FFF7BAB8002C04D0AC
:1046C000812180F854102A46F3E770BDFFF7D7BF69
:1046D00010B50446F7F754FD002813D090F8541095
:1046E000022906D8C16800290CD02046BDE8104038
:1046F0000847832180F854102246BDE8104001206D
:10470000FFF796B810BD00002DE9F0411D46174691
:104710000E468046F7F734FD040030D094F854007C
:1047200003282CD3802802D1032084F8540094F865
:104730004000C00706D0A36C0BB32A46394630466A
:1047400098471CE00F48691E2A4606600571072934
:1047500003D83946401DF3F736FD04F158000949E6
:10476000054602F064F9284602F032F938B1822099
:1047700084F85400014642460120FFF759F8012011
:10478000BDE8F0819C14002010B50C46F7F7F8FC4A
:10479000002815D090F89120E1B2022A01D0032A16
:1047A0000ED190F898208A420AD1052180F8911004
:1047B00090F85410032903D3BDE81040F7F7DABF8F
:1047C00010BD0020401C80B23C28FBD37047000085
:1047D0002DE9F047504C1420012684F86C0041F27A
:1047E00088302080A670E670002525714FF0030800
:1047F00084F805804FF47A70E08041F268002081EF
:104800004220A0725920E07244202073542060732B
:10481000A573E5732674022767741920A0740B2012
:10482000E0740A2020756575A5751020E075257661
:104830006576112239A104F11A00F3F7C4FC3CA1FA
:10484000A4F134000A6840F85F2F496841604FF4D2
:10485000D27024F8330F4FF4FA70608041F22430A4
:10486000E0806E202072C820A4F809004FF47A601E
:10487000A4F80B006573E0814FF416702082A774D2
:10488000A4F81350A4F81550B4F81700DFF8AC9052
:104890006FF30B0000F5A270A4F8170014F8180FBE
:1048A0006FF0310720F0F000103004F8020B3C20CC
:1048B0002080A6703A4649460A20FDF74DF9E0707F
:1048C00084F804803A4649460520FDF745F96071B1
:1048D0000420A071E57125726572A572E5722573D9
:1048E00065732674A4F8115004F8135F6420607196
:1048F00040F25910E08040F2631020813A46494668
:104900001920FDF729F9A0723A4649461C20FDF707
:1049100023F9E072BDE8F087C80600204C565043EA
:1049200035323739584E4430313338313800000091
:10493000533030314830303100000000CDCCCC3D18
:104940002DE9F0410B3020F00706104D19E02068EA
:10495000B04215D3B0420AD9871B201DD4F8048079
:10496000F3F731FCA019C0E90078286004E0606822
:104970002860201DF3F727FC201D2660BDE8F0818C
:10498000251D2C68002CE2D10020F7E7100C002038
:104990000448D0E90010814201D101207047002075
:1049A00070470000E00A002010B50E4C62785AB142
:1049B00000206070E168C4E9030120700A20B1FBA7
:1049C000F0F080B2A08010BDFFF7C0FCE1680844A1
:1049D000E0602078411C2170092801D3012060701B
:1049E000A08810BD7C00002086B0FAF769FA4FF469
:1049F000004162B60803F8F7F1FCFAF733FA6846AB
:104A0000F9F7B6FCF8F79EFCF8F7B6F9F8F704F9F1
:104A1000FFF7DBF9F4F7BAFBF4F788F9F4F754F988
:104A20004FF47A3002F056F84FF4E13002F0AEF86D
:104A300040F2CF2140F2F310FAF7A6FAFFF7C8FED2
:104A4000FCF7C8FAF8F7CAF8FDF7AAFE39493AA008
:104A5000FDF730F9F9F76AFDF5F7AEFEF6F790FFCE
:104A6000384E394F0124B47300253D723748F8F7AA
:104A7000A0FBFC713648F8F7BCFBF8F7F5FC354CA9
:104A8000FBF73EF9FDF726FE207801281BD0607861
:104A9000012822D0A078012825D0E07801282BD049
:104AA000207901282ED0607901283ED0E0790128B4
:104AB000E6D1E571F4F74EFCF9F71AF9F9F760FB66
:104AC000FCF700FBDCE72570B07B08B1F4F7D0F908
:104AD000F4F7E4FBFCF77BFAD2E76570F9F7E2FD47
:104AE000F8F770F8CCE7A5700220F7F767FB1A49D2
:104AF000C860FCF765FAC3E7E570F6F7C5F8F6F7A6
:104B00002FFABDE72571F8F7C7FB144F38688047C7
:104B100078688047B8688047F8688047F7F7B6F844
:104B2000FAF77AF8F5F726FFAAE76571FFF7C0F9FB
:104B3000A6E70000D0720108B0E6B1BEBAC52025D4
:104B4000730D0A0074230020882300207C090020B4
:104B50006C09002010150020380C00206C0000208B
:104B600070B53AB10C4B84189C4203D8A3F500747D
:104B7000A04202D24FF0FF3070BD31B1002302E0FD
:104B8000CD5CC5545B1C9342FAD3011B92B289B22F
:104B9000FCF730FA002070BD0047002070B50546D4
:104BA000F7F7EEFA040003D094F85400022801D875
:104BB000002070BD022084F85400E16809B1284645
:104BC000884794F8910018B3D4F8A8204AB906E0B1
:104BD0000428D4F8A4000AD00321904718E0226DDD
:104BE000B2B10528F4D10021D4F8A400F5E70121E1
:104BF000F3E72946304601F0FFFE68B1D4F8A8205B
:104C00000AB9226D42B10321D4F8A400904703E011
:104C100004F1940504F17006304601F0D1FE00283D
:104C2000E7D0202104F19000F3F7E6FA012070BDEF
:104C30002DE9F0411D4616460F468046F7F7A0FACB
:104C400004002CD094F85400012828D9D4F804C0CA
:104C5000BCF1000F23D02B46324639464046E04790
:104C6000E8B1D4F88C1031B194F84530182204F131
:104C7000700001F0B5FE94F84000C00709D1D4F8E7
:104C8000881031B194F84530102204F1580001F039
:104C9000A7FE032084F854000120BDE8F081002025
:104CA000FBE710B5F7F76CFA002801D090F8540034
:104CB00010BD2DE9FF411E4615460F46F7F760FA75
:104CC00004000ED094F8540002280AD94DB194F88B
:104CD0004000C00705D104F15800804601F070FE85
:104CE00018B1002004B0BDE8F0816946404601F0EB
:104CF00083FE0028F6D0009838609DF804003070DC
:104D00009DF80420501E072804D828460DF10501FF
:104D1000F3F759FA94F85400822802D1032084F85A
:104D200054000120DEE72DE9F04786B01D46DDE99D
:104D30000E9816460F46F7F723FA04000BD094F8A6
:104D40005400022807D9082D05D804F170008246C6
:104D500001F03EFE18B1002006B0BDE8F087F9F77B
:104D60009CFC94F85400832801D0032802D2F9F760
:104D700096FCF0E7CDF8148000978DF80550CDF83B
:104D8000109016B900208DF805009DF80520501EE2
:104D9000072804D831460DF10600F3F714FAFF2076
:104DA0008DF804006946504601F041FE94F89100E8
:104DB00010B92046F7F7DEFCF9F771FC0120CBE7CC
:104DC00000207047104910B500230C464FF4805264
:104DD0000846640705D0C01D20F00700411AD1EB3A
:104DE00002020A49C1E900038118084A0839A2F100
:104DF000140221F0070111604B600B600B1AC0E92F
:104E000000139360536010BD3C240020040B00206D
:104E100030B5134900E011460A688242FBD34B6863
:104E20005C18844204D1406818444860084600E099
:104E300000BF43681C18944209D1094C143C2468F3
:104E4000A24209D052681A4442600A68126802609D
:104E5000814203D0086030BD0460F9E700BF30BD77
:104E6000040B002070B5274D04460026286898B131
:104E700000BFA4B104F00700C0F11000C1438C4290
:104E80003CD82118002939DD6868814236D81D4890
:104E900014300246146806E0FFF794FFE9E700BF0C
:104EA0002CE02046144662688A4202D22268002A18
:104EB000F7D12A68944221D00668226802606068AF
:104EC0000836421A102A05D9601842606160FFF75F
:104ED0009FFF00E000BF61686868401A6860AA68C8
:104EE000904201D2A86000E000BF41F00040606045
:104EF00000202060E868401CE86000E000BF304609
:104F000070BD0000F00A00202DE9F04F9BB005466F
:104F1000402107A8F3F770F9FE4F4FF0000AADF8F3
:104F20005CA087F810A0B5F805804FF6FF7BA8F5C8
:104F3000004020381ED0A8F5004021381AD0DFF8F4
:104F4000D8930126F54CB8F5004F7CD05FDCB8F55E
:104F5000D06F01F0F4844ADCB8F5607F74D03FDC98
:104F6000B8F1800F77D0B8F5C07F6ED0B8F5207F4C
:104F700033D192E06A882E461446B2F5967F04D863
:104F8000E448E91D3830F3F71EF9E248214638308D
:104F9000FEF7E8FE301930F8025CA01E81B2304600
:104FA000F4F716F9064602462946DDA0FCF782FE14
:104FB000B54202D0E0A001F0D0BCD64908F1E0082B
:104FC00087F811A008F0FF0022463831FCF714FBE7
:104FD000E149642088830420B8701BB0BDE8F08FDD
:104FE000B8F5906F6AD0B8F5B06FF6D17DE0B8F53E
:104FF000286F01F0B184F0DCB8F5F06FF9D0B8F5A6
:10500000086FF6D0B8F5186FE7D101F0A5BC48F2EB
:105010000701A8EB01008845F7D009DC6FF40040D8
:1050200040440628D9D2DFE800F02F38474960F81D
:10503000062806D0D1DC0128E7D00228E5D00328D5
:10504000CBD1C6A002E006E036E01DE0FCF732FE60
:1050500087F810A0C1E7E879012801D0C6A0AAE727
:10506000BE7084F8766044F86CAFAC49C4F804A014
:10507000A4F808A0A8682060E8686060BE7089F89D
:1050800000606C31C1A02DE2E879012801D0C7A0F1
:1050900091E70220B870C9A08DE7E979CCA0FCF7B0
:1050A00009FED048D5F8091040F8011FB5F80D10D9
:1050B0008180E97B817190E7CBA07CE7D0A0FCF7F1
:1050C000F9FD287A01280ED0D3A1D5A0FCF7F2FD76
:1050D000287A002881D1A048467101780029B9D1E9
:1050E0000421017079E7D1A1EFE7DFF86C8288F83D
:1050F0000660E87990B1CFA0FCF7DCFDE8790128E3
:105100000ED00028A6D12C7ACEA02146FCF7D2FDE5
:10511000D14888F804400D2C7ED057E3CFA0EBE7B0
:105120002F7AD2A03946FCF7C5FD012F76D0022F89
:1051300075D005F109000290042F71D0072F70D0AF
:10514000062F6FD0082F6ED0092F6DD00A2F6CD08C
:105150000B2FB0D00C2F69D00D2F68D04FF00A085C
:105160000E2F7DD00F2F7CD0102F7BD0112F7AD017
:10517000122F79D0132F78D0142F77D0162F76D006
:105180001D2F75D01E2F74D01F2F73D0202F72D0DB
:10519000212F71D0222F70D0232F6FD0242F6ED0CB
:1051A000252F6DD0262F6CD0272F6BD0282F6AD0BB
:1051B000292F69D02A2F68D02B2F67D0302F66D0A7
:1051C000312F7DD0322F7CD0332F7BD0342F7AD02B
:1051D000352F79D0362F78D0372F77D0502F76D003
:1051E000512F75D0522F74D0532F73D0542F72D0AB
:1051F000552F71D0562F70D0572F6FD0582F6ED09B
:10520000592F6DD05A2F6CD0602F6BD0612F6AD080
:10521000622F69D0632F0BE0D9E2D9E254E166E155
:105220006CE17AE181E19AE289E1A7E1B4E1C0E1D0
:105230005BD0642F87D0652F58D06D2F57D040F2A8
:105240002F206E2F54D06F2F53D0702F52D0712F2C
:1052500051D0722F50D0732F4FD0742F4ED017E0F3
:10526000B5E1C2E1CCE1ECE102E20EE21AE22FE2AA
:105270003BE24AE259E282E293E2A2E2A9E2A9E237
:10528000A9E2A9E2A9E2A9E2A9E2A9E2A9E2A9E2C6
:10529000752F34D0762F33D0772F32D0782F31D06E
:1052A000792F30D07A2F2FD07B2F2ED07C2F2DD05E
:1052B0007D2F2CD07E2F2BD07F2F2AD0802FDDE08A
:1052C00091E291E291E291E291E291E291E291E246
:1052D00091E291E291E291E291E291E291E291E236
:1052E00091E291E291E291E291E291E291E291E226
:1052F00091E291E291E291E291E291E291E291E216
:1053000091E291E291E291E291E291E291E291E205
:1053100091E291E2A82000207901002020150020D0
:105320000A0D44637263202530782C566372632023
:105330002530780A0D0000000A0D202844637263AE
:1053400020213D2056637263292072657475726E48
:1053500021212121210A0D00880100205265636569
:1053600069766520444542554720444344432061C3
:10537000636B0A0D000000007265676973746572E3
:105380006564206661696C65640A0D007265676911
:1053900073746572656420737563636573736564A4
:1053A0002C436F64652025730A0D00004C6F6769FC
:1053B0006E204661696C65640A0D00004C6F676978
:1053C0006E205375636365737365640A0D00000096
:1053D000686561727420636F756E742025640A0DB0
:1053E00000000000B40C00207265636569766520DA
:1053F00073746174652064617461200A0D0000009B
:1054000072656365697665206368617267652064AB
:10541000617461200A0D000044697361626C65006B
:105420006368617267652025730A0D00456E6162CD
:105430006C650000706172616D2077726974650A35
:105440000D0000005265616420706172616D206E14
:10545000756D2025640A0D00221F002070617261A5
:105460006D20726561640A0D000000007061726158
:105470006D20616464722025780A0D0071D0812F3F
:1054800070D0822F6FD0832F6ED0842F6DD0852F58
:105490006CD0862F6BD0872F6AD0882F69D0892F48
:1054A00068D08A2F67D08B2F6FD08C2F6ED08D2F26
:1054B0006DD08E2F6CD08F2F7FF4CCADB5F8091046
:1054C000A4F8DA11DDA048E1697A39B988F80560F5
:1054D00098F8002012B9042288F80020012904D08D
:1054E000DCA1DEA0FCF7E6FB77E5E0A1F9E7687A4E
:1054F000012801D0DFA05EE5E2A05CE50446F2F7FA
:1055000098FE82B2102A214605D2E248F2F75BFEED
:105510002146E1A021E1E5A0E4E76D7AEAA0294671
:10552000FCF7C8FBA4F8695019E16D7AEDA0294693
:10553000FCF7C0FB24F84D5F6580A580F4E70446C6
:10554000F2F777FE82B2102A214615D2D1481038E0
:10555000F2F739FE2146E9A0FCF7ACFB89F80060C0
:10556000E2E7F8E3F8E3F8E3F8E3F8E3F8E3F8E375
:10557000F8E3F8E3F8E3F8E3E6A0EEE0687A012860
:1055800007D084F887A0EAA00CE0EFE3EFE3EFE3B5
:10559000EFE384F88760F6E7687A012805D084F89D
:1055A00089A0E9A0FCF786FBBEE784F88960EEA03D
:1055B000F8E7697A642903D284F88A10F2A0CCE073
:1055C000F7A0FCF777FB5A2084F88A00ACE76D7AE5
:1055D0004046B5FBF0F108FB1152B5FBF8F1F6A01F
:1055E000FCF768FB84F88B509EE76D7AF8A029469B
:1055F000FCF760FB05EB8500400084F88C0093E726
:10560000B5F80950F8A02946FCF754FBB4F8592026
:1056100005EB8500B2EB400F04D90BEA4000A4F87B
:10562000830081E705EB85004100F3A0FCF742FB16
:1056300034F8590F143880B2B0FBF8F16085F5A04A
:1056400050E7B5F80950F8A02946FCF733FBB4F849
:105650005B2005EB8500B2EB400F04D90BEA40005C
:10566000A4F8850060E705EB85004100F3A095E014
:10567000B5F80950F7A02946FCF71CFB05EB85019E
:105680000BEA4100A4F859004EE7B5F80950F6A01E
:105690002946FCF70FFB05EB85010BEA4100A4F856
:1056A0005B0041E76C7AF5A02146FCF703FBF84864
:1056B0008178202901D920218170C9B201EBC10173
:1056C00000EB4101A1F807408178491C817084E416
:1056D000B5F809004146B0FBF1F2B0FBF8F108FB68
:1056E0001202A4F86300EBA066E2687A012803D0F6
:1056F000022801D0EDA05EE484F88D00012802D0DC
:10570000F0A1F1A029E0F5A1FBE7687A00EB8001A8
:105710000BEA41004146B0FBF1F2B0FBF8F108FBA7
:105720001202A4F85300EEA046E2B4F89010B4F8C8
:105730005320687A914213D94546B2FBF5F2B1FB8A
:10574000F5F1EDA0FCF7B6FAB4F853000A3880B2D0
:10575000B0FBF5F1A4F89000F2A0FCF7ABFA41E23F
:1057600000EB80010BEA41004146B0FBF1F2B0FBD7
:10577000F8F108FB1202A4F89000F0A01CE2687A8D
:1057800000EB80010BEA41006421B0FBF1F201FB68
:105790001202B0FBF1F1A4F8B300EFA0FCF78AFA13
:1057A0001BE4687A00EB80010BEA41006421B0FB46
:1057B000F1F201FB1202B0FBF1F1A4F8B100EDA08F
:1057C000FAE1697AA4F8B710F1A0C6E733E333E34E
:1057D00033E3E5E1F1E1FDE105E20DE234E23BE234
:1057E00049E258E268E274E284E288E28CE290E204
:1057F000A2E2C2E2CEE2DFE2F9E213E31EE31EE33D
:105800001EE31EE31EE31EE31EE31EE31EE31EE390
:105810001EE31EE31EE31EE31EE31EE31EE31EE380
:105820001EE31EE31EE31EE31EE31EE31EE31EE370
:105830001EE31EE31EE31EE31EE30000536F6343FB
:10584000616C6962726174696F6E2020256420202A
:10585000200A0D0064697361626C6500636861729F
:1058600067696E672025730A0D000000656E61622E
:105870006C6500006F70656E2072656C61790A0D51
:1058800000000000636C6F73652072656C61790ABB
:105890000D00000030150020626C7565746F6F7428
:1058A00068206E616D652025730A0D00626C756558
:1058B000746F6F7468206E616D65206D69737461BB
:1058C0006B652025730A0D0048656172742042657E
:1058D00061742054696D6520256420207365630A16
:1058E0000D0000004F76657254656D7056616C75E1
:1058F000652025642020200A0D0000005379735094
:1059000061726150696C65442E736E3A25730A0D9D
:10591000000000005379735061726150696C6544F6
:105920002E736E206661756C742025730A0D00005D
:10593000517569636B2043686172676520456E61CC
:10594000626C650A0D000000747269636B6C6520FF
:105950004368617267696E6720536F6320456E61AB
:10596000626C6520300A0D00747269636B6C65208F
:105970004368617267696E6720536F6320456E618B
:10598000626C6520310A0D00747269636B6C65434B
:1059900068617267696E67536F6325640A0D000062
:1059A000747269636B6C654368617267696E675393
:1059B0006F632039300A0D00747269636B6C652067
:1059C000706F7765722025642E25646B770A0D0051
:1059D000747269636B6C652063757272656E742591
:1059E00064410A0D00000000426D734D6178566FEE
:1059F0006C742564200A0D00256420426D734D618E
:105A000078566F6C74202564206661696C640A0D99
:105A100000000000426D52657175697265566F6CC9
:105A200074202564200A0D00426D734D6178437522
:105A30007272656E74202564200A0D0072657120F3
:105A40002564206F766572206D6178202564200AB8
:105A50000D000000426D734D6178566F6C74202507
:105A600064200A0D00000000426D734D617843759B
:105A70007272656E742564200A0D0000736574747B
:105A8000696E6720736F63282564290A0D00000082
:105A90009C170020754261744D6178456E65726790
:105AA000792025642E25640A0D0000004368617288
:105AB00067696E674D6F6465204661756C740A0D89
:105AC00000000000435600004368617267696E671A
:105AD0004D6F64653A2573200A0D000043430000B2
:105AE0004F766572506F776572203A25642E256473
:105AF0006B77680A0D000000526571756972655018
:105B00006F776572202564206B77204F7665725021
:105B10006F776572203A25646B772C6661756C74BB
:105B20000A0D000052657175697265506F77657274
:105B3000202564206B77200A0D00000052657175E6
:105B4000697265506F776572203A25642E25646B03
:105B500077680A0D00000000426174526174656448
:105B6000566F6C74616765203A25642E2564560A69
:105B70000D0000004261744D617843686172676591
:105B8000566F6C203A25642E2564560A0D000000DD
:105B9000426174436F756E74203A25640A0D0000EB
:105BA000B5F809004146B0FBF1F2B0FBF8F108FB93
:105BB0001202A4F85F00B1A058E3B5F8090041460D
:105BC000B0FBF1F2B0FBF8F108FB1202A4F85900A7
:105BD000B1A04BE36D7AB5A02946FCF76BF83235DE
:105BE00084F8B55044E36D7AB7A02946FCF762F813
:105BF000323584F8B650F8E3687A84F8B0000128AA
:105C000010D0022810D0032810D0042810D0052866
:105C100010D0062810D0072810D0082810D0FF2850
:105C200010D0E2E3AFA0BDE4B4A0BBE4B9A0B9E4F6
:105C3000BFA0B7E4C4A0B5E4C9A0B3E4CEA0B1E46A
:105C4000D5A0AFE4DAA0ADE4B5F80900A4F85D0092
:105C5000B0FBF8F1DCA080E5697AA1F10A005A28CE
:105C600003D884F89310DDA077E5E5A0FCF722F8CF
:105C700084F893A0B9E3B5F8091040F6C412A1F571
:105C80007A70904205D8A4F8A610B1FBF8F1E2A012
:105C900063E5E9A061E5687A012808D084F8A8A046
:105CA00094F8A800012805D0EDA1EFA055E584F8EF
:105CB000A860F5E7F3A1F8E7B5F809004146B0FBA5
:105CC000F1F2B0FBF8F108FB1202A4F86300EFA0B8
:105CD000CCE2B5F8090000EB80010BEA4100414637
:105CE000B0FBF1F2B0FBF8F108FB1202A4F88E0051
:105CF000ECA0BBE2697AA4F84D10F1A02DE5697A19
:105D0000A4F84F10F4A028E5697AA4F85110F8A07F
:105D100023E5687A012809D084F892A094F89200CB
:105D2000012806D0AFF61011F7A016E584F89260AE
:105D3000F4E7AFF60811F7E71121F948F2F75CFA3A
:105D4000F74855F8091F953840F8951F6968416074
:105D5000298901810EE0CEE3D3E3D8E3DCE3E0E37D
:105D6000E4E3E8E3ECE3F0E3F0E3F0E3F0E3F0E3B3
:105D7000F0E3F0E3EBA00299EFE4E94855F8091FDE
:105D8000953840F89F1FA9888180A9798171EBA07F
:105D90000299E2E4687A012809D084F874A100BF6E
:105DA00094F87401012805D0ECA1EEA0D5E484F8A4
:105DB0007461F5E7F0A1F8E7B5F80910A1F130003A
:105DC000FC2806D201EB81010BEA4100A4F8750121
:105DD00002E0EDA0FBF76EFFB4F875114046B1FB91
:105DE000F0F208FB1212B1FBF8F1F0A03EE2B5F8B8
:105DF0000910A1F10B00592806D201EB81010BEA31
:105E00004100A4F8770102E0EFA0FBF753FFB4F8DC
:105E100077114046B1FBF0F208FB1212B1FBF8F12A
:105E2000F3A023E2697AA1F10B008B2802D2A4F837
:105E30007911ECE1E8E1B6E3B1E3BDE3F2E1F6E1CB
:105E4000FAE116E230E238E240E253E266E279E259
:105E500093E2AFE2C2E2DBE2EAE2F9E2FEE202E36F
:105E600007E30BE30FE313E317E31BE31FE323E372
:105E700027E32BE32FE333E337E30000546F746130
:105E80006C4361706163697479203A25642E2564DE
:105E900041480A0D00000000426D734D6178566F55
:105EA0006C743A25642E2564760A0D00754261747F
:105EB0004D617854656D70506C75733530203A259E
:105EC00064200A0D00000000754261744D696E5433
:105ED000656D70506C75733530203A2564200A0D5D
:105EE000000000007563426174547970653AC7A67A
:105EF000CBE1B5E7B3D8200A0D000000756342611D
:105F000074547970653AC4F8C7E2B5E7B3D8200A8B
:105F10000D0000007563426174547970653AC1D711
:105F2000CBE1CCFAEFAEB5E7B3D8200A0D00000004
:105F30007563426174547970653AC3CCCBE1EFAEBE
:105F4000B5E7B3D8200A0D007563426174547970C7
:105F5000653AEEDCCBE1EFAEB5E7B3D8200A0D0031
:105F60007563426174547970653AC8FDD4AAEFAE86
:105F7000B5E7B3D8200A0D00756342617454797097
:105F8000653ABEDBBACFCEEFEFAEC0EBD7D3B5E705
:105F9000B3D8200A0D000000756342617454797013
:105FA000653AEED1CBE1EFAEB5E7B3D8200A0D00EC
:105FB0007563426174547970653AC6E4CBFBB5E70A
:105FC000B3D8200A0D000000546F74616C566F6CDA
:105FD000746167653A256420200A0D005265717569
:105FE000697265566F6C746167654469666665724F
:105FF000656E63652825642956200A0D000000009F
:10600000202825642956206F7665722072616E679C
:1060100065200A0D0000000053696D756C617465A0
:106020006443757272656E74426174566F6C74204D
:106030002564560A0D00000053696D756C61746526
:106040006443757272656E74426174566F6C74202D
:106050002564562D2D3130302D333530560A0D0044
:10606000434C4F534500000025732044656275671B
:106070005F506167655F66756E6374696F6E200A55
:106080000D0000004F50454E000000007542617445
:106090004D6178456E65726779202564202E2564F0
:1060A000200A0D0053746F70566F6C746167652021
:1060B0003A25642E2564205620200A0D0000000099
:1060C0004F76657254656D703056616C75653A2512
:1060D0006420200A0D0000004F76657254656D70D3
:1060E0003156616C75653A256420200A0D00000068
:1060F0004F76657254656D703256616C75653A25E0
:106100006420200A0D0000005369676E616C4C6FBB
:106110007373466C616720257320200A0D00000010
:10612000B51500205665686963686C65496E666FD1
:1061300028302D39293A25730A0D00005665686903
:1061400063686C65496E666F2056494E2831302D64
:106150003137293A25730A0D000000006561737913
:1061600000000000576F726B4D6F64656C202573E3
:1061700020200A0D0000000070726F66657373695D
:106180006F6E616C00000000444352657175697266
:1061900065566F6C742025643A4F766572283438E2
:1061A0002D333030292020200A0D00004443526551
:1061B0007175697265566F6C743A25642E2564207A
:1061C0005620200A0D000000444352657175697223
:1061D0006543757272656E742564413A4F766572D7
:1061E0002831302D31303041292020200A0D000087
:1061F00044435265717569726543757272656E7458
:10620000256441200A0D0000ECA0FBF753FDB4F813
:1062100079114046B1FBF0F208FB1212B1FBF8F124
:10622000EEA023E0697A84F87B11F2A013E5697A85
:1062300084F87C11F5A00EE5B5F80910A1F1300045
:10624000CA2806D201EB81010BEA4100A4F87D01C6
:1062500002E0F3A0FBF72EFDB4F87D114046B1FB40
:10626000F0F208FB1212B1FBF8F1F6A0FBF722FDE9
:10627000BBE0B5F80910A1F114005A2806D201EBD1
:1062800081010BEA4100A4F87F0102E0F4A0FBF7D2
:1062900011FDB4F87F114046B1FBF0F208FB121279
:1062A000B1FBF8F1F7A0E1E7687A962801D284F80B
:1062B000810194F88111FAA0CDE4687A962801D280
:1062C00084F8820194F88211FBA0C4E4687A012862
:1062D0000AD084F890A100BF94F89001012806D05C
:1062E000AFF6CC61F9A0B6E484F89061F4E7AFF6BC
:1062F000C461F7E7687A01280AD084F887A100BF53
:1063000094F88701012806D0AFF6F461F5A0A2E465
:1063100084F88761F4E7AFF6EC61F7E7687A012863
:106320000AD084F888A100BF94F88801012806D01B
:10633000AFF61C71EFA08EE484F88861F4E7AFF645
:106340001471F7E7687A032804D884F889010128D2
:1063500003D005E084F889A147E0EBA0FBF7AAFC95
:1063600094F88901022802D1ECA0FBF7A3FC94F871
:106370008901032839D1EEA055E494F88901B5F8D4
:106380000950012803D12946EEA0FBF793FC94F8AD
:106390008901022803D12946F0A0FBF78BFC94F871
:1063A0008901032803D12946F2A0FBF783FCA4F856
:1063B0008A511AE0687A01280AD084F88CA100BFBB
:1063C00094F88C01012806D0AFF6B471EFA042E436
:1063D00084F88C61F4E7AFF6AC71F7E7687A0128CE
:1063E00008D002280AD003280DD089F800601BB01D
:1063F000BDE8F08F84F89761EBA014E4022084F8E4
:106400009701EEA00FE4032084F89701F0A00AE4BE
:10641000B5F80910A4F89811A1F1C902824205D279
:1064200001EB81020BEA4200A4F85900EDA012E44E
:10643000B5F80910A1F1C902824205D201EB81022F
:106440000BEA4200A4F85D00A4F89A11EDA00BE459
:10645000B5F80910A4F89C11F2A005E4B5F80910EC
:10646000A4F89E1103E0B5F80910A4F8A011F7A054
:106470000EE4B5F80910A4F8A2113AE0B5F8091035
:10648000A4F8A41135E0B5F80910A4F8A61130E07D
:10649000B5F80910A4F8A8112BE0B5F80910A4F874
:1064A000AA1126E0B5F80910A4F8AC1121E0B5F85E
:1064B0000910A4F8AE111CE0B5F80910A4F8B01149
:1064C00017E0B5F80910A4F8B21112E0B5F80910F8
:1064D000A4F8B4110DE0B5F80910A4F8B61108E05D
:1064E000B5F80910A4F8B81103E0B5F80910A4F83C
:1064F000BA11DEA007E4B5F80910A4F8BC11E3A0B6
:1065000006E4B5F80910A4F8BE11FEF7DBBFB5F834
:106510000910A4F8C011F8E7B5F80910A4F8C211E1
:10652000F3E7B5F80910A4F8C411EEE7B5F80910BF
:10653000A4F8C611E9E7B5F80910A4F8C811E4E712
:10654000B5F80910A4F8CA11DFE705E009E00DE08D
:1065500011E015E019E01DE0B5F80910A4F8CC1120
:10656000D3E7B5F80910A4F8CE11CEE7B5F80910B5
:10657000A4F8D011C9E7B5F80910A4F8D211C4E7FE
:10658000B5F80910A4F8D411BFE7B5F80910A4F8BC
:10659000D611BAE7B5F80910A4F8D811B5E788F80C
:1065A00004A0A0F802A051468246418000F050FBB2
:1065B0000027DFF8F0B2A0E1C1E1000044434D61E3
:1065C00078506F7765722564203A4F76657228316E
:1065D0002D31356B2909200A0D00000044434D611F
:1065E00078506F7765723A25642E2564206B7709A1
:1065F0000A0D000044435F496E64756374616E6305
:106600006554656D70202564200A0D0044435F4980
:1066100047425454656D70202564200A0D00000027
:1066200044434D6178566F6C74202564563A4F761A
:1066300065722834382D32303056292020200A0D3A
:106640000000000044432044434D6178566F6C7451
:106650003A25642E2564205620200A0D00000000F3
:1066600044432044434D617843757272656E7425CE
:10667000643A4F7665722832302D3131302920202E
:10668000200A0D0044432044434D617843757272E3
:10669000656E743A25642E2564204120200A0D0081
:1066A00043617061636974616E636554656D7031D7
:1066B000202564200A0D00004443426F7854656D24
:1066C0007032202564200A0D00000000446F7562BE
:1066D0006C65426174746572794D6F6465202573D1
:1066E0000A0D000056494E205472616E73202573C6
:1066F0000A0D0000426C75655369676E616C4C6FE2
:10670000737325730A0D00004368617267654D6FEE
:1067100064652D2D6B77680A0D0000004368617277
:1067200067654D6F64652D2D74696D650A0D0000F8
:106730004368617267654D6F64652D2D534F430A41
:106740000D0000004368617267654D6F64652D6BD5
:106750007768282564290A0D0000000043686172EB
:1067600067654D6F64652D74696D65282564290A18
:106770000D0000004368617267654D6F64652D53BD
:106780004F43282564290A0D0000000068696768E6
:1067900020766F6C74616765206D6F64756C652021
:1067A00025730A0D00000000536F6353696D756C0B
:1067B00061547970652D310A0D000000536F6353E9
:1067C000696D756C61547970652D320A0D00000099
:1067D000536F6353696D756C61547970652D330A1D
:1067E0000D0000000A0D20536F6353696D756C61D5
:1067F0004D6178566F6C7420202564205620200A45
:106800000D0000000A0D20536F6353696D756C61B4
:106810004D696E566F6C7420202564205620200A26
:106820000D0000000A0D20536F6343616C696272B2
:106830006174696F6E566F6C742020256420283057
:106840002E31295620200A0D000000000A0D205389
:106850006F6343616C6962726174696F6E566F6CCD
:106860007420202564205620200A0D00536F6343B6
:10687000616C6962726174696F6E566F6C7420200E
:106880002564205620200A0D00000000536F63434A
:10689000616C6962726174696F6E202025642020CA
:1068A0000A0D0000E4010020E819002690F8099084
:1068B0001BF8362049464A4519D10BEBC60828A0DB
:1068C00098F80120FBF7F6F9BAF8023004F1090054
:1068D000534498F801201844D8F80410F1F773FCD9
:1068E000BAF8021098F801000844AAF80200761CD1
:1068F000F6B2612EDCD37F1CFFB2A742D4D3BAF824
:106900000220A11C1144AAF8021041F20501AAF8C4
:106910000510E9798AF8071050468AF808400021E6
:1069200005E06A184318527A491C5A72C9B2A1424A
:10693000F7D317AA07A91348F4F704FC57E5E87939
:106940000128FBD184F8B9A078210F48F1F754FC55
:10695000F8F7A6FA0DA000E012A0FBF7ABF946E5A8
:106960007265616420706172616D2061646472207F
:106970003078257820706172616D206C656E2025FD
:10698000640A0D00221F0020DA150020526563659D
:10699000697665207265636F7264732061636B0A48
:1069A0000D000000526563656976652044434443E9
:1069B0002073746174652061636B0A0D0000000030
:1069C000418819B1806808B10020704701207047E4
:1069D00041880088814201D3012070470020704720
:1069E00010B50380002444808160828002FB031282
:1069F000C0E90321416110BD10B5044640880B4633
:106A000098B1A06888B1A28818466169F1F7DBFBEC
:106A1000A088616901446161E268914201D3A16883
:106A200061616188491E618010BD002010BD10B5F4
:106A3000044640882288904213D2A06888B1A28878
:106A40002069F1F7C0FBA188206908442061E16852
:106A5000884201D3A06820616088401C60800120CA
:106A600010BD002010BD000010B5F2F74BF90F4C1F
:106A700018B100206060012010BDF7F74DFD606087
:106A8000A1682731216088420ED309480078072881
:106A900008D0084800698047022803D00020E0732E
:106AA000022010BD0120FAE7002010BD282400209C
:106AB00060230020580000200168426809BA12BA19
:106AC000C0E9002170470168426809BA12BAC0E9FA
:106AD0000021704730B5044687B001210420F7F744
:106AE00035FC01214804F7F719FC0420ADF810002B
:106AF00003208DF812001820224D8DF8130004A9F0
:106B00002846F5F737F80820ADF8100048208DF832
:106B1000130004A92846F5F72DF826208DF8140057
:106B200001218DF815108DF816108DF8171005A895
:106B3000F6F718FC0020ADF804000094ADF806004C
:106B4000ADF80800ADF80C000C200F4CADF80A00B1
:106B500069462046FAF7D6F9012240F2255120462F
:106B6000FAF7B7F9012240F224412046FAF7B1F9C9
:106B700001212046FAF77DF980212046FAF770F9C5
:106B800007B030BD000801400044004070B5054624
:106B900086B001211120F7F7D9FB0121C804F7F7CE
:106BA000BDFB4FF48060ADF8100003248DF8124057
:106BB0001820244E8DF8130004A93046F4F7DAFFAC
:106BC000F014ADF8100048208DF8130004A93046E9
:106BD000F4F7D0FF34208DF814008DF815408DF8AF
:106BE000164001208DF8170005A8F6F7BBFB002022
:106BF000ADF80400ADF80600ADF80800ADF80C00E3
:106C00000C20114CADF80A00009569462046FAF7B1
:106C100079F901212046FAF72CF9012240F2255199
:106C20002046FAF756F9012240F226612046FAF78B
:106C300050F9012240F224412046FAF74AF906B001
:106C400070BD000000100140004C0040FDF788BFFF
:106C5000254810B5B0F859100A22B1FBF2F32349C8
:106C60000B80B0F85B30B3FBF2F34B80B0F88330AD
:106C7000B3FBF2F30B82B0F85330B3FBF2F30B83A8
:106C8000B0F88E30B3FBF2F38B82B0F88530B3FBF3
:106C9000F2F34B8290F88B30B3FBF2F38B7690F8E3
:106CA0008C30B3FBF2F3CB76B0F89030B3FBF2F359
:106CB000CB82B0F8B130B3FBF2F4B0F8B340B4FB20
:106CC000F2F4B3FBF2F2CC838A8390F8B620323A26
:106CD00081F8212090F8B520323A81F8202090F8F0
:106CE000790181F8220010BD20150020BC20002071
:106CF00070B5174E002500BF05EB450000EBC50041
:106D000006EB001494F8540003281BD394F8910068
:106D1000012803D122780421FCF78AFD94F8910020
:106D200002280FD194F8AC00401CC0B284F8AC002B
:106D3000022807D3032084F891002278042101203F
:106D4000FCF776FD6D1CEDB2022DD5D370BD0000B1
:106D50003C130020D8FF0000F8339F43D9FF000008
:106D600058699543DAFF0000BA298C43DBFF000025
:106D7000C77B8343DCFF000071BD7643DDFF00006D
:106D8000A09A6743DEFF000000805943DFFF000048
:106D9000E75B4C43E0FF0000E71B4043E1FF0000DE
:106DA0001BAF3443E2FF00005A042A43E3FF000014
:106DB0008B0C2043E4FF00001DBA1643E5FF0000E2
:106DC00042000E43E6FF0000B6D30543E7FF000094
:106DD0007B54FC42E8FF0000C3F5ED42E9FF0000F0
:106DE0005879E042EAFF000068D1D342EBFF00008F
:106DF000E6EEC742ECFF0000AFC5BC42EDFF00006D
:106E0000C749B242EEFF00002E70A842EFFF00001B
:106E1000B22E9F42F0FF0000C07B9642F1FF0000BF
:106E20008A4E8E42F2FF0000AB9E8642F3FF0000C6
:106E30009AC87E42F4FF000007307142F5FF00005F
:106E4000FE656442F6FF0000645D5842F7FF0000F3
:106E5000230A4D42F8FF0000C5604242F9FF0000DE
:106E60006D563842FAFF000048E12E42FBFF000059
:106E7000B5F72542FCFF000000911D42FDFF000018
:106E8000DDA41542FEFF00009F2B0E42FFFF000015
:106E9000011E0742000000005A7500420100000078
:106EA000A156F441020000005474E84103000000C0
:106EB0005238DD4104000000FC98D241050000007A
:106EC0004A8CC84106000000D509BF4107000000F8
:106ED000CE08B64108000000D881AD41090000008D
:106EE000916DA5410A00000039C59D410B000000CD
:106EF000758296410C0000008A9F8F410D000000B2
:106F0000F01689410E00000088E382410F00000066
:106F100069007A4110000000B7D16E4111000000F5
:106F20006132644112000000CE195A411300000082
:106F30006F815041140000007C6147411500000042
:106F400039B43E41160000001973364117000000A5
:106F5000F6972E41180000004F1E2741190000002F
:106F6000000020411A000000DA3819411B0000001F
:106F700028C412411C000000939D0C411D0000001C
:106F800020C106411E000000022B01411F0000002D
:106F900025AFF74020000000D786ED40210000001B
:106FA000A1D6E340220000009E98DA4023000000B2
:106FB000E7C6D14024000000145CC9402500000051
:106FC0001153C14026000000DFA6B9402700000091
:106FD000FC52B240280000001153AB4029000000D1
:106FE000DBA2A4402A000000963E9E402B00000039
:106FF0007D2298402C0000000A4B92402D0000009A
:10700000E1B48C402E000000E65C87402F000000B9
:1070100010408240300000002CB77A403100000060
:107020006059714032000000D061684033000000B8
:1070300092CB5F40340000001092574035000000B2
:10704000DEB04F4036000000E22348403700000029
:107050002EE740403800000027F739403900000093
:10706000DF4F33403A00000063EE2C403B0000004D
:107070006CCF26403C000000B3EF20403D000000F4
:10708000984C1B403E00000054E315403F000000B8
:107090001CB1104040000000D0B30B404100000084
:1070A000A7E8064042000000D34D02404300000024
:1070B000BEC1FB3F44000000FB3FF33F4500000022
:1070C0001B12EB3F460000002B35E33F470000005A
:1070D000E8A4DB3F480000005F5ED43F49000000A9
:1070E0004A5ECD3F4A000000B6A1C63F4B000000FB
:1070F0000326C03F4C0000003EE8B93F4D000000B1
:1071000075E5B33F4E000000041CAE3F4F00000089
:10711000A488A83F50000000062AA33F51000000A9
:1071200037FD9D3F520000009300993F530000003F
:107130002332943F54000000EF8F8F3F5500000032
:1071400001188B3F5600000008C9863F5700000019
:1071500062A1823F580000002D3E7D3F5900000093
:10716000AE81753F5A0000004E0B6E3F5B00000081
:107170001FD7663F5C0000002AE35F3F5D00000010
:10718000CF2C593F5E00000018B2523F5F00000054
:1071900065704C3F600000001765463F61000000CD
:1071A000DE8E403F620000001CEB3A3F63000000AF
:1071B000D977353F640000006E34303F6500000031
:1071C000931D2B3F66000000A032263F67000000A1
:1071D0009F71213F6800000040D91C3F69000000FA
:1071E0008C67183F6A000000331B143F6B000000DF
:1071F000E5F20F3F6C00000052ED0B3F6D00000008
:107200002D09083F6E000000CC45043F6F000000D0
:1072100038A1003F700000009335FA3E7100000075
:107220006362F33E720000008FC7EC3E7300000003
:107230007862E63E740000007F30E03E750000009A
:10724000A531DA3E76000000FA61D43E77000000F6
:107250007FC1CE3E78000000944DC93E7900000009
:107260003A06C43E7A00000082E7BE3E7B00000082
:107270006BF1B93E7C0000005721B53E7D00000057
:107280009678B03E00000000A9370108ED370108EC
:107290007D36010800000000000000000000000032
:1072A0000000000001000000A9370108ED370108C7
:1072B0007D36010800000000000000000000000012
:1072C0000000000030003000300030003000C60008
:1072D0004134305533300000000000000100000050
:1072E00040790108813B010801000000DC780108B9
:1072F0009F3C010801000000D47801089D3C010872
:107300000100000034790108A13C010801000000DF
:107310002C790108FD3C01080100000020790108DA
:10732000FB3C010801000000E4780108F93C010879
:107330000100000044790108353C0108010000000B
:10734000CC780108013D01080100000054790108D2
:10735000393C0108010000004C7901082D3B01086F
:1073600001000000BC780108A53C010801000000F4
:1073700068790108853B0108010000005C7901087B
:10738000D93B01080100000074790108C93A0108DD
:10739000010000000879010891D0000801000000F8
:1073A000F078010869D00008010000001479010894
:1073B00039D4000801000000FC78010881A8000809
:1073C00000C1814001C0804101C0804100C18140B5
:1073D00001C0804100C1814000C1814001C08041A5
:1073E00001C0804100C1814000C1814001C0804195
:1073F00000C1814001C0804101C0804100C1814085
:1074000001C0804100C1814000C1814001C0804174
:1074100000C1814001C0804101C0804100C1814064
:1074200000C1814001C0804101C0804100C1814054
:1074300001C0804100C1814000C1814001C0804144
:1074400001C0804100C1814000C1814001C0804134
:1074500000C1814001C0804101C0804100C1814024
:1074600000C1814001C0804101C0804100C1814014
:1074700001C0804100C1814000C1814001C0804104
:1074800000C1814001C0804101C0804100C18140F4
:1074900001C0804100C1814000C1814001C08041E4
:1074A00001C0804100C1814000C1814001C08041D4
:1074B00000C1814001C0804101C0804100C18140C4
:1074C00000C0C101C30302C2C60607C705C5C40484
:1074D000CC0C0DCD0FCFCE0E0ACACB0BC90908C8F4
:1074E000D81819D91BDBDA1A1EDEDF1FDD1D1CDCE4
:1074F00014D4D515D71716D6D21213D311D1D01054
:10750000F03031F133F3F23236F6F737F53534F443
:107510003CFCFD3DFF3F3EFEFA3A3BFB39F9F838B3
:1075200028E8E929EB2B2AEAEE2E2FEF2DEDEC2CA3
:10753000E42425E527E7E62622E2E323E12120E013
:10754000A06061A163A3A26266A6A767A56564A403
:107550006CACAD6DAF6F6EAEAA6A6BAB69A9A86873
:1075600078B8B979BB7B7ABABE7E7FBF7DBDBC7C63
:10757000B47475B577B7B67672B2B373B17170B0D3
:1075800050909151935352929656579755959454C3
:107590009C5C5D9D5F9F9E5E5A9A9B5B9959589833
:1075A000884849894B8B8A4A4E8E8F4F8D4D4C8C23
:1075B0004484854587474686824243834181804093
:1075C00000000000947D010801000000F87C010823
:1075D00002000000C87C010803000000747C010860
:1075E00004000000887C010805000000787E010886
:1075F00006000000307B0108070000001C7E010827
:10760000080000002C7E010809000000607C0108D1
:107610000A000000547B01080B000000A87B010851
:107620000C000000FC7B01080D0000009C7C0108A0
:107630000E000000A87C01080F000000447C010837
:1076400010000000107E010811000000347D0108C8
:10765000120000006C7D0108130000005C7D010831
:1076600014000000E47D010815000000D47D01082D
:1076700016000000F47D0108170000007C7D010861
:1076800018000000B07D010819000000487D0108C5
:107690001A000000B87C01081B000000047E0108ED
:1076A0001C000000607E01081D000000747B0108C2
:1076B0001E000000887B01081F0000009C7B010861
:1076C000200000003C7E0108210000006C7E0108C3
:1076D00022000000647B010824000000087C0108EF
:1076E00025000000147C010826000000247C01080D
:1076F000270000003C7B010828000000507C0108A6
:1077000029000000507E01082A000000E87C0108E2
:107710002B000000D47B01082C000000B87B01087E
:107720002D000000F07B01082E000000C47D010840
:107730002F000000347C010830000000087D0108A3
:10774000310000001C7D010832000000D87C0108D7
:1077500033000000A07D01080007070209030C02A6
:107760000E0200008711C1008793C2001617910016
:10777000171791008873C0000C401F000D401F00B8
:1077800000401F0001401F0002401F0003401F0077
:1077900004401F0005401F0006401F0007401F0057
:1077A00008401F0009401F000A401F0000008A0215
:1077B000020002007602B6030200050084034006C0
:1077C000020005000E063A07020005001C076009CA
:1077D0000200050000000E001A00260040004A00CA
:1077E00054006B0075008800CA00D400E000E4007B
:1077F000E800EC00F000F400F8000C0A0A18080891
:1078000015081140080A020202020202020087F172
:107810008AF197F189F189F093F195F180F190F176
:1078200010F08CF184F100A001A0802F812F822F15
:10783000832F842F90F110F08CF184F100A001A02F
:10784000812F822F832F0000130055005F006B00F3
:107850006F00730077007B001100400008000A00F1
:107860000200020002000200020010111419222E70
:10787000273E3128857F00000D0A37373755706461
:107880002D2D747970653A253078202C7665723A02
:107890002530782C54627974653A2530782C204351
:1078A00072633A2530782C5061673A2530782C5035
:1078B0006C656E3A2530780D0A0000005265616CE7
:1078C0007948696768343030000000004B43353632
:1078D000000000004F464644434443004F4E44439B
:1078E0004443000053455441504E5057440000005B
:1078F00041435F7245634C4F53450000414352651D
:107900006C61794F4646000041435F72454F5045D8
:107910004E000000414352656C61794F4E000000FB
:1079200053455441504E555345520000544553540D
:10793000424D5300524541444D4153530000000015
:1079400053455400526573657400000041436375EC
:1079500074000000444363757400000043433243E5
:10796000435265616C790000434331435052656175
:107970006C79000047554E54656D705265616C79A5
:107980000000000052657365727665643100000086
:1079900048414E440000000049444C4500000000AE
:1079A00052554E4E494E470053544F500000000070
:1079B000494E495400000000535441525400000005
:1079C0006368617267655F4D6F64655F3132560051
:1079D00052454144590000005265736572766564F2
:1079E000000000005265736572766174696F6E5FA6
:1079F00041435F6368617267655F6D6F6465000036
:107A000044435F6368617267655F6D6F6465000022
:107A100041435F6469736368617267655F6D6F643A
:107A20006500000044435F64697363686172676561
:107A30005F6D6F64650000004E6F726D616C5F6D0D
:107A40006F64650052656D6F74655F636F6E74720D
:107A50006F6C5F6D6F6465006368617267655F621C
:107A60006174746572795F686561745F6D6F646578
:107A70000000000052656D6F74655F62617474652B
:107A800072795F686561745F6D6F64650000000006
:107A900044656661756C745F6D6F6465000000001D
:107AA00041435F4368617267696E670044435F43A7
:107AB00068617267696E670041435F43686172671E
:107AC000000000004E6F726D616C5F4F70657261F7
:107AD00074696F6E0000000041435F636861726704
:107AE000655F636F6E6E65637400000041435F64A1
:107AF00069736368617267655F636F6E6E656374F7
:107B00000000000048616C665F636F6E6E656374B1
:107B1000000000004E6F5F636F6E6E65637400005F
:107B2000436F6E6E6563745F4661756C7400000030
:107B3000534F43203130302500000000B3E4B5E757
:107B4000D7AED6D0D6B9B1A8CEC428C6FAD3C329E9
:107B500000000000B3E4B5E7D0E8C7F3B5E7D1B95A
:107B6000CEAA3000564355B9A4D7F7C4A3CABDD294
:107B7000ECB3A300424D53C8C8B9DCC0EDBCD3C8B8
:107B8000C8D2ECB3A3000000424D53C8C8B9DCC052
:107B9000EDD6C6C0E4D2ECB3A3000000424D53BE04
:107BA000F9BAE2CAA7D0A700B5E7B3D8B8DFCEC20A
:107BB000D4A4BEAF00000000B3B5D4D8B4A2C4DCD6
:107BC000D7B0D6C3C0E0D0CDC7B7D1B9B1A8BEAF8A
:107BD00000000000B3B5D4D8B4A2C4DCD7B0D6C37B
:107BE000C0E0D0CDB9FDD1B9B1A8BEAF0000000052
:107BF000534F43B5CDB1A8BEAF000000534F43B9BA
:107C0000FDB8DFB1A8BEAF00424D53CDA8D1B6B389
:107C1000ACCAB100B3E4B5E7D7AECDA8D1B6B3AC2A
:107C2000CAB10000B3B5C1BECEB4C9CFB8DFD1B9B7
:107C300000000000B3E4B5E7D7AED6D0D6B9B1A8FE
:107C4000CEC40000424D53C4DAB2BFCDA8D0C500A7
:107C5000434D4C20B2CECAFDB2BBBACFCACA000057
:107C6000B3E4B5E7B5E7C1F7D0E8C7F3B9FDB5CDE3
:107C700000000000D6B1C1F7BCCCB5E7C6F7D5B35C
:107C8000C1ACB9CAD5CF0000BDBBC1F7BCCCB5E70C
:107C9000C6F7D5B3C1ACB9CAD5CF0000424D53C564
:107CA000F6D7B2B9CAD5CF00424D53C4DAB2BFBE7F
:107CB000F8D4B5B9CAD5CF00424D53CDE2B2BFBE5C
:107CC000F8D4B5B9CAD5CF00CAE4C8EBC7B7D1B9A3
:107CD000B9CAD5CF000000004B4C3330B8DFD1B962
:107CE000D1B9B9CAD5CF00004B4C3330B5CDD1B9DD
:107CF000B9CAD5CF00000000CAE4C8EBB9FDD1B9BC
:107D0000B9CAD5CF00000000B0E5D4D8CEC2B6C8FD
:107D1000B9FDB8DFB9CAD5CF00000000D6B1C1F7B0
:107D2000C7B9D7F9CEC2B6C8B9FDB8DFB9CAD5CF81
:107D300000000000424D53D7DCB5E7D1B9BCECB22E
:107D4000E2B9CAD5CF000000B5A5CCE5B5E7D1B9F9
:107D5000BCECB2E2B9CAD5CF00000000424D53CE10
:107D6000C2B6C8BCECB2E2B9CAD5CF00424D53B5D9
:107D7000E7C1F7BCECB2E2B9CAD5CF00B3B5D4D8ED
:107D8000B4A2C4DCD7B0D6C3B9FDB3E4B9CAD5CF69
:107D900000000000CEB4B6A8D2E5B9CAD5CF000025
:107DA000B3ACB3F6B6A8D2E5B9CAD5CF000000008F
:107DB000BDBBC1F7B3E4B5E7BFDACBF8BDF4B9CAD0
:107DC000D5CF0000B3E4B5E7B9FDC1F7B9CAD5CF47
:107DD00000000000B8BABCABBDD3B4A5C6F7B9CAA1
:107DE000D5CF0000D5FDBCABBDD3B4A5C6F7B9CA8D
:107DF000D5CF0000D4A4B3E4BDD3B4A5C6F7B9CAA7
:107E0000D5CF0000B5E7B3D8C8C8CAA7BFD800000F
:107E1000424D53D4A4B3E4CAA7B0DC00B5A5CCE569
:107E2000B5E7D1B9B9FDB8DF00000000B5E7D0BEB5
:107E3000CEC2B6C8B9FDB8DF00000000B5A5CCE5DC
:107E4000B5E7B3D8C7B7D1B9BEAFB8E600000000F8
:107E500043435320BDFBD6B9B3E4B5E700000000AF
:107E6000424D53BDFBD6B9B3E4B5E700564355BD0B
:107E7000FBD6B9B3E4B5E700CAE4C8EBB9FDC1F776
:107E8000000000004B433100595831004B43320091
:107E90005958320048565F4453475F434845434A68
:107EA0005F3200004B4333004B4335004B433800F7
:107EB0004B43390043414E315F53544200000000B0
:107EC00043414E325F53544200000000454C535F23
:107ED0004F46460048565F4453475F434845434A30
:107EE0000000000043414E325F454E00454C535F59
:107EF0004F4E00004D43555F52554E005057335F73
:107F0000335600005057355600000000434F4E478F
:107F10005F525800434F4E475F5458003C7F010862
:107F200000000020180C00006C8A0008048501087D
:107F3000180C0020687B0000B81D01088133E8039D
:107F400084A24A0440090102030406070809023713
:107F5000A61391C41408F5BF140831C31B08AD0C57
:107F60001389A414081DEF1408CDBC140839D202DB
:107F70001D08023A01180A894701087F460108CD09
:107F8000041AD1041A0910411A14E4B26429F49AAB
:107F9000F46800091CD5FBB3B5D0ADD2E963030A80
:107FA00008092AFD350108313601083401484BFF24
:107FB000FFBC01281A02E413EC045B2001085A03F9
:107FC000082305101340151B2004081A3008230647
:107FD000021A6D081A07081A89081A08281A8B0845
:107FE0001A09201A20081A0A101AA7081A0F081AC4
:107FF000AC081A0E081AAB081A0D081AAA081A0CAF
:10800000081AA9085A0B601A13481A7B101A12088A
:108010001A79081A11081AA5081A10081AA3081ABA
:10802000140829281A16081A83101A18381AD008A2
:108030001A1F0813D2201B201E081AD4081A1D0864
:108040001AAD181A20081ADA101A21081AD8081AB4
:1080500022081AD7185A24601A23081A7F085A27A8
:10806000481A26081ADD281A25081ADC081A2820BA
:108070001A7D181A29101AB3081A2A101AC6081AD3
:108080002B101AC8085A30881A31081AD0301A3200
:10809000181A6D101A33081A6F081A34081A710862
:1080A0001A35081AB20823360A1AB5082337071AF0
:1080B000BF081A50181394161B2051401A95081A1D
:1080C00052081A97081A53181A99081A54081A9B32
:1080D000081A55081A9C081A56201A9D081A57089B
:1080E0001A9F081A58181AA1081A59081AA2081A29
:1080F0005A081AB0081A60081AA7081A61081AA8BC
:10810000081A62081AA9081A63381AAA081A651008
:108110001AAC081A66081AAD081A6D081AB7081AB8
:108120006E201AB8081A6F081ABA081A70081ABC12
:10813000081A71081ABE081A72081AC0081A7308B9
:108140001AC2081A74081AC4081A75081AC6081A36
:1081500076081AC8081A77081ACA081A78081ACCB2
:10816000081A79081ACE081A7A081AD0081A7B0851
:108170001AD2081A7C081AD4081A7D081AD6081AC6
:108180007E081AD8081A7F081ADA081A80081ADC3A
:10819000081A81081ADE081A82081AE0081A8308E9
:1081A0001AE2081A84081AE4081A85081AE6081A56
:1081B00086081AE8081A87081AEA081A88081AECC2
:1081C000081A89081AEE081A8A081AF0081A8B0881
:1081D0001AF2081A8C081AF4081A8D081AF6081AE6
:1081E0008E081AF8081A8F081AFA08814502040640
:1081F000082D0102030404200B0607080971290158
:10820000080401130DD51B0809081A55082331036A
:1082100013D9DA1B0857081A8D101A58081AD108F2
:108220001A59081311D61B085D081A49081A5F0865
:108230001A6908239B051A89081AE6101AA9082A40
:10824000E72812D71B0880181A39081A1158130585
:10825000DB640827046334075ADF08811FF14301F8
:1082600008B9A56812A639A8811AF7181AD514DA20
:1082700025181A67185AED189A411C1AFD1813018F
:10828000A71B088504A91C1E3544010821141AE9FE
:10829000641AFD04291829201A2D181A35181A7184
:1082A000049A11481E2D450108491401101A6160F5
:1082B000DA958C411AF5181AFB042A6D8019541AA4
:1082C00039042A310419481A65141B854018180905
:1082D000410108F53F010845081E45420108D9083B
:1082E0001A2D1C1A9914B96412EB140823C31B0825
:1082F0008908139DC41B083D0813F1BF1B084908DA
:108300001A15181A31081AED1001701394068220FC
:108310001EC47A0108A0041AAC041E98790108B0A2
:10832000041A90041AD0041AB8041AA0042AA80C3B
:1083300019201E147B010804041AD80C1AEC041A24
:10834000200C2A8430190C1A38041AF00C1A100860
:108350001119041A24041AE4101AC0041A440C1A3D
:1083600058041A74041AD81072281387BC73083280
:108370008B8DCB0C1A6D0C720A1331B07308051378
:10838000C38A6B0814248AC70C9A690C8B05AA0C43
:1083900013E5D402180813E1D11B089F041AC9047D
:1083A0003925440C01409A010C9A020C118A800C68
:1083B00039055A0818290669249A0418293D690CB8
:1083C000293C3C100140502912690C2905593C5A9E
:1083D000106C398029051924390C2924190C5129CC
:1083E0001159549A209C29776954494D490C3918E0
:1083F0005A143C29616948011713A1CF14083C089D
:108400001B2048041350091F20847E0108FC081A11
:108410008C0813080A1B20A4081A14081AA8081AA2
:1084200020081AAC081A2C081AB0081A38081E04BA
:108430007F010844081AF4101A50081A88081A5CB8
:10844000081A90081A68081AFC081A74081AC00852
:108450001A80081AE4081A8C081AEC081A98081AE4
:10846000CC081AA4081AB4081AB0081AD4081ABCFE
:10847000081A94081AC8081A0C601AD4081A1408A2
:108480004BF5D0AC1A5404690C9A600C9A6C0C9A97
:10849000780C9A840C1A90044B55D10C1A9C044BFE
:1084A00009D20C9AA80C9AB4309AC00C9ACC0C9AA7
:1084B000D80C9AE40C9AF00C1AFC045AB90C8B08EC
:1084C000090C1A140C69249A200C1A2C0C01340380
:1084D00016F40102631F022F02123D1C01086D04F5
:1084E0001A91041AC5041AE5041E85010108050441
:1084F0001AED041AB9041A51041B11021C04280AAB
:04850000010800006E
:04000005080081511D
:00000001FF
